:020000040000FA
:10800000805C0020D5800000F1800000BB5801009A
:108010000000000000000000000000000000000060
:10802000000000000000000000000000F5800000DB
:108030000000000000000000F7800000211702008F
:10804000FB800000FB80000079CE010085CE01009E
:1080500021C60000351D020095220200A122020067
:108060009D6B0100A56B0100BDEB0100C5EB01009C
:108070002D590100355901001D1D0200251D02006A
:108080002D1D02006F6A01003D1D0200451D02000A
:108090004D1D020069CE010081480200D1DE0100C1
:1080A000DB8C000071CE01006948020071480200BB
:1080B000CB6C0100676A01004DD300006DBA00006F
:1080C0000348854600F0C0FD00480047CD8C000005
:1080D000805C002009480A4A002100A1814200D9A1
:1080E00002440848084A0260084880470848004798
:1080F000FEE7FEE7FEE7FEE7FEE7FEE70000002002
:108100000000000008ED00E000800000451C0200B7
:10811000C180000030B50B4601460020202201241A
:1081200009E00D46D5409D4205D31D469540491BAB
:108130002546954040191546521E002DF1DC30BDF4
:1081400070B500242546002801DA012440420029A8
:1081500001DA01254942FFF7DDFFAC4200D0404281
:10816000002C00D0494270BDF0B51FB40646002077
:1081700082B005464024019100901BE001992246FF
:108180000F46304600F05AFC049A059B801A99412C
:1081900010D310461946224600F040FC361A8F4193
:1081A0000197224601200021009F00F037FC38187B
:1081B0004D4100902046641E0028DFDC019B0098A2
:1081C0002946324607B0F0BD38B50446C0681821CC
:1081D000401E4843A16840183C214843616840184C
:1081E0003C2148432168451860690C2148432169B6
:1081F00040186921C900401A3021FFF7A1FF114A38
:1082000050434219084600921A2902DB0E495118C0
:1082100000910C21FFF794FF0C4A5043009A8018FC
:1082200000900B4806E0491E425C074B5A43009BF6
:10823000D21800920029F6DC2146684600F02AFC9C
:10824000009838BD801F8607805101008033E1010E
:1082500098DB020003460B439B0703D009E008C9E3
:10826000121F08C0042AFAD203E00B780370401CE6
:10827000491C521EF9D27047D2B201E00270401C74
:10828000491EFBD270470022F6E710B513460A4696
:1082900004461946FFF7F0FF204610BD421E5378F2
:1082A000521C002BFBD10B781370491C521C002B65
:1082B000F9D17047421C0178401C0029FBD1801A7B
:1082C000704703460A780270401C491C002AF9D105
:1082D000184670470321001D401E037812021A43FE
:1082E000491EF9D510467047034610B508330722DA
:1082F000040E090221435B1E1C7800022043521E1B
:10830000F6D510BD034603220870000A491C521E10
:10831000FAD51846704770B504460D46072310700D
:108320000E06000A3043090A521C5B1EF7D5204690
:10833000294670BDF8B502464A40D40F42004B00B2
:1083400052085B089A4202D20246084611464A0089
:1083500023D0C30D4A00DDB2120EAD1A202D35DA3E
:1083600049020126490AF6058A19002C00D052421A
:1083700020214F1B1146B9402A411018C20D9A42C4
:1083800021D0002C17D0012D08DCDA05801AD20F7D
:108390008019D207DBB200F0BFFBF8BDDA05801A06
:1083A000012340001B06C01880185A428018CA0FCB
:1083B0001043490007E04908C2071143DA05801A53
:1083C00080194008801800F09FFBF8BD6100012271
:1083D000511A001BF7E70122D2075140AAE70122F8
:1083E000D2075040A6E7024670B54A40D30FDB07DC
:1083F00040002DD04A002AD0010E140E00021202B5
:108400000919400A520A8418E50104465443000A37
:10841000120A2E045043A4194219200CC543AA186D
:10842000120C0125AD03521C521912047F39240489
:1084300000D0521C104301D44000491EC2B20C06A9
:10844000C0092018401C4008802A02D003E0002008
:1084500070BD40084000002900DA0020184370BDBC
:1084600070B502464A40D50F40004A00ED0740086B
:108470005208002814D0002A12D0C40DD30D410296
:108480000120C0055202490A520AE41A09181218BA
:108490007D34914201D3641C00E04900002C01DAD4
:1084A000002070BD0023914201D3891A0343400884
:1084B00049000028F7D100290AD0914202D10121B8
:1084C000C90705E0914201D2012101E00121C94320
:1084D000E005C018401900F017FB70BDF0B5074665
:1084E0000846584087B0C00F049048000E46590017
:1084F00040084908BC1A884105D2384631461E4614
:1085000017460B4602465800400810434CD0300D29
:10851000039040055900400D490D0590401A029006
:10852000402872DA18030121000B09050843019065
:1085300004980092002805D00199524200208841F9
:1085400000920190029840210A1A0199009800F0C7
:1085500065FA05460C466B4607CB00F080FAC01959
:108560007141039A0E0D0023D71756401A467A40E0
:10857000164344D0049A002A2DD0029A012A039A65
:1085800015DC1205C01A914101263605001C714107
:10859000D20F059ED2070093019202962A462346E7
:1085A00000F000FB07B0F0BD38463146FAE716058B
:1085B000224A0F46B218C01AB74101210905001C12
:1085C0004F4100187F41114618187941E20F1043BE
:1085D0006D19644113E0E2076D0815436408C20792
:1085E0001443039A01261205C01A91413605001C56
:1085F0007141CE07400830434908C01851412A460E
:10860000234600F0C2FACDE7FFE7049801224000BC
:10861000C117121A00238B4104983146C417381A27
:10862000A141EEE730B40124E407634030BC55E7D4
:1086300030B40124E407614030BC4FE70000E0FFA4
:10864000F0B51FB488B00B990998002448400999E7
:10865000C00F490049080991C0070B9900904900D3
:1086600049080B9109990898A64608431CD00B9914
:108670000A98084318D0099801244000420D480088
:10868000410D099824050003000B204309900B9825
:108690000003000B20430B9050181C494018002287
:1086A00001901446104605E0002001460DB0F0BDD3
:1086B000032801DA034600E003239C46C11A0AAEF0
:1086C0000AE05F0008ADED5B4F00F75B7D430027DC
:1086D000AA187C41491C5B1E6145F2DD410004ABD8
:1086E0005A522104120C0A43240C401C0828DFDBD8
:1086F000019802900099704601910090059B049AA0
:108700000799069800F04EFAD0E700000DFCFFFF35
:10871000F0B50C465C4085B0E40FE40703944C00D0
:1087200000266408590094464908024602962243EE
:1087300021D062460A431ED06200570D4A000E0344
:108740002303550D012402462C492405781B1B0BDD
:10875000360B401823432643614600901C46501AAE
:10876000B44103D30098401C009002E09218009896
:108770005B41002803DA0020014605B0F0BD00206F
:10878000012109050746864611E064461D46141B73
:10879000B54106D36546521BB341744607430C43AB
:1087A000A646CD0740084908284392185B41054674
:1087B0000D43EAD11046184313D060461946504085
:1087C0007140084306D06046101AB34106D2012218
:1087D000002306E000220123DB0702E00122D2434E
:1087E0005310009874460105381C6141029C039D9A
:1087F0000019694100F0C9F9BFE70000FD0300005E
:10880000C217C10F504010B54018CA079623002167
:1088100000F082F910BD10B500229623114600F039
:108820007BF910BD0EB5C217C10F5040CA074018E2
:108830000021054B0293019200910A460B4600F07D
:10884000B1F903B000BD0000330400000EB50549C6
:108850000291002100910A460B46019100F0A2F915
:1088600003B000BD33040000410040020122400A71
:10887000D205090E80187F2901DA00207047962959
:1088800003DC9622511AC8407047963988407047D9
:1088900041000A0E40020121400AC90510B54018E6
:1088A0007F2A02DA0020014610BD0021962A03DC4F
:1088B00096239A1AD04010BD963A00F0AFF810BD3A
:1088C00070B5CD0F4A0009030123090B1B0519439D
:1088D0000B4BED070024520D9A4201DA002070BDC7
:1088E000074B34339A4203DC9A1A00F0A7F802E0EF
:1088F0000449511888402C43F1D0404270BD00001B
:10890000FF030000CDFBFFFF4A0009030123090B11
:108910001B051943094B10B5520D9A4201DA00208C
:1089200010BD064B34339A4203DC9A1A00F086F8E5
:1089300010BD03495118884010BD0000FF0300001E
:10894000CDFBFFFFC20FD207400040080BD0C10D86
:108950000723DB01C91840020905400A1143C20878
:1089600040071143704700200146704710B50029A9
:1089700004DB0124E40740428C412146002B04DB48
:108980001C460123DB075242A3418B4200D18242A5
:1089900010BD000010B5002904DB0124E4074042AB
:1089A0008C412146002B04DB1C460123DB0752428D
:1089B000A341994200D1904210BD0000CB0FDB07CC
:1089C000490010B5490802460A4307D00A0D07249A
:1089D0000903E401090B121B002A01DC002010BD71
:1089E000C900440F0C43C100E018D205801800F004
:1089F0008BF810BD0122D207002800DB101A0029D5
:108A000000DB511A814270470122D207002800DBA7
:108A1000101A002900DB511A8842704710B5202A2D
:108A200004DB0146203A9140002010BD91402023F4
:108A30009C1A0346E3401943904010BD10B5202A0C
:108A400004DB0846203AD040002110BD0B46D3403D
:108A5000D0402024A21A91400843194610BD10B5F9
:108A6000202A06DBCB170846203A1041C1170B43DA
:108A700006E00B461341D0402024A21A914008433F
:108A8000194610BD10B5024900F004F810BD0000F1
:108A9000544C002070B50C4600683C21FFF73AFBAF
:108AA00021603C21FFF736FB61601821FFF732FBA4
:108AB0000546A1600721001DFFF72CFBA1610F48AF
:108AC000A90008180E49FFF725FB02464432880822
:108AD0006261E0613B2802D3910700D0401C002175
:108AE000084B0A462161995C814203D8401A521C06
:108AF0002261F8E7401CE060204670BD6C0B00006E
:108B0000B5050000A4DB0200002904DA401C49007E
:108B100001D140084000704770B40024050C05D115
:108B20001024000402D1002921D01124050E01D106
:108B300000020834050F01D10001241D850F01D169
:108B40008000A41C002801DB4000641C002908D020
:108B500020252E1B0D46F540A14000D001212943C0
:108B6000084301061B1B000ADB1D02D5002070BC58
:108B70007047DB05181880180029F8DA401C4900F6
:108B8000F5D170BC40084000704710B5002B08DAE2
:108B90000024401C614192185B411A4301D14008F6
:108BA000400010BDF0B51FB482B005460C0003D0E4
:108BB00008461BF0DDFF02E01BF0DAFF2030024622
:108BC000009021462846FFF729FF049B059A04469A
:108BD0000F4618431143084314D0184610431BD0C6
:108BE000009840210A1A18460599FFF727FF054605
:108BF0000E46009A05990498FFF710FF084305D028
:108C0000012004E02046394607B0F0BD0020C1171E
:108C100005430E432C43374300990E986305401AD1
:108C20007905E40A00220C43FD0A0A3002D500202F
:108C30000146E9E70105101969410C9C0D9D0019D9
:108C40006941FFF7A2FFDFE7064C0125064E05E06C
:108C5000E36807CC2B430C3C98471034B442F7D35D
:108C6000FFF732FAB0DD0200D0DD020070B58D18DA
:108C70000478401CA207920F01D10278401C2311F6
:108C800006D10378401C03E006780E70401C491C96
:108C9000521EF9D1002B15D002780C268A1A3440C6
:108CA000401C0C2C03D0A401121B9B1C08E0047870
:108CB0002402121B401CF8E714780C70491C521C4B
:108CC0005B1EF9D5A942D3D3002070BD10B518F0B2
:108CD000B9FF22F01FFF002010BD10B5C046C046EE
:108CE000C046C04610BDF7B58AB00D460595059D36
:108CF0002846E917090F09180905090E04910027EC
:108D000028E0002407E0380101190A98405C694610
:108D10000855601CC4B2102CF5DB002605E00C9849
:108D2000805D06A98855701CC6B2102EF7DB0122A3
:108D300006A968461CF04AF8002407E06846015D71
:108D4000380102190A988154601CC4B2102CF5DB5A
:108D5000781CC7B204988742D3DB0DB0F0BDFFB5D5
:108D60008DB014460D98002802D0012854D154E04B
:108D700025462C462046E917090F09180911491CF8
:108D800009050E0C301BC0B2089008980790E8B295
:108D9000069007E0069A0E99079888540698401C9A
:108DA000C0B206900698B042F4DB002005902CE09B
:108DB000002708E005980001C1190E98405C01A940
:108DC000C855781CC7B2102FF4DB002705E01098B7
:108DD000C05D09A9C855781CC7B2102FF7DB002267
:108DE00009A901A81BF0F2FF002708E001A8C15D56
:108DF00005980001C2190E988154781CC7B2102F33
:108E0000F4DB0598401CC0B20590F117090F8919D1
:108E10000A1105998A42CBDC53E025462C462046B0
:108E2000E917090F09180911491C09050E0C301B17
:108E3000C0B2089008980790069507E0069A0E9928
:108E4000079888540698401C80B206900698B04255
:108E5000F4DB002005902CE0002708E005980001D5
:108E6000C1190E98405C01A9C855781CC7B2102FD3
:108E7000F4DB002705E01098C05D09A9C855781CEF
:108E8000C7B2102FF7DB002209A901A81BF09EFF33
:108E9000002708E001A8C15D05980001C2190E98DD
:108EA0008154781CC7B2102FF4DB0598401CC0B267
:108EB0000590F117090F89190A1105998A42CBDC2F
:108EC00000BF00BF11B0F0BD10B5044645480078A2
:108ED0000A3803001BF063FE0B070D17212B353FEB
:108EE00049535F697F002B2C02D10B203D4908704C
:108EF00075E0432C03D10C203A49087002E00A20A7
:108F0000384908706BE0452C03D10D2035490870B5
:108F100002E00A203349087061E0522C03D10E2090
:108F20003049087002E00A202E49087057E0452CAD
:108F300003D10F202B49087002E00A20294908704C
:108F40004DE0472C03D110202649087002E00A208A
:108F50002449087043E03A2C03D1112021490870BC
:108F600002E00A201F49087039E0202C03D11220AA
:108F70001C49087002E00A201A4908702FE0302CC2
:108F800005DB332C03DC13201649087002E00A20AD
:108F90001449087023E02C2C03D1142011490870C7
:108FA00002E00A200F49087019E020463038C1B2AB
:108FB000012023F0A3FC312C01D0352C07D1032054
:108FC000C0430949087500200649087002E00A20DC
:108FD0000449087003E00A200249087000BF00BF7E
:108FE00010BD00006C0E0020133A002010B504469E
:108FF000384800780A3803001BF0D1FD09060C162A
:10900000202A343E485266002B2C02D10B203149D5
:1090100008705DE0432C03D10C202E49087002E05B
:109020000A202C49087053E0472C03D10D20294910
:10903000087002E00A202749087049E0412C03D15A
:109040000E202449087002E00A20224908703FE0FF
:10905000542C03D10F201F49087002E00A201D493B
:10906000087035E0542C03D110201A49087002E032
:109070000A20184908702BE03A2C03D11120154919
:10908000087002E00A201349087021E0202C03D167
:1090900012201049087002E00A200E49087017E0FB
:1090A00020463038C1B2022023F028FC312C07D1F1
:1090B0000320C0430849087500200649087002E0F3
:1090C0000A200449087003E00A200249087000BF22
:1090D00000BF10BD6C0E0020133A00202B49097808
:1090E0000A2902D00B2944D112E00021284A11702C
:1090F00030280CDB39280ADC11460A780978491C2B
:10910000234B1970234988540B21204A11703AE0EF
:1091100030280ADB392808DC1D490A780978491CFF
:109120001B4B19701B49885422E04B280DD100219C
:10913000174A117000221749CA730A21134A117085
:109140000321C943144A117512E0114909780F2906
:1091500004DB0321C943104A117503E00221C9430E
:109160000D4A117500220B49CA730A21074A117072
:1091700009E00A21054A11700021054A1170C91E33
:10918000054A117500BF00BF704700006C0E00203B
:10919000A30E00201C2F0020133A002070B50446B7
:1091A000B24800780A3803001BF0F9FC2C171D2781
:1091B000313B455B6597A1ABB5BBC9E0F8FEEDEC73
:1091C000EBEAEAEAEAEAEAEAEAEAEAEAEAEAEAEAFE
:1091D000EAEAEAEAEA6F79838DEA2B2C02D10B20C6
:1091E000A24908703FE14D2C03D10C209F49087023
:1091F00002E00A209D49087035E1492C03D10D2079
:109200009A49087002E00A20984908702BE1502C16
:1092100003D10E209549087002E00A209349087096
:1092200021E14C2C03D10F209049087002E00A2064
:109230008E49087017E1572C06D100218C488172A5
:1092400010208A4908700BE0452C06D1012188487E
:10925000817232208549087002E00A208349087033
:1092600001E1522C03D111208049087002E00A204C
:109270007E490870F7E0492C03D112207B49087021
:1092800002E00A2079490870EDE0582C03D1332020
:109290007649087002E00A2074490870E3E0452C22
:1092A00003D134207149087002E00A207149087026
:1092B000D9E0432C03D135206C49087002E00A2024
:1092C0006A490870CFE0552C03D112206749087015
:1092D00002E00A2065490870C5E0542C03D1132030
:1092E0006249087002E00A2060490870BBE0452C22
:1092F00003D114205D49087002E00A205B49087020
:10930000B1E03A2C03D115205849087002E00A2038
:1093100056490870A7E0302C02D116205349087036
:10932000A1E02C2C0AD11720504908700020504988
:1093300088710A214E48001FFEF7A5FF93E02C2CF0
:1093400010D0302C11DB392C0FDC494880790928EA
:109350000BDA474881798079401C454A9071101F8B
:10936000445402E01820414908707CE02C2C14D1B0
:109370003F48807A002809D119203C4908700CE048
:1093800070E027E01CE015E00EE007E03848807A46
:10939000012802D11A203549087064E02C2C02D132
:1093A0001A20324908705EE02C2C02D11B202F4974
:1093B000087058E02C2C02D11C202C49087052E077
:1093C0002C2C06D11D202949087000212A488172C1
:1093D000C17248E02C2C3BD00D2C39D02649C87ADC
:1093E000897A0002084301218902884228DA20484C
:1093F0000838FEF76FFF451C1D4908392846FEF75F
:1094000081FF302C01DB392C07DD412C01DB462CA0
:1094100003DD612C25DB662C23DC1748C17A807ABA
:1094200009020143144AD07A927A00021043401C88
:1094300082B211488272120AC2720C30445410E097
:1094400000210D488172C1720A200849087008E0A5
:1094500000200749487201202039C8750A200349B5
:10946000087000E000BF00BF70BD0000B10E00201A
:10947000333A00206C0E00201334002000B52F4931
:1094800009780A390B001BF08AFB08050B151F2908
:10949000333D47522B2802D10B21284A11704AE054
:1094A000432803D10C21254A117002E00A21234AE6
:1094B000117040E0532803D10D21204A117002E0C1
:1094C0000A211E4A117036E0432803D10E211B4A9F
:1094D000117002E00A21194A11702CE04F2803D1C3
:1094E0000F21164A117002E00A21144A117022E07D
:1094F0004E2803D11021114A117002E00A210F4AAF
:10950000117018E0202803D111210C4A117002E0DB
:109510000A210A4A11700EE0312804D10321C943FF
:10952000074A117502E00A21044A117003E00A217A
:10953000024A117000BF00BF00BD00006C0E002089
:10954000133A002000B5424909780A390B001BF094
:1095500026FB0A06101A242E38424A5D6A782B2808
:1095600003D10B213A4A117002E00A21384A1170E6
:109570006BE0432803D10C21354A117002E00A2127
:10958000334A117061E0532803D10D21304A117024
:1095900002E00A212E4A117057E0512803D10E2112
:1095A0002B4A117002E00A21294A11704DE03A2835
:1095B00003D10F21264A117002E00A21244A1170BA
:1095C00043E0202803D11021214A117002E00A2132
:1095D0001F4A117039E0014630391E4A11701121BD
:1095E0001B4A117031E02C2803D11221184A117046
:1095F0000BE0184909780A2251430246303A89188B
:10960000144A11701221124A11701EE04F2809D11C
:1096100013210F4A11700F4909781F2902DD00211B
:109620000C4A117011E04B2807D10321C9430A4AA3
:1096300011750A21064A117002E00A21044A1170CC
:1096400003E00A21024A117000BF00BF00BD000004
:109650006C0E0020720E0020133A002070B50446F4
:10966000D04800780A3803001BF099FA0C070D1750
:10967000212B353E5F80A0C0E0F32B2C02D10B20C4
:10968000C84908708BE1432C03D10C20C5490870F0
:1096900002E00A20C349087081E1432C03D10D2068
:1096A000C049087002E00A20BE49087077E14C2CDE
:1096B00003D10E20BB49087002E00A20B9490870A6
:1096C0006DE14B2C03D10F20B649087002E00A204F
:1096D000B449087063E1222C05D11020B14908700B
:1096E0000020B14908705AE12F2C10D0302C1BDB20
:1096F000392C19DCAC4800780A214843AA49087083
:109700002046303809784018A74908700CE0A6496F
:10971000097808466430A549FEF7F4FD0020A24907
:10972000087011209F49087039E12F2C10D0302C7F
:109730001BDB392C19DC9C4800780A2148439A49E4
:1097400008702046303809784018974908700CE0B6
:1097500095490978481E9549091FFEF7D3FD002059
:109760009149087012208F49087018E12C2C10D0F4
:10977000302C1ADB392C18DC8B4800780A2148433E
:1097800089490870204630380978401886490870A1
:109790000BE08649083984480078FEF7B3FD0020C5
:1097A0008149087013207F490870F8E03A2C10D0E6
:1097B000302C1ADB392C18DC7B4800780A2148430E
:1097C0007949087020463038097840187649087081
:1097D0000BE076490C3974480078FEF793FD0020C1
:1097E0007149087014206F490870D8E03A2C10D0E5
:1097F000302C1ADB392C18DC6B4800780A214843DE
:109800006949087020463038097840186649087060
:109810000BE06649103964480078FEF773FD0020BC
:109820006149087015205F490870B8E0222C11D0FA
:10983000302C0DDB392C0BDC5B4800780A214843C7
:109840005949087020463038097840185649087040
:10985000A0E0A0E05549143953480078FEF752FDC6
:109860005248FEF737FD0546643D50492846FEF74D
:1098700049FD4E48001FFEF72DFD451C4B49091FB1
:109880002846FEF73FFD49481438FEF723FD0546FC
:109890000A21FEF755FC060144481438FEF71AFD6C
:1098A00005460A21FEF74CFC0E4341498E713F48A4
:1098B0001038FEF70FFD05460A21FEF741FC0601B0
:1098C0003A481038FEF706FD05460A21FEF738FC37
:1098D0000E4337494E7135480C38FEF7FBFC054600
:1098E0000A21FEF72DFC060130480C38FEF7F2FC89
:1098F00005460A21FEF724FC0E432D490E712B4824
:109900000838FEF7E7FC05460A21FEF719FC0601B8
:1099100026480838FEF7DEFC05460A21FEF710FC53
:109920000E4323498E702148001FFEF7D3FC0546E5
:109930000A21FEF705FC06011C48001FFEF7CAFCC1
:1099400005460A21FEF7FCFB0E4319494E701748E5
:10995000FEF7C0FC05460A21FEF7F2FB060113489C
:10996000FEF7B8FC05460A21FEF7EAFB0E43104954
:109970000E7008460078232802DB084614F0DFFF4B
:109980000020094908700A20064908700320C043D6
:109990000849087503E00A200249087000BF00BFAB
:1099A00070BD0000A50E0020A60E0020913A0020F8
:1099B000A70E0020133A00202E4909780A2906D064
:1099C0000B290ED00C2916D00D294DD11CE04928A9
:1099D00003D10B21274A117002E00A21254A117098
:1099E00046E0442803D10C21224A117002E00B21E9
:1099F000204A11703CE03A2805D100211E4A11701E
:109A00000D211C4A117033E0522823D04B2814D06A
:109A1000302801DB392803DD412824DB462822DCFD
:109A20001549097815291EDA13490A780978491C5D
:109A3000114B19701149885415E000210E4A11701C
:109A400000220E490A75111F0D4A11750A21094A93
:109A5000117008E00021084A1170C91E084A1175EA
:109A60000A21044A117003E00A21024A117000BF62
:109A700000BF70476C0E0020AE0E00202C2F00207F
:109A8000133A002000B5344909780A390B001BF05D
:109A900086F807050F19232D37415D002B2803D1C8
:109AA0000B212D4A117002E00A212B4A117051E05E
:109AB000432803D10C21284A117002E00A21264ACA
:109AC000117047E0472803D10D21234A117002E0AD
:109AD0000A21214A11703DE0532803D10E211E4A6C
:109AE000117002E00A211C4A117033E04E2803D1A4
:109AF0000F21194A117002E00A21174A117029E05A
:109B00003A2803D11021144A117002E00A21124AA6
:109B100011701FE04B280CD0302816DB392814DCDC
:109B20000E490A780978491C0C4B19700C49885465
:109B30000BE00021094A11700A21074A1170002226
:109B40000749CA73111F074A117503E00A21024A27
:109B5000117000BF00BF00BD6C0E0020A40E0020DD
:109B60000C2F0020133A002000B53D4909780A392E
:109B70000B001BF014F80A06101A242E3842485223
:109B80005C6E452803D10B21354A117002E00A2191
:109B9000334A117061E0562803D10C21304A11700C
:109BA00002E00A212E4A117057E0452803D10D2109
:109BB0002B4A117002E00A21294A11704DE04E280B
:109BC00003D10E21264A117002E00A21244A1170A5
:109BD00043E0542803D10F21214A117002E00A21E9
:109BE0001F4A117039E03A2803D110211C4A117024
:109BF00002E00A211A4A11702FE0302802D1112107
:109C0000174A117029E02C2803D11221144A11702F
:109C100002E00A21124A11701FE0312803D11321FA
:109C20000F4A117002E00A210D4A117015E0352823
:109C300007D10321C9430B4A11750A21084A117043
:109C400006E00221C943074A11750A21044A11702E
:109C500003E00A21024A117000BF00BF00BD0000EE
:109C60006C0E0020133A002010B5044631480078ED
:109C70000A2804D00B280FD00C2855D12DE02C2C0D
:109C800006D10B202B49087000202B49088002E0E8
:109C90000A20284908704BE02C2C1AD0302C1BDBF2
:109CA000392C19DC244800880A21484322490880BD
:109CB00020463038098840181F4908800846008827
:109CC0001A2809D10C201B49087000201A49088065
:109CD00002E00A20174908702AE00D2C20D0302C11
:109CE00021DB392C1FDC144800880A214843124923
:109CF000088020463038098840180F49088021F034
:109D0000F7F90D49098888420DD1232005F060F844
:109D10000320C043094908750A200649087002E07B
:109D20000A200449087003E00A200249087000BFB5
:109D300000BF10BD6C0E0020B20E0020133A0020B0
:109D400000B5344909780A390B001AF028FF0906D2
:109D5000101A242E384248526000452803D10B21A6
:109D60002C4A117002E00A212A4A117050E056284C
:109D700003D10C21274A117002E00A21254A1170F3
:109D800046E0452803D10D21224A117002E00A2144
:109D9000204A11703CE04E2803D10E211D4A11705B
:109DA00002E00A211B4A117032E0542803D10F212E
:109DB000184A117002E00A21164A117028E03A2868
:109DC00003D11021134A117002E00A21114A1170C7
:109DD0001EE0302802D111210E4A117018E02C2803
:109DE00003D112210B4A117002E00A21094A1170B5
:109DF0000EE0362807D10321C943074A1175002117
:109E0000044A117002E00A21024A117000E000BF0A
:109E100000BF00BD6C0E0020133A002070B5044650
:109E2000564800780A3803001AF0B9FE0805A10F59
:109E300019232D3A59A14E2C03D10C204F490870FB
:109E400002E00A204D49087095E04E2C03D10D2008
:109E50004A49087002E00A20484908708BE04D2CFE
:109E600003D10E204549087002E00A2043490870DA
:109E700081E0492C03D10F204049087002E00A20FC
:109E80003E49087077E03A2C06D100213C488171A8
:109E900010203A49087002E00A20384908706AE048
:109EA0002C2C14D0302C19DB392C17DC3448807959
:109EB000092808DA324881798079401C304A90714B
:109EC000101F44540AE000202D49887106E000214B
:109ED0002C488172C1721120284908704BE02C2C4B
:109EE0003BD00D2C39D02749C87A897A0002084323
:109EF00001218902884228DA21480838FEF7EAF968
:109F0000451C1F4908392846FEF7FCF9302C01DBB7
:109F1000392C07DD412C01DB462C03DD612C25DBD0
:109F2000662C23DC1748C17A807A09020143154A5E
:109F3000D07A927A00021043401C82B21148827299
:109F4000120AC2720C30445410E000210D48817294
:109F5000C1720A200949087008E0002008494872C7
:109F60000120203988750A200449087003E00A207E
:109F70000249087000BF00BF70BD00006D0E0020D8
:109F8000333A00201334002000B54B4909780A39D0
:109F90000B001AF004FE0D080E1826303A444E58F5
:109FA000626C76808A003A2802D10B21424A1170F5
:109FB0007FE0202803D10C213F4A117002E00A21E2
:109FC0003D4A117075E0522803D10D213A4A1170B3
:109FD00006E00221C943394A11750A21364A117037
:109FE00067E0452803D10E21334A117002E00A21AF
:109FF000314A11705DE0472803D10F212E4A1170BC
:10A0000002E00A212C4A117053E0492803D11021A3
:10A01000294A117002E00A21274A117049E05328A9
:10A0200003D11121244A117002E00A21224A117041
:10A030003FE0542803D112211F4A117002E00A2187
:10A040001D4A117035E0452803D113211A4A1170B9
:10A0500002E00A21184A11702BE0522803D1142182
:10A06000154A117002E00A21134A117021E04528B7
:10A0700003D11521104A117002E00A210E4A117015
:10A0800017E0442803D116210B4A117002E00A217F
:10A09000094A11700DE04B2806D10321C943074A34
:10A0A00011750A21044A117003E00A21024A117055
:10A0B00000BF00BF00BD00006C0E0020133A00205E
:10A0C00000B5264909780A390B001AF068FD070522
:10A0D0000B11171D23294100542802D10B211F4ABF
:10A0E000117039E0492802D10C211C4A117033E06B
:10A0F0004E2802D10D21194A11702DE0442802D1B9
:10A100000E21164A117027E03A2802D10F21134A76
:10A11000117021E0202802D11021104A11701BE09B
:10A12000332804D10321C9430D4A11750CE03628A8
:10A1300004D10321C9430A4A117505E0312803D12E
:10A140000221C943064A11750A21044A117003E02D
:10A150000A21024A117000BF00BF00BD6C0E002032
:10A16000133A002010B50446304800780A3803003E
:10A170001AF015FD07050F19232D37415600542CF1
:10A1800003D10B202949087002E00A2027490870F2
:10A190004AE0492C03D10C202449087002E00A202F
:10A1A0002249087040E04E2C03D10D201F49087051
:10A1B00002E00A201D49087036E0442C03D10E202D
:10A1C0001A49087002E00A20184908702CE03A2C5D
:10A1D00003D10F201549087002E00A2013490870C6
:10A1E00022E0202C03D110201049087002E00A2040
:10A1F0000E49087018E0342C0AD1232004F0E8FD41
:10A200000320C0430A4908750A200849087006E07F
:10A210000220C043064908750A200449087003E07B
:10A220000A200249087000BF00BF10BD6C0E00205C
:10A23000133A002070B50446F84800780A38030045
:10A240001AF0ADFC120A154A7EB0B9E1F8F6F5F441
:10A25000F3F2F1F0EFEEEDEC2C2C07D10020F049F9
:10A260000870F04908800B20EC4908705EE22C2C45
:10A270001DD100200021EB4A118000BF0CE0E9490C
:10A2800009880A225143E74A1180E749095C12888C
:10A290008918E44A1180401CE14909788842EEDBC4
:10A2A0000021DF4A11700C21DC4A117013E0DC48F8
:10A2B00000780A280CDA20463038C1B2DA48D84A89
:10A2C00012788154D6480078401CD549087002E0C5
:10A2D0000020D2490870EDE32C2C1DD10020002174
:10A2E000D24A116000BF0CE0D04909680A225143EC
:10A2F000CE4A1160CC49095C12688918CB4A1160BA
:10A30000401CC74909788842EEDB0021C44A11701D
:10A310000D21C24A117012E0C14800780A280BDAF8
:10A3200020463038C049BE4A12788854BC4800786C
:10A33000401CBB49087002E00020B8490870B9E32E
:10A340002C2C1AD100200021B94A118000BF0CE04A
:10A35000B74909880A225143B54A1180B249095CBC
:10A3600012888918B24A1180401CAD490978884288
:10A37000EEDB0E21A94A117013E0A94800780528E8
:10A380000CDA20463038C1B2A748A54A1278815469
:10A39000A3480078401CA249087002E000209F49B1
:10A3A000087087E3222C05D100209D4908700F20FA
:10A3B0009A4908707EE3222C13D100250A219D487A
:10A3C000FDF761FF00BF04E09748405D994948559B
:10A3D0006D1C934800788542F6DB10208F49087089
:10A3E00010E08F4800780A2809DA8F488C490978EC
:10A3F00044548B480078401C8949087002E00020D2
:10A400008649087056E32C2C07D100208449087037
:10A41000854908701120814908704BE346E39CE2AE
:10A420008CE280E256E24AE213E280E108E17EE05B
:10A4300072E0FFE72E2C57D179480078012804D12B
:10A44000794840787C4908803AE0754800780228CD
:10A4500009D1754840780A214843734989784018E2
:10A46000754908802CE06E48007803280FD16E48AB
:10A470004078642148436C4989780A225143401846
:10A480006949C978401800B26B49088018E06448EF
:10A490000078042814D1644840787D21C9004843DD
:10A4A000614989786422514341185F48C0780A2283
:10A4B000504308185C490979401800B25E49088089
:10A4C0005D4800880A21484300B25B49088056482D
:10A4D0000078012804D108460088404200B2088074
:10A4E00012204E49087016E02D2C03D101204E4950
:10A4F000087010E04A48007804280CDA204630380A
:10A50000C1B247480078401C474A1154444800787B
:10A51000401C43490870CDE22C2C07D10020404953
:10A5200008704149087013203C490870C2E22C2C85
:10A530005CD13B480078012804D13B4840783F4932
:10A5400008803AE036480078022809D13648407839
:10A550000A214843344989784018384908802CE05A
:10A560002F48007803280FD12F48407864214843B2
:10A570002D4989780A22514340182B49C97840183F
:10A5800000B22E49088018E025480078042814D12C
:10A59000254840787D21C9004843234989786422B1
:10A5A000514341182048C0780A22504308181E49D8
:10A5B0000979401800B221490880204800880A2102
:10A5C000484300B21D49088017480078012804D18B
:10A5D00008460088404200B20880002010490870F8
:10A5E0001149087014200D49087016E02D2C03D174
:10A5F00001200D49087010E00948007804280CDAA1
:10A6000020463038C1B206480078401C064A115432
:10A6100003480078401C024908704BE26C0E002091
:10A62000750E0020800E0020A93A0020840E002024
:10A63000880E0020B43A00208A0E00208C0E0020E4
:10A640002C2C5CD1FE480078012804D1FD484078CC
:10A65000FD4908803AE0FA480078022809D1F94813
:10A6600040780A214843F74989784018F64908801C
:10A670002CE0F348007803280FD1F2484078642199
:10A680004843F04989780A2251434018ED49C97876
:10A69000401800B2EC49088018E0E9480078042826
:10A6A00014D1E84840787D21C9004843E5498978BC
:10A6B000642251434118E348C0780A2250430818E5
:10A6C000E0490979401800B2DF490880DE48008877
:10A6D0000A21484300B2DC490880DA4800780128A2
:10A6E00004D108460088404200B208800020D449C6
:10A6F0000870D44908701520D449087016E02D2C34
:10A7000003D10120CF49087010E0CD48007804281B
:10A710000CDA20463038C1B2C9480078401CC94A1A
:10A720001154C7480078401CC5490870C2E12C2C60
:10A7300073D1C348007801280BD1C2484078C4497E
:10A740000880084600880A21484300B2C0490880B2
:10A750004FE0BB480078022810D1BA4840780A215F
:10A760004843B84989784018B949088008460088A4
:10A770000A21484300B2B64908803AE0B048007860
:10A78000032816D1AF48407864214843AD49897801
:10A790000A2251434018AB49C978401800B2AC496D
:10A7A0000880084600880A21484300B2A84908806A
:10A7B0001FE0A348007804281BD1A24840787D21DF
:10A7C000C90048439F4989786422514341189D48F4
:10A7D000C0780A22504308189A490979401800B2F3
:10A7E0009B490880084600880A21484300B29849DE
:10A7F000088094480078012805D195480088404297
:10A8000000B29349088000208D4908708D49087076
:10A8100016208E4908701BE0FFE72D2C03D1012084
:10A820008849087014E08648007804280DDA20462C
:10A830003038C1B2834A82480078401C11548048A5
:10A840000078401C7E49087002E00A207F490870A9
:10A8500030E12C2C1FD1002000217E4A118000BF46
:10A860000CE07C4909880A2251437A4A11807549D3
:10A87000095C12888918774A1180401C7049097850
:10A880008842EEDB00216E4A11706E4A117017216A
:10A890006E4A117012E06A48007804280BDA2046EC
:10A8A00030386849664A1278885465480078401CF8
:10A8B0006349087002E00A2064490870FAE0222C1B
:10A8C00007D100205E4908705E49087018205F4972
:10A8D0000870EFE0222C14D1002000BF04E0594999
:10A8E000095C5D4A1154401C554909788842F6DBE1
:10A8F0000021534A1170534A11701921534A1170A3
:10A9000010E04F4800780A2809DA4E484C49097887
:10A9100044544B480078401C4949087002E000202C
:10A920004A490870C6E02C2C07D100204449087021
:10A93000444908701A2045490870BBE02C2C07D107
:10A9400040480078454908801B204049087003E0D2
:10A95000204630383B490870ACE02D2C03D1012053
:10A9600038490870A1E0302C17DB392C15DC34484D
:10A97000007804280DDA20463038C1B2314A304818
:10A980000078401C11542E480078401C2C49087057
:10A990008BE00A202D49087087E0294800780128BB
:10A9A0000BD1284840782E490880084600880A21A3
:10A9B000484300B22A49088013E021480078022861
:10A9C0000FD1204840780A2148431E498978401811
:10A9D00023490880084600880A21484300B22049DC
:10A9E000088017480078032816D11648407864215B
:10A9F0004843144989780A22514340181149C978BB
:10AA0000401800B216490880084600880A214843C9
:10AA100000B21349088032E00948007804282ED19A
:10AA2000084840787D21C900484306498978642256
:10AA3000514341180348C0780A225043081811E0D6
:10AA4000750E0020A93A00208E0E00206C0E00200A
:10AA5000900E0020920E0020BE3A0020940E00209E
:10AA6000960E002014490979401800B21349088055
:10AA7000084600880A21484300B2104908800E4861
:10AA80000078012805D10D480088404200B20B49EA
:10AA9000088000200A490870074908700A200949FF
:10AAA00008700320C0430849087503E00A200549DF
:10AAB000087000BF00BF70BDA93A0020960E0020AC
:10AAC000750E00206C0E0020133A00202A490978E8
:10AAD0000A2906D00B290AD00C291ED00D2945D1F0
:10AAE00025E04F2802D10B21234A117042E04B2868
:10AAF00006D10121214A11700C211F4A11700BE06F
:10AB0000522806D100211D4A11700C211A4A1170D9
:10AB100002E00A21184A11702CE00D2803D10D2102
:10AB2000154A117002E00A21134A117022E00A2826
:10AB300018D112490978002904D00321C943104AC9
:10AB4000117503E00221C9430D4A11750D49097AB7
:10AB50000B2903D10A21084A117006E00021064A98
:10AB6000117002E00A21044A117003E00A21024A2E
:10AB7000117000BF00BF70476C0E0020A20E0020B5
:10AB8000133A00201334002000B5224909780A390D
:10AB90000B001AF004F808050B11171D23292F3993
:10ABA0002B2802D10B211B4A117031E0512802D110
:10ABB0000C21184A11702BE0492802D10D21154AA9
:10ABC000117025E04F2802D10E21124A11701FE0AA
:10ABD000502802D10F210F4A117019E0452802D1E7
:10ABE00010210C4A117013E04E2802D11121094A9C
:10ABF00011700DE03A2803D10321C943064A1175AB
:10AC00000A21044A117003E00A21024A117000BFB0
:10AC100000BF00BD6C0E0020133A00200E490978D9
:10AC20000A2902D00B2911D105E0572802D10B21A6
:10AC3000094A11700EE04E2804D10321C943074A86
:10AC4000117502E00A21044A117003E00A21024A48
:10AC5000117000BF00BF70476C0E0020133A002037
:10AC6000144909780A2904D00B2908D00C291BD1D2
:10AC70000FE0452802D10B210E4A117018E045283B
:10AC800003D10C210B4A117002E00A21094A11700C
:10AC90000EE0502804D10321C943074A117502E090
:10ACA0000A21044A117003E00A21024A117000BF10
:10ACB00000BF70476C0E0020133A002000B56349B6
:10ACC00009780A390B0019F06AFF0B07111B252FB1
:10ACD00039434D697394BB00222803D10B215B4A91
:10ACE000117002E00A21594A1170ADE0722803D1B7
:10ACF0000C21564A117002E00A21544A1170A3E057
:10AD0000652803D10D21514A117002E00A214F4AF2
:10AD1000117099E0632803D10E214C4A117002E0B2
:10AD20000A214A4A11708FE0762803D10F21474A41
:10AD3000117002E00A21454A117085E0222803D1F2
:10AD40001021424A117002E00A21404A11707BE052
:10AD50002C2803D111213D4A117002E00A213B4AFF
:10AD6000117071E000213A4A9172D172394A118012
:10AD7000302806D10121384A51721221334A11700C
:10AD80000BE0312806D10221334A517212212F4A99
:10AD9000117002E00A212D4A117055E02C2803D1D0
:10ADA00013212A4A117002E00A21284A11704BE04F
:10ADB0000A2810D030281BDB392819DC25490988DE
:10ADC0000A225143234A11800146303912888918DA
:10ADD000204A11800CE01F49098801229202914209
:10ADE00003DA1421194A117002E00021174A117088
:10ADF0002AE0174AD17A927A09021143154A128839
:10AE0000914212DA124AD17A937A0A021A43104B0B
:10AE1000D97A9B7A09021943491C8BB20C498B726F
:10AE20001B0ACB720C31885409E00321C9430A4A3A
:10AE3000203A1175012191750A21044A117003E02D
:10AE40000A21024A117000BF00BF00BD6F0E002032
:10AE500013340020700E0020333A002010B5044651
:10AE6000484800780A38030019F099FE0B07111BB7
:10AE7000252F39434D57616E8600442C03D10B209A
:10AE80004049087002E00A203E49087078E0492CE9
:10AE900003D10C203B49087002E00A2039490870B0
:10AEA0006EE0532C03D10D203649087002E00A20D1
:10AEB0003449087064E0432C03D10E2031490870F6
:10AEC00002E00A202F4908705AE04F2C03D10F20CE
:10AED0002C49087002E00A202A49087050E0562CDC
:10AEE00003D110202749087002E00A202549087084
:10AEF00046E0452C03D111202249087002E00A20C7
:10AF0000204908703CE0522C03D112201D490870E2
:10AF100002E00A201B49087032E03A2C03D11320CA
:10AF20001849087002E00A201649087028E02C2C05
:10AF300009D10020144908700A211448FDF7A3F92B
:10AF40001420104908701BE02C2C0CD00E480078FF
:10AF50000A2810D20C4801780078401C0A4A107068
:10AF60000A48445407E00320C04308492B390875B8
:10AF70000A200449087003E00A200249087000BF53
:10AF800000BF10BDAF0E0020B00E00203E3A0020E2
:10AF90000148007870470000250100200348007830
:10AFA000002801D1012070470020FCE72401002087
:10AFB000002004490978002901D1012000E0002087
:10AFC000704700002401002070B555480078030048
:10AFD00019F0E5FD050405102593A3009EE001206E
:10AFE00000F070FD002804D10EF04FFE02204C4905
:10AFF000087093E04B48007800F008F9012000F059
:10B0000017F900F079F917F0E5F84749086017F0EB
:10B01000E1F8464908600320414908707EE00120BC
:10B0200000F022F9012855D117F0D4F83F49086003
:10B0300017F0D0F83C490968401A3D490968884230
:10B040005AD3002400F01CF904463A48406800191D
:10B050003849486038480078002803D108468460A1
:10B06000046013E033488068A04201D2204601E02A
:10B07000304880682F49886008460068A04201D99E
:10B08000204601E02B4800682A4908602A480078D9
:10B09000401CC0B22849087028490978884215DB4D
:10B0A00000252448406823490968401A21498968D5
:10B0B000451A22480078811E2846FDF72BF82049C2
:10B0C0000968086004201649087002E0022014494B
:10B0D000087011E017F07EF814490968401A6428D6
:10B0E0000AD900F00FF917480078022108431549E2
:10B0F000087004200A49087010E000F0A1F800F080
:10B10000EDFB0021102016F09DFC01200E4909687E
:10B11000087000200249087000E000BF00BF70BD49
:10B120002401002035010020380100203C010020CE
:10B130002C0100203C1C002034010020360100209E
:10B1400028010020250100203001002010B500F06A
:10B1500077F800F0C3FB0021102016F073FC10BD3F
:10B16000F8B505460C4616461F46032C00D20324AC
:10B17000502C00D950241B4906980860192D0ADD6F
:10B180001948007801210843174908700120154922
:10B1900009680870F8BD1548076000201149096862
:10B1A00008701349087013494860086088600E49A8
:10B1B00008701148057011490C70114806600EF0B6
:10B1C0007EFD0121102016F03DFC00F091FB00F007
:10B1D00041F80121084614F0C1F80120094908701E
:10B1E00000BFD7E730010020250100202801002002
:10B1F000340100203C1C00203501002036010020D5
:10B200002C0100202401002070470000014607485F
:10B210004068FF22F13290430A01FF23F1331A40C4
:10B220001043024A50600020704700000024004094
:10B230000249496B8143014A5163704780240040B1
:10B2400003484068400840000149486070470000DA
:10B25000002400400348406840084000401C014969
:10B26000486070470024004001460448006B0840D5
:10B27000002801D0012070470020FCE78024004016
:10B280000148006A704700008024004010B5044661
:10B29000002C01D1042010BD012016494860022075
:10B2A0001AF08CFB6078A1880843E1880843618824
:10B2B0000843218908430F49496808430D494860FC
:10B2C0000846806809158843217889020122920284
:10B2D0001140084307498860084680680421884374
:10B2E000A17A8900042211400843024988600020A5
:10B2F000D1E70000002400400120014908607047A8
:10B30000C02400400020014908607047C02400406C
:10B3100030B50A4600210EE0D400A41A074D641986
:10B32000635C04785C4004700478AA256C40047067
:10B33000401C4C1CE1B20729EEDB30BDCCD9020029
:10B34000F0B587B013F06AF910210840002810D03A
:10B35000042013F08BF9FA480088401CF849088053
:10B36000E1210901F6480088FCF7EAFE88B2F449B9
:10B37000088013F053F920210840002822D005202E
:10B3800013F074F9EF480078401CEE490870084645
:10B3900000783C2816DB00200870EB48FCF79AFF89
:10B3A000E12109014418E8492046FCF7ABFFE648D3
:10B3B000001DFCF78FFF0446233CE349091D20468E
:10B3C000FCF7A0FFE1480078002804D001280ED047
:10B3D00002287DD1A5E102F0AFFD002806D1D848B2
:10B3E0000088DB4908600120D8490870CAE102F0F2
:10B3F000A3FD01286DD1002106910591D048008858
:10B40000D3490968884207D3CD480088D0490988C4
:10B41000401AD049088009E0C9480088E1210901A3
:10B420004018CB490988401ACA49088008201FF0F3
:10B4300017FE772807D1C74800884B21C90040185C
:10B44000C44908800BE008201FF00AFE552806D1E9
:10B45000C0480088E121C9004018BE490880002189
:10B46000082021F07FF9B8480C30FCF733FFB949C8
:10B4700009884418B4490C312046FCF743FFB24810
:10B48000417C027C08021043401C81B2AE4801742A
:10B49000090A417406A80FF0C9FA05A80FF0B8FA16
:10B4A0000A216A461820105EFCF74AFE00B2069098
:10B4B0000A216A461420105EFCF742FE00B2059095
:10B4C00004201FF0CDFD01283DD1A248008801E0F5
:10B4D00054E125E1FDF7BAF906469F4A9F4BFDF777
:10B4E000AFF8019100909848001DFCF7F3FE064666
:10B4F000FDF7ACF90446019B009AFDF793F8039120
:10B500000290FDF701FA9049091D0490FCF7FAFE3C
:10B5100004F0ACFA002815D191480078401C9049FD
:10B52000087007218E480078FCF70AFEC8B28C49E3
:10B53000087008460178022021F014F901210A2040
:10B5400021F010F9E8E069461820085E002820DAAA
:10B5500080480088FDF77AF906467F4A814BFDF75F
:10B560006FF8019100907848001DFCF7B3FE064685
:10B57000FDF76CF90446019B009AFDF753F803911F
:10B580000290FDF7C1F97049091D0490FCF7BAFE5D
:10B59000C2E069461420085E7721C943884220DA58
:10B5A0006C480088FDF752F904466B4A6D4BFDF775
:10B5B00047F8039102906448001DFCF78BFE044697
:10B5C000FDF744F901910090039B029AFDF72AF8D8
:10B5D0000646FDF799F95C49091D0490FCF792FEB7
:10B5E0009AE069461420085E7221C943884220DA35
:10B5F00058480088FDF72AF906465B4A5B4BFDF781
:10B600001FF8019100905048001DFCF763FE0646AC
:10B61000FDF71CF90446019B009AFDF703F803911E
:10B620000290FDF771F94849091D0490FCF76AFE84
:10B6300072E069461420085E6821C943884222DA14
:10B6400044480088FDF702F90646434A5242484BF7
:10B65000FCF7F6FF04460D463B48001DFCF73AFE9A
:10B660000646FDF7F3F822462B4601910090FCF7C1
:10B67000D9FF03910290FDF747F93349091D049062
:10B68000FCF740FE48E069461420085E5921C94392
:10B69000884220DA2F480088FDF7D8F804462E4A61
:10B6A0002E4BFCF7CDFF019100902748001DFCF7C1
:10B6B00011FE0446FDF7CAF80646019B009AFCF706
:10B6C000B1FF03910290FDF71FF91F49091D049076
:10B6D000FCF718FE20E01F480088FDF7B7F8044685
:10B6E0001D4A5242234BFCF7ABFF019100901648D4
:10B6F000001DFCF7EFFD0446FDF7A8F80646019B88
:10B70000009AFCF78FFF03910290FDF7FDF80E49B8
:10B71000091D0490FCF7F6FD02200C49087000BFDB
:10B7200030E001F08FF9012808D1134B1822D02105
:10B73000054801F0EBFB00200449087022E00000FE
:10B740003C0C00203E0C0020702C00202D0C002012
:10B75000300C0020400C00203333333333331F4090
:10B76000500C002033B330406666666666662D4036
:10B77000CCCC2140CCCC1A402C0C002000203049ED
:10B78000087000BF00BF2F480078002802D00128B1
:10B790004FD10BE00AF000FD002806D12A480088AE
:10B7A0002A49086001202749087046E00AF0F4FCA5
:10B7B00001283DD12448008824490968884207D3DC
:10B7C0002148008821490988401A2149088009E058
:10B7D0001D480088E121090140181C490988401AC8
:10B7E0001B4908801B4800681949098840181949F5
:10B7F0000860084600683C2817D9084600683C38AD
:10B8000008601548FCF766FD04463C3412492046A2
:10B81000FCF778FD1048001FFCF75CFD0446153C62
:10B820000D49091F2046FCF76DFD002005490870F1
:10B8300003E000200349087000BF00BF07B0F0BD5F
:10B840002D0C00202E0C00203C0C0020340C00207D
:10B85000400C0020380C0020782C0020074800788D
:10B86000002809D106480078002805D1054800784D
:10B87000002801D1012070470020FCE72D0C00209A
:10B880002E0C0020510C002001468020084000288A
:10B8900001D008467047302905DB392903DC08460A
:10B8A0003038C0B2F6E7612905DB662903DC0846BB
:10B8B0005738C0B2EEE7412905DB462903DC0846CC
:10B8C0003738C0B2E6E70846E4E701460A110A2322
:10B8D0005A430B071B0FD218D0B2704703480068B9
:10B8E0000221084001490860704700000024004020
:10B8F00010B505480068012108430349086002208B
:10B900001AF05CF810BD00000024004030B502467B
:10B9100000201402044D63191C68240C24048DB209
:10B920002C431C6030BD0000000C004030B50246C6
:10B9300000201402044D63195C68240C24048DB2A9
:10B940002C435C6030BD0000000C004010B5014687
:10B9500000200B02014C1A19906810BD000C004029
:10B9600030B5024600201402024D63199C689960AC
:10B9700030BD0000000C004070B5024600201402EB
:10B98000054D63191C6BAD14AC430D030126360342
:10B9900035402C431C6370BD000C004010B50146BF
:10B9A00000200B02034C1A19D3685B085B005B1C78
:10B9B000D36010BD000C004010B5014600200B0202
:10B9C000034C1A19D3685B085B00D36010BD0000FC
:10B9D000000C004070B503460A4600201C02224DB0
:10B9E0006119CC68AD00AC4315782D0303263603EE
:10B9F00035402C43CC60CC6801256D02AC435578B2
:10BA00006D020126760235402C43CC60CC6875105F
:10BA1000AC4395782D02761035402C43CC60CC6831
:10BA20007025AC43D5782D01702635402C43CC6071
:10BA3000CC680825AC431579ED00082635402C4329
:10BA4000CC60CC680425AC435579AD000426354064
:10BA50002C43CC60CC680225AC4395796D0002265E
:10BA600035402C43CC6070BD000C004010B500F098
:10BA700009F910BD70B5044600252C2C1BDA16F010
:10BA8000A9FB0546A0000D490858A84203D8A0000C
:10BA900008582D1A06E0A000084908580021C9439B
:10BAA000081A4519A00006490858A84201D80020E4
:10BAB00070BD0120FCE70020FAE700009815002087
:10BAC0004816002070B504460025182C1BDA16F025
:10BAD00081FB0546A0000D490858A84203D8A000E4
:10BAE00008582D1A06E0A000084908580021C9434B
:10BAF000081A4519A00006490858A84201D8002094
:10BB000070BD0120FCE70020FAE70000D8140020F7
:10BB1000381500200148007870470000A806002072
:10BB200010B50648FCF7E0FB054B064A43404A4087
:10BB3000134301D1012010BD0020FCE7F6220020B4
:10BB4000B8A7F6E5D4C3B2A1014800787047000059
:10BB50001804002070B504460025002616F03AFBB4
:10BB6000064609480068351A0848844203D1A542B0
:10BB700001D3012070BD0648844203D1A54201D300
:10BB80000120F7E70020F5E76400002050C3000023
:10BB9000C02709000148007870470000A90600206E
:10BBA000FFB583B006460F461C4638461FF084FB9F
:10BBB000029005981FF080FB0190607821780002C8
:10BBC0000843002806DD6078217800020843164902
:10BBD00088420FDB6078217800020843124908315F
:10BBE00088421EDD60782178000208430E49093141
:10BBF000884216DA6078217800020843B04203D008
:10BC000009480F3086420CD1A01C1FF055FB054699
:10BC10000298854205D30198854202D8012007B0D9
:10BC2000F0BD0020FBE70000F0FF000001480078B5
:10BC3000704700003206002001480068704700008D
:10BC400034060020002002498872C8727047000044
:10BC5000C72E00200020014908707047A40400206E
:10BC600000200149C8757047133A0020002001499F
:10BC700008707047180400200020014908707047C0
:10BC80003206002010B5012016F0E4FA01280DD18B
:10BC900016F0DAFA574908600846006856498842A3
:10BCA00005D116F0EDFAFF205449087096E051488E
:10BCB00000685149884246D216F0E2FA50480078AE
:10BCC000002803D04E48007801281ED101204C499D
:10BCD000087048490968484A501A4949491CFCF704
:10BCE00011FB4849C968491C4805400D4549C968C8
:10BCF000C90AC9020143434AD16016F0B7FA424863
:10BD00000078401C4049087068E03D48401CFCF742
:10BD1000E1FA38490968384A511A88420FD239493C
:10BD2000C968491C4805400D3649C968C90AC90295
:10BD30000143344AD160FF20304908704EE0FF20B3
:10BD40002E4908704AE02B4800682B49884245D9A3
:10BD500016F096FA2A480078002803D02848007880
:10BD600002281ED102202649087022490968224A69
:10BD7000881A2349491CFCF7C5FA2249C968491E9B
:10BD80004805400D1F49C968C90AC90201431D4A37
:10BD9000D16016F06BFA1C480078401C1A490870F4
:10BDA0001CE01748401CFCF795FA12490968124A32
:10BDB000891A88420FD21349C968491E4805400DA7
:10BDC0001049C968C90AC90201430E4AD160FF205F
:10BDD0000A49087002E0FF2008490870022016F0A6
:10BDE00039FA012804D116F04BFAEE200349087005
:10BDF00010BD00000005002000093D00F6040020F1
:10BE0000F804002000200040F704002010B50020B6
:10BE100015F0F0FD002015F001FE112015F060FE78
:10BE2000022015F04BFE0121022015F07DFC0220BE
:10BE300015F07AFE042015F02DFE0121002015F0EA
:10BE400073FC002015F070FE0121062002F000FDB9
:10BE5000002002F061FD01211C2015F0F3FD10BD52
:10BE600000200149087070477009002010B500F0EB
:10BE700001F810BDF8B5B3480078030018F08FFE44
:10BE800005040FD9FEFDFC000020AF490870012019
:10BE9000AC490870FF202D3020F072FC50E119F001
:10BEA000D0F900287ED10D24A8480688A848056846
:10BEB000002751E0E85D0A2808DAE85D3030C2B2B8
:10BEC0002046611C8CB2A3490A543EE0E85D642818
:10BED00016DAE85D0A21FCF733F93030C2B22046A9
:10BEE000611C8CB29B490A54E85D0A21FCF728F9D1
:10BEF0003031CAB22046611C8CB296490A5424E003
:10BF0000E85D6421FCF71CF93030C2B22046611CA8
:10BF10008CB290490A54E85D0A21FCF711F90A2114
:10BF20000090FCF70DF93031CAB22046611C8CB28A
:10BF300088490A54E85D0A21FCF702F93031CAB297
:10BF40002046611C8CB283490A542E222046611C73
:10BF50008CB280490A547F1C042FABDB601E84B274
:10BF600022222046611C8CB27A490A542C22204697
:10BF7000611C8CB277490A5477493046FCF7E0F8E7
:10BF80003030C2B22046611C8CB272490A547249E8
:10BF90003046FCF7D5F800917D21C9000098FCF7E8
:10BFA000CFF800E044E03030C2B22046611C8CB2D1
:10BFB00068490A547D21C9003046FCF7C1F8009158
:10BFC00064210098FCF7BCF83030C2B22046611CF6
:10BFD0008CB260490A5464213046FCF7B1F80091F4
:10BFE0000A210098FCF7ACF83030C2B22046611C40
:10BFF0008CB258490A540A213046FCF7A1F8303176
:10C00000CAB22046611C8CB252490A540D22204605
:10C01000611C8CB24F490A54122221464D4810F03F
:10C0200017FA232020F0B8FB02204649087000BF11
:10C0300086E00EF069FC001D002809D14249087015
:10C04000032040490870FF202D3020F099FB26E0A6
:10C0500019F0FCF8002804D00EF056FCC01C002893
:10C060001DD139480078401C3749087008460078CF
:10C07000012811DB002002E05EE027E010E00870FC
:10C080003648FCF727F9A521017000202D490870DA
:10C09000A8203349087002E001202A4908704FE0C7
:10C0A00019F0CFF8002810D12E480068FCF702F9EB
:10C0B00084B21B2221462B48006810F0C9F90220E7
:10C0C00020F06AFB04201F49087039E00EF01CFCC8
:10C0D000001D00280DD11C4908702048FCF7FAF813
:10C0E000A3210170002017490870A9201C4908707D
:10C0F00021E019F0ABF800281DD113480078401C4E
:10C10000114908700846007801280DDB00200870EE
:10C110001248FCF7DFF8A5210170002009490870DA
:10C12000A8200F49087006E0032006490870FF2088
:10C130002D3020F025FB03E000200249087000BFED
:10C1400000BFF8BDAA0C0020620D0020BC0C00202E
:10C15000B80C0020630D002010270000412F0020A4
:10C16000A20C0020980D002010B500F001F810BDC1
:10C1700070B5C1480078002804D003280AD00428EC
:10C180007ED13CE10320BC490870FF202D3020F017
:10C19000F7FA6FE119F055F8002872D1082400254C
:10C1A00004E0B648405DB64948556D1C082DF8DBE3
:10C1B000B44A517A127A090211430846B249FBF790
:10C1C000BFFF3030C2B22046611C8CB2AC490A5469
:10C1D000AC4A517A127A090211430846AA49FBF780
:10C1E000AFFF0E467D21C9003046FBF7A9FF303076
:10C1F000C2B22046611C8CB2A1490A54A14A517AAC
:10C20000127A0902114308467D21C900FBF798FF05
:10C210000E4664213046FBF793FF3030C2B2204611
:10C22000611C8CB296490A54964A517A127A0902D4
:10C23000114308466421FBF783FF0E460A2130466E
:10C24000FBF77EFF3030C2B22046611C8CB28C49B5
:10C250000A548C4A517A127A0902114308460A217B
:10C26000FBF76EFF3031CAB22046611C8CB28449A4
:10C270000A542C222046611C8CB281490A5401E0E8
:10C28000F4E0BBE0002545E07E48001DFCF722F805
:10C29000405D00110A280CDB7A48001DFCF71AF8F3
:10C2A000405D001137302146621C94B2744A5054EC
:10C2B0000BE07448001DFCF70DF8405D00113030B4
:10C2C0002146621C94B26E4A50546E48001DFCF721
:10C2D00001F8405D0007000F0A280DDB6948001DCA
:10C2E000FBF7F8FF405D0007000F37302146621C66
:10C2F00094B2634A50540CE06248001DFBF7EAFF19
:10C30000405D0007000F30302146621C94B25C4A49
:10C3100050546D1C5B49487A097A00020843A842D0
:10C32000B2DC5A48007B80210840002828D05748BA
:10C33000007B8007800F002822D02C222046611C21
:10C340008CB24F490A5431222046611C8CB24C49B0
:10C350000A5430222046611C8CB249490A542046B6
:10C36000611C8CB246490A540D222046611C8CB2D5
:10C3700043490A5437222146414810F069F836E013
:10C380004248807A552804D0404876308078552835
:10C3900022D12C222046611C8CB239490A54312208
:10C3A0002046611C8CB236490A5430222046611C5A
:10C3B0008CB233490A542046611C8CB230490A546D
:10C3C0000D222046611C8CB22D490A543722214689
:10C3D0002B4810F03DF80AE00D222046611C8CB27B
:10C3E00027490A5416222146254810F031F8042026
:10C3F00020F0D2F904202049087000BF3AE00EF086
:10C4000083FA001D00280DD121490870A920214977
:10C4100008701C48FBF75EFFA4210170002016493C
:10C42000087022E00EF070FAC01C002803D018F04B
:10C430000DFF002819D116480078401C14490870D7
:10C440000846007801280DDB002008700D48FBF736
:10C4500041FFA5210170A8200E490870002006495F
:10C46000087002E004200449087003E0002002493B
:10C47000087000BF00BF70BDAC0C002012DA0200D3
:10C480004B2F0020412F002010270000342C0020CB
:10C490009C0D0020A20C002000200149087070476C
:10C4A000AA0C002070B546480078002806D0012864
:10C4B00005D0032874D006287CD123E07EE000F06C
:10C4C000C1FA01281DD13F48007840280FD0DC2256
:10C4D0003D493E48FBF7BEFE3D4BDC2201214902AF
:10C4E0003A4800F013FD03203549087009E0384B45
:10C4F000DC2236490120400200F0C2FC062030490F
:10C5000008705BE000F09EFA012846D10025002467
:10C510002EE0A1002D4A8818FBF7DCFE0021C9435C
:10C52000884201D1002525E0A100284A8818FBF7A0
:10C53000D1FE064631462748FCF75CFA09D3A10034
:10C54000224A8818FBF7C6FE06462349FCF752FA32
:10C5500001D200250EE0A1001C4A8818FBF7BAFEA4
:10C5600006460021FCF746FA00D00125601CC4B243
:10C57000372CCEDB00BF002D0BD1DC221249134833
:10C58000FBF768FE124BDC22012149020F4800F044
:10C59000BDFC03200A49087000BF0FE000E009E07D
:10C5A00000F050FA012804D10C4908700020044919
:10C5B000087003E000200249087000BF00BF70BD92
:10C5C000490B0020A02B0020ACDA02008B42002097
:10C5D000480B002000007A4400007AC44A0B002077
:10C5E0000146002906D10D48407F012800D170473F
:10C5F0000020FCE7012906D10848807F012800D1EE
:10C60000F5E70020F3E7022906D10448C07F01289E
:10C6100000D1ECE70020EAE70020E8E7EC2E00205C
:10C6200010B5C046C04610BD10B511F075FA01280E
:10C6300004D112F033FF012800D110BD0020FCE727
:10C6400010B511F073FA13F099FD10BD10B511F08B
:10C65000D5FA13F0F1FF13F0B5F914F009F910BD94
:10C66000F1B584B08F480078002801D105B0F0BD45
:10C670008D48FBF72FFE441C8B492046FBF742FEFA
:10C680008948FBF727FE04461421FBF743FD0129E7
:10C6900008D186490498FBF735FE8449091D0498A2
:10C6A000FBF730FE8148FBF715FE0446214604984F
:10C6B000FCF7AAF903D27D490498FBF723FE7B48D7
:10C6C000001DFBF707FE044621460498FCF792F98B
:10C6D00004D27649091D0498FBF714FE724808300D
:10C6E000FBF7F8FD054629460498FBF723FE0446B0
:10C6F0006D490831FBF706FE6B48FBF7EBFD04467E
:10C700001421FBF707FD032908D26748FBF7E2FD78
:10C7100004461421FBF7FEFC002936D16248FBF7E2
:10C72000D9FD07466048FBF7D5FD064611361421B2
:10C730003046FBF7EFFC40003D1A2846FCF76BF84B
:10C7400004465948001DFBF7C5FD02905748001DDF
:10C75000FBF7C0FD07465548FBF7BCFD019052486A
:10C760000830FBF7B7FD00900199FBF734FE064651
:10C770003946FBF730FE05460299FBF7DBFD214603
:10C780000390FBF76DFE049022E04748FBF7A2FD03
:10C7900007464548FBF79EFD14210390FBF7BAFCC2
:10C7A00040003E1A3046FCF736F804463E48083052
:10C7B000FBF790FD06463C48001DFBF78BFD074646
:10C7C0003146FBF7B7FD05462146FBF749FE0490CD
:10C7D0003548FBF77FFD04461421FBF79BFC00293D
:10C7E00027D13148001DFBF775FD03902F48001D30
:10C7F000FBF770FD02902D48FBF76CFD07462A48B9
:10C800000830FBF767FD39460190FBF7E4FD06466B
:10C810000299FBF7E0FD05460399FBF78BFD044603
:10C820002149091DFBF76EFD1F4908310020FBF768
:10C8300069FD1D48FBF74EFDE121C900884217D96B
:10C8400019490020FBF75EFD1749091D0020FBF781
:10C8500059FD154908310020FBF754FD12490C31F0
:10C860000020FBF74FFD104910310020FBF74AFD77
:10C87000049802F06BF804460B492839FBF742FD97
:10C8800009482838FBF726FD044608493439FBF7E8
:10C8900039FD05482838FBF71DFD044604F06CFD02
:10C8A00000BFE3E65D06002064220020282200206D
:10C8B00010B500F0C7F8012807D105480078002816
:10C8C00001D1012010BD0020FCE70020FAE70000A4
:10C8D000470B002010B54C480078030018F05FF9B2
:10C8E0000A060711213141516171868E8AE00020CC
:10C8F00046490870012046490870022042490870E4
:10C9000080E014F0BBFD41480078012808D10020E8
:10C910003E49087001203E49087003203A490870DA
:10C9200070E0FFF7BFFD39480078012808D10020EA
:10C9300036490870012036490870042032490870D1
:10C9400060E002F033F831480078012808D1002077
:10C950002E49087001202E49087005202A490870C8
:10C9600050E015F0A3FC29480078012808D10020E8
:10C9700026490870012026490870062022490870BF
:10C9800040E012F0D3F821480078012808D10020B7
:10C990001E49087001201E49087007201A490870B6
:10C9A00030E011F043FF19480078012808D1002039
:10C9B00016490870012016490870082012490870AD
:10C9C00020E000F03FF801280FD1124800784028FD
:10C9D00008D040200F4908700F4B012200210D485C
:10C9E00000F094FA0920084908700BE000F02AF8DA
:10C9F000012802D100200449087003E00020024908
:10CA0000087000BF00BF10BD470B00204A0B00207C
:10CA1000490B0020A02B0020480B002010B5FFF789
:10CA200059FF00F087F810BD10B5044609F0EAFA86
:10CA3000012805D100F006F8002801D0012010BD22
:10CA40000020FCE703480078002801D1012070474E
:10CA50000020FCE75000002003480078002801D1A6
:10CA6000012070470020FCE75000002000B585B091
:10CA7000072103A818F092FF0C21684618F08EFFDA
:10CA80000021684641738173C1730174417403AA24
:10CA900003210120000308F095FD00216846417341
:10CAA000012141740021C173017403AA08214020AF
:10CAB00008F088FD03AA0921402008F083FD012227
:10CAC0000821402008F0CCFD01220921402008F077
:10CAD000C7FD002203210120000308F0D9FD114801
:10CAE0001149086001220421104812F04FFC102067
:10CAF00011F036FA14F06EFF00900D4801904021BD
:10CB000068460172552141720021817269460648CA
:10CB1000006808F029FF012202210C2000F0B2FA7F
:10CB200005B000BD0004004084000020202000402B
:10CB3000A086010010B5C5480078030018F02FF852
:10CB40000906071019C4E5FDFCFBFA007CE103208F
:10CB5000BE49087010F09CF9BD4812F08FFC73E1DB
:10CB60000320BA49087010F0AFF9B94812F086FCFA
:10CB70006AE1B748FEF7EEFF002859D0B5480068D3
:10CB800008F0E9FEB448007800283FD109F042FAE5
:10CB900001281DD1B0480078401CAF49087002F050
:10CBA0006DFF00220621AD4812F0F0FB00220321A8
:10CBB0000120000308F06CFD00220421A84812F0B7
:10CBC000E5FBA34812F05AFC0720A04908707AE060
:10CBD000A1480078401CA049087002F04FFF0022D5
:10CBE00006219E4812F0D2FB0022032101200003FF
:10CBF00008F04EFD00220421994812F0C7FB94482A
:10CC000012F03CFC0820914908705CE00020924939
:10CC1000087002F033FF002203210120000308F016
:10CC200037FD8B4812F02AFC0420884908704AE03E
:10CC300009F0E8F901282FD109F0ECF901280BD10E
:10CC400002F01CFF002084490870864812F016FC90
:10CC500006207E49087036E015F0BCFA8249096862
:10CC6000401AC8282FD902F009FF00207A4908701D
:10CC700000220621794812F089FB002203210120BD
:10CC8000000308F005FD00220421754812F07EFB28
:10CC900000206E49087016E07448008801280FD102
:10CCA00015F098FA72490968401A7249884207D902
:10CCB00000206E49088005216648006808F0B0FE33
:10CCC000032062490870BFE06148FEF743FF002877
:10CCD00017D0FFF7CBFE01220321100308F0D8FC88
:10CCE000012206215D4812F051FB052159480068D8
:10CCF00008F096FE564812F0C1FB05205349087013
:10CD000002E00420514908709EE05148FEF722FFDE
:10CD100000283CD04F480068406908281DD10421F4
:10CD20004C48006808F07CFE002206214B4812F0B7
:10CD30002DFB03E084E067E04AE02CE000220321C1
:10CD40000120000308F0A4FC00220421444812F052
:10CD50001DFB00203D4908701CE047480078402139
:10CD6000884345490870002206213C4812F00EFB1A
:10CD7000002203210120000308F08AFC0022042184
:10CD8000374812F003FB00203049087002E005200C
:10CD90002E49087058E03348FEF7DCFE002813D017
:10CDA000002206212D4812F0F1FA00220321012071
:10CDB000000308F06DFC00220421294812F0E6FA75
:10CDC00000202249087002E00620204908703BE05C
:10CDD00017F05AFD1E48FEF7BDFE002813D0FFF7DE
:10CDE00045FE01220321100308F052FC0122062116
:10CDF0001A4812F0CBFA01220421194812F0C6FA9F
:10CE00000220124908701FE017F03EFD1048FEF79F
:10CE1000A1FE002813D0FFF729FE012203211003F1
:10CE200008F036FC012206210C4812F0AFFA01226C
:10CE300004210B4812F0AAFA01200449087003E00B
:10CE400000200249087000BF00BF10BD5000002044
:10CE5000C027090084000020510000200804004081
:10CE60002020004050C300006C0000207A00002009
:10CE70006800002088130000820000207047000036
:10CE8000F8B505460F4614461E4640201649087060
:10CE90000020307028190121C903884221DC002CB0
:10CEA0001DDD881184421ADC104805801048076097
:10CEB0001048048010480660012204210F4812F037
:10CEC00065FA01220321100308F0E2FB012206218A
:10CED0000B4812F05BFA01200A490870F8BD0020E7
:10CEE000FCE70020FAE7000082000020800000201C
:10CEF0005800002072000020600000202020004028
:10CF0000080400405000002070470000F8B50746B4
:10CF10000D4614461E4660204D49087000203070B2
:10CF200028190121C90388427EDC002C7DDD88118F
:10CF300084427ADC47480580474807602846E9175D
:10CF4000890E091889118901691A444A118010460D
:10CF500000884021081A424908802046E117890EBE
:10CF600009188902090C3F4A1180E117890E091836
:10CF700089118901611A3C4A11803A4800880028C9
:10CF800027D136480088001940281ADD012037498A
:10CF9000088033480088201A84B22046E117890EA1
:10CFA000091889112F4A1180E117890E0918891172
:10CFB0008901611A2C4A1180294800882C4908806F
:10CFC00029E000202949088027480088284908804E
:10CFD00021E001202549088020480088002803D14D
:10CFE00040202349088016E01D480088201A84B29A
:10CFF0002046E117890E091889111A4A1180E11794
:10D00000890E091889118901611A174A118014487B
:10D010000088174908801748066001220421164835
:10D0200012F0B4F9012201E010E00DE00321100339
:10D0300008F02EFB01220621104812F0A7F9022069
:10D040000F4908700120F8BD0020FCE70020FAE736
:10D050008200002080000020580000207400002082
:10D0600076000020780000207C0000207E00002058
:10D0700072000020600000202020004008040040D2
:10D080005000002070B504460E4615462046002884
:10D0900005DBC206D20E01219140144A116000BF87
:10D0A0003146204617F08AFD012D0ED1204600287A
:10D0B00009DB00BF00BFC206D20E012191400C4A1D
:10D0C000116000BF00BF00BF0FE0204600280ADB50
:10D0D000C206D20E01219140054A80321160BFF391
:10D0E0004F8FBFF36F8F00BF00BF70BD80E200E0C5
:10D0F00000E100E0F7B588B0154600247F20C005A8
:10D1000007900C20069000BF09E0A0018B4A11583F
:10D110000898FBF76FFC00D805E0601CC4B20698C5
:10D12000401EA042F1DC00BF85492846FBF762FCA7
:10D130007FD884492846FBF75DFC3CD8A1017F4A93
:10D14000891848690999FBF74EF907460999FBF7D1
:10D150004AF90646A001794A801801690898FBF748
:10D1600042F903900999FBF73EF90746A101734A7A
:10D170008918C8680999FBF736F90390A0016F4A2E
:10D18000801881680898FBF72EF90190A0016B4A7E
:10D19000801841680198FBF7CDF802900399FBF7DE
:10D1A000C9F839460490FBF7C5F831460590FBF7FE
:10D1B000C1F80790BBE0A101604A8918886A099903
:10D1C000FBF711F906460999FBF70DF90590A00147
:10D1D0005A4A8018416A0898FBF705F903900999A3
:10D1E000FBF701F90646A101544A8918086A099912
:10D1F000FBF7F9F80390A001504A8018C16908981C
:10D20000FBF7F1F80190A0014C4A80188169019860
:10D21000FBF790F802900399FBF78CF8074631462C
:10D22000FBF788F804900599FBF784F807907EE0F7
:10D23000FFE745492846FBF7DDFB3CD8A1013F4A03
:10D240008918886A0999FBF7CEF806460999FBF711
:10D25000CAF80590A001394A8018416A0898FBF77E
:10D26000C2F807460999FBF7BEF80646A101334A02
:10D270008918086A0999FBF7B6F80290A0012F4AAD
:10D280008018C1690898FBF7AEF80190A0012B4AFD
:10D29000801881690198FBF74DF807460299FBF762
:10D2A00049F831460390FBF745F804900599FBF7E0
:10D2B00041F807903BE0A101204A8918C86B099901
:10D2C000FBF791F806460999FBF78DF80590A00148
:10D2D0001A4A8018816B0898FBF785F80746099968
:10D2E000FBF781F80646A101144A8918486B099991
:10D2F000FBF779F80290A001104A8018016B08989A
:10D30000FBF771F80190A0010C4A8018C16A0198DE
:10D31000FBF710F807460299FBF70CF8314603902B
:10D32000FBF708F804900599FBF704F807902846E6
:10D330000799FBF758F80BB0F0BD0000F00F002084
:10D3400000800444000098420080094410B5C046A3
:10D35000C046C046C04610BDF0B589B004460E4672
:10D360000027002006900590049003900290019001
:10D370000A2E01DA09B0F0BD0025CEE1A9006058FF
:10D380000021FBF741FB06D8A9006058FB4909685A
:10D39000FBF730FB0CD3A90060580021FBF72AFBF8
:10D3A0007ED2A9006058F6490968FBF72DFBF7D239
:10D3B0000498401CC0B20490781CC7B2022F70D1F0
:10D3C000012D49D1ED49A0680968FBF71DFB05D97E
:10D3D000EB49A0680968FBF70DFB7DD8E749E068D9
:10D3E0000968FBF711FB05D9E549E0680968FBF717
:10D3F00001FB0BD8E14920690968FBF705FB27D938
:10D40000DF4920690968FBF7F5FA21D90021E068B6
:10D41000FBF7F0FA0BD1D94920690968FBF7F4FA58
:10D4200016D9D74920690968FBF7E4FA10D9D3491E
:10D43000E0680968FBF7E8FA05D9D149E0680968AE
:10D44000FBF7D8FAC9D800212069FBF7D3FA43D1FA
:10D4500005950120069063E10F2DF8D1C749E06AD8
:10D460000968FBF7D1FA05D9C549E06A0968FBF7F5
:10D47000C1FAB2D8C149206B0968FBF7C5FA05D9D2
:10D48000BF49206B0968FBF7B5FA0ED8BB49606B42
:10D490000968FBF7B9FA2CD9B949606B096801E052
:10D4A00038E12CE0FBF7A6FA23D90021206BFBF72B
:10D4B000A1FA0BD1B149606B0968FBF7A5FA18D93D
:10D4C000AF49606B0968FBF795FA12D9AB49206B3D
:10D4D0000968FBF799FA00E0FAE005D9A849206B42
:10D4E0000968FBF787FAADD80021606BFBF782FA79
:10D4F000ADD102200690681EC0B2059010E1032F46
:10D500007EDB0D2F7CDCF01EA84261DD691C8900EA
:10D5100060589A490968FBF777FA07D9691C8900AE
:10D52000605897490968FBF765FA51D8A91C89002A
:10D53000605892490968FBF767FA07D9A91C890066
:10D5400060588F490968FBF755FA0FD8E91C890024
:10D5500060588A490968FBF757FA35D9E91C8900F0
:10D56000605887490968FBF745FA2DD9A91C89003D
:10D5700060580021FBF73EFA0FD1E91C8900605882
:10D580007E490968FBF740FA1ED9E91C89006058FA
:10D590007B490968FBF72EFA16D9A91C8900605847
:10D5A00076490968FBF730FA07D9A91C8900605849
:10D5B00073490968FBF71EFA0AD8E91C890060580C
:10D5C0000021FBF717FA03D1059501200690A7E08B
:10D5D000052D7DDBE91E8900605868490968FBF765
:10D5E00013FA07D9E91E8900605865490968FBF7F5
:10D5F00001FA6DD8291F890060586049096800E068
:10D600004EE0FBF701FA07D9291F890060585C49F1
:10D610000968FBF7EFF90FD8691F8900605857496F
:10D620000968FBF7F1F935D9691F89006058544939
:10D630000968FBF7DFF92DD9291F890060580021FF
:10D64000FBF7D8F90FD1691F890060584B49096869
:10D65000FBF7DAF91ED9691F890060584849096843
:10D66000FBF7C8F916D9291F890060584349096892
:10D67000FBF7CAF907D9291F890060584049096892
:10D68000FBF7B8F947D8691F890060580021FBF7FC
:10D69000B1F940D102200690A81EC0B205903FE02B
:10D6A0000E2F38D13549A06B0968FBF7ADF905D9C4
:10D6B0003349A06B0968FBF79DF910D82F49E06B3F
:10D6C0000968FBF7A1F907D92D49E06B096800E06B
:10D6D00021E0FBF78FF902D80320069020E02749CC
:10D6E00020680968FBF790F905D925492068096881
:10D6F000FBF780F90FD8214960680968FBF784F9C6
:10D7000005D91F4960680968FBF774F903D804203C
:10D71000069005E00027681CC5B2B54200DA2DE688
:10D7200000BF0698002863D1089020E0002515E08E
:10D730006A1C9200A158AA00A058FBF765F90BD209
:10D74000A80020580390681C80002058A900605051
:10D75000691C890003986050681CC5B2701E089946
:10D76000401AA842E4DC0898401CC0B20890701E21
:10D7700008998842DADC022007900EE03C0600207F
:10D78000400600200798800021580298FAF7D2FD41
:10D7900002900798401CC0B20790B01E07998842BB
:10D7A000F0DC301FFBF72CF8014600900298FAF7E6
:10D7B00057FE029009F09AFA0A2818D10498032813
:10D7C00015DB00210298FBF71FF904D29449029857
:10D7D000FBF710F909D300210298FBF70BF906D2E9
:10D7E00090490298FBF710F9F9D20020029014E159
:10D7F000069801284DD10598401CC0B205900598A7
:10D80000301AC6B2002509E0059828188000215872
:10D810000298FAF78FFD0290681CC5B2B542F3DB9F
:10D820003046FAF7F8FF014600900298FAF718FE22
:10D83000019000210198FBF7E7F804D27A4901989A
:10D84000FBF7D8F809D300210198FBF7D3F819D2D8
:10D8500076490198FBF7D8F814D27548FAF73AFDE3
:10D86000962808D872480C30FAF734FD962802D86A
:10D8700000200290D1E08321C9050298FAF7F0FD5B
:10D880000290CAE08321C9050298FAF7E9FD0290E7
:10D89000C3E00698022845D1002507E0A8002158DA
:10D8A0000298FAF747FD0290681CC5B205988542B8
:10D8B000F4DB0598FAF7AFFF014600900298FAF7FB
:10D8C000CFFD019000210198FBF79EF804D2564944
:10D8D0000198FBF78FF809D300210198FBF78AF82C
:10D8E00019D252490198FBF78FF814D25048FAF731
:10D8F000F1FC962808D84E480C30FAF7EBFC962835
:10D9000002D80020029088E08321C9050298FAF726
:10D91000A7FD029081E08321C9050298FAF7A0FDD6
:10D9200002907AE0069803283AD1E16BA06BFAF7EF
:10D9300001FD0290012189070298FAF791FD0190FB
:10D9400000210198FBF760F804D237490198FBF7F2
:10D9500051F809D300210198FBF74CF819D233494B
:10D960000198FBF751F814D23148FAF7B3FC962826
:10D9700008D82F480C30FAF7ADFC962802D80020C2
:10D9800002904AE08321C9050298FAF769FD0290E6
:10D9900043E08321C9050298FAF762FD02903CE05A
:10D9A0000698042839D161682068FAF7C3FC029010
:10D9B000012189070298FAF753FD0190002101988F
:10D9C000FBF722F804D218490198FBF713F809D3A2
:10D9D00000210198FBF70EF819D214490198FBF7C2
:10D9E00013F814D21248FAF775FC962808D8104894
:10D9F0000C30FAF76FFC962802D8002002900CE059
:10DA00008321C9050298FAF72BFD029005E08321D6
:10DA1000C9050298FAF724FD02900298AAE40000D2
:10DA20008FC2753D8FC275BD0AD7233D0AD723BD6E
:10DA300048220020FEB504460E4600200290142E17
:10DA400000DD1426276820680190002518E0A80052
:10DA500021580198FAF7D8FF02D2A8002058019067
:10DA6000A80021583846FAF7C5FF01D2A800275868
:10DA7000A80021580298FAF75DFC0290681CC5B214
:10DA8000B542E4DB39460298FAF7A5FC009001990B
:10DA9000FAF7A1FC0290B01EFAF7B2FE0146009020
:10DAA0000298FAF7DDFCFEBDF3B597B00E460020F4
:10DAB000169014901390002515E0AA001799895824
:10DAC0002846EA0F12185210920003AB9950691CB5
:10DAD0008A0017998958EA0F1218521092000BAB5E
:10DAE0009950A81CC5B2B542E7DB00253AE00024F6
:10DAF0002FE0621C920003AB9958A2009858FAF7E5
:10DB000083FF0DD2A00003A908581590601C800067
:10DB10000858A10003AA5050611C89001598505064
:10DB2000621C92000BAB9958A2009858FAF76CFF50
:10DB30000DD2A0000BA908581590601C8000085851
:10DB4000A1000BAA5050611C890015985050601C10
:10DB5000C4B2F10F89194910491E491BA142C8DC02
:10DB6000681CC5B2F10F89194910491EA942BEDCD3
:10DB700001270FE0B80003AA11581498FAF7DAFB4E
:10DB80001490B8000BAA11581398FAF7D3FB13900E
:10DB9000781CC7B2F10F89194910491EB942E9DC56
:10DBA000301FFAF72DFE029013991498FAF7C2FB72
:10DBB00001900299FAF754FC1690169819B0F0BD2E
:10DBC00010B50020C7494870022088700021C54860
:10DBD000C17006210171002141718171DD20C149AF
:10DBE000C871E521BF480172D6214172CA218172F4
:10DBF000BD49C172090A01730020BA494873002166
:10DC0000B8488173C173012101740721417419213E
:10DC100081740020B349C8740021B2480175417570
:10DC2000012181750721C175992101760F21417666
:10DC3000002181760020AB49C876012008770721B2
:10DC4000A8484177192181770021C17730211C3004
:10DC5000017101214171022181710721C1711921D5
:10DC6000017201460931A148FAF74CFB01219D4898
:10DC700020304172002109304170142181708C21C3
:10DC8000C170052108380173002141739849801C37
:10DC90000173090A41730121C01E4174042111302E
:10DCA0004170632181707421C1706E210171622104
:10DCB000417151210F3041714921401D41704E2168
:10DCC00081704721C17044210171412141714F216F
:10DCD00081714A21C1714921017243214172482158
:10DCE00081722D21C1724E210173472141734E2152
:10DCF00081734221C1730021401F4175153041706D
:10DD00008170C170017141718171153801771C30CA
:10DD100041708170C1700171417181710121001DDB
:10DD2000C1700021C01C41708170C170017133212C
:10DD30004171782181710021C01E81720421C1725C
:10DD400018210B30417000218170AA21C17000217F
:10DD500001710B3801744174014612310020FAF749
:10DD6000D1FA604976310020FAF7CCFA5D497A3170
:10DD700001200004FAF7C6FA5A497E310120000456
:10DD8000FAF7C0FA5749823101200004FAF7BAFACB
:10DD90005449863101200004FAF7B4FA51498A3116
:10DDA00001200004FAF7AEFA4E498E31012000043A
:10DDB000FAF7A8FA5A214B4880308174C1740020C8
:10DDC00004E00022474994310A54401C2028F8DB23
:10DDD0000F21444880300175AA2114300172552169
:10DDE000817211214173232181737F21C17302212B
:10DDF000017432214174002181740521C1740175BF
:10DE000000214175072181751421C175D2210C3083
:10DE10000175002141753749801C0175090A41755A
:10DE20000821801E0176102141760F218176042180
:10DE3000C17605211B30417001211B384177E1215A
:10DE4000C900801C0177090A417728211E30017022
:10DE500000214170811C0020FAF754FA002121486A
:10DE6000C0308171C171014608310020FAF74AFAC9
:10DE70001C49D0310020FAF745FA1A49D4311E481E
:10DE8000FAF740FA1749D8310020FAF73BFA15495A
:10DE9000DC310020FAF736FA00211248D030018236
:10DEA0004182014614311548FAF72CFA0D48943096
:10DEB000017C763001717638417C7630417176385C
:10DEC000817C7630C1707638C17C7630817176384D
:10DED000017D73380173090A41737330417D7630D7
:10DEE000C17110BDA02B002033160000B80B00003C
:10DEF000520300001A2B0000E0D14D00000040400A
:10DF000010B516F009FA0B480078002804D0012853
:10DF100003D0022807D103E009E000F017F806E07B
:10DF200000F0A4F903E000200249087000BF00BF20
:10DF300010BD0000AA0B002003480078002801D182
:10DF4000012070470020FCE7AB0B002010B5BB4858
:10DF5000007808287CD007DC030016F020FE0812A9
:10DF6000447C7C5B8EAAB07C162872D004DC092825
:10DF700070D00A286FD1F7E017286DD01828F9D192
:10DF80001DE101F067FD01282CD1AD48C07A401C8D
:10DF9000AB49C872C87A0A21FAF7D2F8C8B2A849C0
:10DFA000C872E1210901242011F0C0F9A5480088B8
:10DFB000401CA44908800D2000F08EFD0002000ED8
:10DFC000AA2801D10EF046FF55219F4881702320D9
:10DFD00000F08AFD482000F087FD0CF03FF9012099
:10DFE000964908701BE10CF041FD002803D0042085
:10DFF000924908700DE00CF02FFD002809D09348DD
:10E000000DF0AAFB9249252011F090F904208B49CC
:10E01000087004E10CF02AFD00281ED001F026FD56
:10E02000092806D102208B49087006208349087010
:10E0300022E08948027BC37A10021843014601227C
:10E040008548C01D0BF018FF05207C49087013E0BF
:10E050004FE0A2E060E0DEE0A9E07C480078A5287F
:10E0600004D02520FDF706FD002805D1F1207949CF
:10E070000870062071490870D1E00120FEF7B0FA5F
:10E08000002806D001207349087006206B490870EB
:10E090000EE06E480078A52804D02520FDF7EAFCA4
:10E0A000002805D1F1206B490870062063490870EB
:10E0B000B5E002F009FA072060490870AFE0674A4E
:10E0C00067496448007801F035FF01F091FD0128AF
:10E0D0000ED101F0A7FD012803D10820574908708F
:10E0E00006E03221262011F021F90A205349087058
:10E0F00095E00CF0B1FC01280DD1544B012257489A
:10E10000018857480EF05CF96421262011F00EF9C1
:10E1100009204A49087082E0232000F0D3FC01283E
:10E1200004D02620FDF7A6FC00280FD1232000F004
:10E13000DBFC022047490870002143484170012060
:10E140000BF0FCFE07203D4908700CE03F480078CA
:10E15000A52808D132213C48417003203D49087070
:10E160000720364908705AE0482000F0ABFC002830
:10E1700006D0482000F0B8FC3221262011F0D6F855
:10E180002620FDF777FC002806D101F0BBFC012812
:10E1900002D116202949087041E00CF05DFC0028EE
:10E1A00004D012F023FE17202449087037E00CF049
:10E1B00053FC002802D01820204908702FE0FEF7F9
:10E1C00041FC012826D10D2000F086FC0002000E43
:10E1D000AA280FD100211C487638817000202149DF
:10E1E00008700B460122962117487438FEF78EFE00
:10E1F00000F0C8FE0BF0DEFF15F054FDFDF730FE19
:10E20000FDF720FD00211048817000200B490870A7
:10E210001549087003E000200849087000BF00BFDE
:10E22000FFF78AFE002807D12420FDF723FC0028F1
:10E2300002D118200149087010BD0000AB0B00206E
:10E24000C72E0020B20B0020AA2C0020A20B002019
:10E25000B80B0000B40B0020A02B0020A00B002066
:10E26000C72C0020B80B0020AA0B002010B5FD48D9
:10E270000078030016F093FC190E3D5EF175A0DBEB
:10E28000F2EFEEEDF1F1ECEBEAE9E8E7E6E5E4E3E5
:10E29000E2E1F10001F0DEFB012829D1F248C07A69
:10E2A000401CF149C872C87A0A21F9F749FFC8B27F
:10E2B000ED49C872E1210901242011F037F8EB483B
:10E2C0000088401CE94908800D2000F005FC000290
:10E2D000000EAA2801D10EF0BDFD232000F004FCA1
:10E2E000482000F001FC0BF0B9FF0120DD49087067
:10E2F00090E20CF0BBFB00280DD01CF055FC002870
:10E3000005D00DF001FE0220D649087011E004206E
:10E31000D44908700DE00CF09FFB002809D0D448C8
:10E320000DF01AFAD349252011F000F80420CD4948
:10E3300008706FE20CF090FB012811D11CF034FC46
:10E34000012803D10520C749087009E0C8480DF02D
:10E3500003FAC849252010F0E9FF0420C1490870DC
:10E3600058E20CF083FB002812D0002104201EF09C
:10E37000F9F9C148027BC37A100218430146012211
:10E38000BD48C01D0BF078FD0520B649087012E0AD
:10E39000B7480078A52804D02520FDF76BFB00289E
:10E3A00009D1012104201EF0DDF9F120B3490870E4
:10E3B0000620AC4908702DE20120FEF711F9002873
:10E3C00025D01CF0F1FB012805D1AC4908700620CE
:10E3D000A44908702AE007201CF042FE01280FD152
:10E3E000002107201EF0BEF901201CF039FE044672
:10E3F0002146262010F09AFF0A209A49087015E05D
:10E4000001209E4908700620964908700EE0984841
:10E410000078A52804D02520FDF72CFB002805D185
:10E42000F1209649087006208E490870F2E102F04A
:10E430004BF807208B490870ECE1BBE1B2E1A7E1A2
:10E440008BE180E15EE142E12EE1F8E0F1E0D8E02D
:10E45000B4E059E033E01FE000E0D7E1884A8949A1
:10E460008648007801F05EFE01F0CCFB012812D155
:10E4700001F0DEFB012803D108207A4908700AE088
:10E4800001201CF0EDFD04462146262010F04EFF31
:10E490000A2074490870BDE10CF0DEFA01280DD1A4
:10E4A000734B01227648018876480DF089FF64217C
:10E4B000262010F03BFF09206A490870AAE12320BA
:10E4C00000F000FB012804D02620FDF7D3FA002835
:10E4D0000FD1232000F008FB00206B4908700220B8
:10E4E0006649087000216948417007205D4908703D
:10E4F00009E05F480078A52805D103205F4908702E
:10E5000007205849087085E1482000F0DBFA002810
:10E510000BD0482000F0E8FA01201CF0A1FD0446D1
:10E520002146262010F002FF47E02620FDF7A2FA40
:10E53000002842D101F0E6FA01283ED101F08AFA22
:10E5400001280FD14848C07A401C4749C872C87A90
:10E550000A21F9F7F5FDC8B24349C87205204149BF
:10E5600008702AE01CF020FB012815D147487638B6
:10E57000007B8021084000280AD044487638007B80
:10E580008007800F002803D014203649087014E05B
:10E590000D203449087010E006201CF061FD0128B0
:10E5A00008D104201CF05CFD002803D10D202D496A
:10E5B000087002E016202B4908702BE101F0A2FA46
:10E5C00001281DD10CF048FA002819D000202B4951
:10E5D00008702E482238827E437E1002184301467E
:10E5E00002222A480D380BF047FC01201CF038FDB0
:10E5F00004462146262010F099FE0E201949087085
:10E6000008E10220FDF7ECFF002806D001201B499D
:10E6100008700F20134908700AE02620FDF72AFA37
:10E62000002805D1F120154908700F200D49087008
:10E63000F0E001F03DFF10200A490870EAE0104ABE
:10E6400010490E48007801F0F9FA01F0C7FA0128E4
:10E6500029D101F0E1FA01281AD1112001490870ED
:10E6600021E00000AB0B0020C72E0020B20B0020E1
:10E67000A20B0020B80B0000A02B0020B40B002040
:10E68000A00B0020C72C0020B50B0020AA2C0020D6
:10E6900001201CF0E5FC04462146262010F046FE31
:10E6A000132063490870B5E00CF0D6F901280DD1AC
:10E6B000604B02226048018860480DF081FE3221E3
:10E6C000262010F033FE122059490870A2E02320C2
:10E6D00000F0F8F9012809D1232000F005FA022002
:10E6E000574908701020524908700AE02620FDF7AB
:10E6F000C1F9002805D103205149087010204C4968
:10E70000087087E0482000F0DDF9002803D115F0FB
:10E71000CFFA01280AD1482000F0E6F901201CF0C8
:10E720009FFC04462146262010F000FE2620FDF71F
:10E73000A1F9002806D101F0E5F9012802D116203F
:10E740003B49087066E00CF087F9012804D10DF010
:10E75000C7FB1520364908705CE00CF07DF90128F4
:10E7600015D11CF021FA02280ED101213548017281
:10E7700015F098FAFDF774FBFDF764FA00202C49B8
:10E7800008703149087002E016202949087041E0FC
:10E790000CF062F9002804D012F028FB172024495D
:10E7A000087037E00CF058F9002802D018202049F2
:10E7B00008702FE0FEF746F9012826D10D2000F061
:10E7C0008BF90002000EAA280FD100211D487638CF
:10E7D000817000201D4908700B46012296211948BE
:10E7E0007438FEF793FB00F0CDFB0BF0E3FC15F063
:10E7F00059FAFDF735FBFDF725FA002111480172A2
:10E8000000200B4908701049087003E000200849F7
:10E81000087000BF00BFFFF78FFB002807D124203E
:10E82000FDF728F9002802D118200149087010BD11
:10E83000AB0B0020A20B0020A00B0020C72C002057
:10E84000B40B0020AA2C0020AA0B0020B80B00203B
:10E85000F0B58BB005460E4600242A480A900020E9
:10E860000990202101A8F9F70EFD274F012D0ED0A8
:10E87000022D0CD0042D0AD0062D08D0082D06D06C
:10E880000C2D04D00420099009980BB0F0BD1E484F
:10E89000006A01214902884371020122520211409B
:10E8A000084319490862002407E0A00017490858E6
:10E8B0006843A10001AA5050641C082CF5D3002421
:10E8C0001CE010480A9011E00A98411E0A910028A5
:10E8D0000AD00F480C49C8620E48C862A00001A9BE
:10E8E0000858A100785001E00720CEE7A000385872
:10E8F000A10001AA51588842E6D1641C082CE0D33B
:10E900000998C2E7FFFFFF0000000240E0D50200C7
:10E910005A5A0000A5A5000010B501460020084A7B
:10E92000084BDA62084ADA621A46126A0C239A43E2
:10E930008B000C2423401A43024B1A6210BD0000C6
:10E940005A5A000000000240A5A5000070B5044618
:10E95000472109062046FAF757F801D2002070BD7A
:10E960008F21C9052046F9F73EFD0546F9F77CFFE2
:10E97000F5E7000010B5002408F0D4F80446094873
:10E980000088201A80B208490860064804800846BA
:10E99000006805210902884203D3032000020249CE
:10E9A000086010BDB8060020B406002070B53D48D0
:10E9B0000078002806D0012805D0032862D0062858
:10E9C0006AD123E06CE0FEF73DF801281DD13648FE
:10E9D000007840280FD0482234493548F9F73AFCEE
:10E9E000344B48220D2189013148FEF78FFA03206C
:10E9F0002C49087009E02F4B48222D490D20800139
:10EA0000FEF73EFA06202749087049E0FEF71AF89B
:10EA1000012836D1012500241EE0A100244A8818CF
:10EA2000F9F758FC0021C943884201D1002515E0BF
:10EA3000A1001F4A8818F9F74DFC1F49884207D8E2
:10EA4000A1001B4A8818F9F745FC1C49884201D2ED
:10EA5000002503E0601CC4B2122CDEDB00BF002DD9
:10EA60000BD1482211491248F9F7F4FB114B482207
:10EA70000D2189010E48FEF749FA03200949087063
:10EA800000BF0DE0FDF7DEFF012804D10C4908703E
:10EA900000200449087003E000200249087000BF0C
:10EAA00000BF70BD490B0020A02B002064DA0200DB
:10EAB00043420020480B00209919010066E600003F
:10EAC0004A0B002001465B2902DA0248405C70478D
:10EAD0000020FCE7C83C002001468800014A10588D
:10EAE00070470000FC2A002001465B2904DA002060
:10EAF000024A5054012070470020FCE7C83C002027
:10EB000070B50646002406F0C3F8C4B2E007C00F93
:10EB100000280ED0A548007802218843801CA34914
:10EB200008700846C0784021884340309F49C8702B
:10EB30000BE09E480078022188439C4908700846F3
:10EB4000C078402188439949C8700220204002289B
:10EB50000ED19648007820218843203093490870D0
:10EB60000846C0782021884320309049C8700BE0C7
:10EB70008E480078202188438C4908700846C07868
:10EB8000202188438949C87004202040042807D1E7
:10EB90008648407840084000401C8449487005E0A1
:10EBA0008248407840084000804948700820204052
:10EBB000082807D17D48407804218843001D7B49FF
:10EBC000487005E0794840780421884377494870C7
:10EBD00020202040202807D1744840780221884313
:10EBE000801C7249487005E07048407802218843D3
:10EBF0006E4948704020204040280ED16B48007874
:10EC000040084000401C694908700846C0788021CF
:10EC1000884380306549C8700BE06448007840083C
:10EC20004000624908700846C078802188435F49E7
:10EC3000C8708020204080280ED15C480078402198
:10EC400088434030594908700846C07804218843F9
:10EC5000001D5649C8700BE0544800784021884395
:10EC6000524908700846C078042188434F49C8704B
:10EC7000FCF790FF012807D14C48407810218843C9
:10EC800010304A49487005E04848407810218843D0
:10EC9000464948701020204010280ED14348007883
:10ECA000082188430830414908700846C07810217F
:10ECB000884310303D49C8700BE03C48007808217B
:10ECC00088433A4908700846C0781021884337497C
:10ECD000C8700EF09BF90A2807D1344840782021EB
:10ECE000884320303149487005E030484078202181
:10ECF00088432E4948702D484078C02188432B49CD
:10ED000048700FF00BFE01280ED12848007804212E
:10ED10008843001D254908700846C07808218843AB
:10ED200008302249C8700BE020480078042188434D
:10ED30001E4908700846C078082188431B49C870DE
:10ED4000FCF7EEFE012807D11848407808218843D7
:10ED500008301649487005E0144840780821884377
:10ED6000124948701148C07840084000401C0F49C3
:10ED7000C8700846807840084000401C8870092010
:10ED80001CF06EF9094989780843084988700EF02B
:10ED900057F90546C00F4019C005000E0349087118
:10EDA00005223046F9F756FA70BD0000F012002037
:10EDB00003480078002801D1012070470020FCE7BB
:10EDC000000F002010B50DF0DDF813F0E5FA10BDCE
:10EDD0005B2802DA0121014A11547047C83C002027
:10EDE00070B504460E460025FE2020706070682035
:10EDF000A0701020E0705E484078102809D100BF54
:10EE000004E05C48415D281D21546D1C072DF8DB92
:10EE100024E05948407801280DD100205649487017
:10EE2000002505E05448801C415D281D21546D1CBF
:10EE3000072DF7DB09E0002505E04E480E30415D67
:10EE4000281D21546D1C072DF7DB494840781128F7
:10EE500004D14948417A201DFCF75AFA44484078C9
:10EE6000492811D006DC11280BD045280AD04628A5
:10EE70004CD108E0512808D0542807D0642845D147
:10EE800005E000BF00BF00BF00BF00BF00BF3848A3
:10EE90008078E07239480078001D2073344800798A
:10EEA000607333484079A07331488079E07330480B
:10EEB000007A2074002505E03148415D2846113074
:10EEC00021546D1C2D4800888542F5DB2848407888
:10EED000912805D12648017A20461130FCF718FA0E
:10EEE0002348027A207B0B30C1B2A01C0FF0E6FD54
:10EEF00022490988113160541621204800881230B7
:10EF000021541E480088133030802FE01848807844
:10EF1000E0721A480078C01C2073154800796073AD
:10EF200013484079A07312488079E073002505E00A
:10EF30001348415D2846103021546D1C0F4800884D
:10EF40008542F5DB207B0B30C1B2A01C16F0FCF82B
:10EF50000A49098810316054162108480088113088
:10EF60002154064800881230308000BF00BF70BDB9
:10EF70006F460020F52B002065460020001400207D
:10EF80007C4600201FB54020AB490860AB48F9F72C
:10EF9000A1F9A9494860A948001DF9F79BF9A649BC
:10EFA0008860A6480830F9F795F9A349C860A348D6
:10EFB0000C30F9F78FF9A0490861A0481030F9F733
:10EFC00089F99D4948619D481430F9F783F99A49B8
:10EFD00088619A481C30F9F77DF99749C8619748CC
:10EFE0007238007F95497239497F09020843934975
:10EFF0007239897F090408438F4908628F4856385F
:10F00000007A8E495639C979090208438B49563925
:10F010008979090408438849486289488862874891
:10F020001238C07885490F39497809020843834965
:10F030000F3989780904084380490F39C9780906CE
:10F0400008437D49C8627D480F3800797B490F39F4
:10F0500049790902084379490F3989790904084334
:10F060007549086375480E30007D7449223149782E
:10F0700009020843714922318978090408436F491C
:10F080002231C978090608436B4948636B4822302E
:10F0900000796A49223149790902084367492231D6
:10F0A00089790904084365492231C9790906084369
:10F0B0006149886361482230007A60492231497A87
:10F0C000090208435D492231897A090408435B49F2
:10F0D0002231C97A090608435749C8635748223084
:10F0E000007B56492231497B0902084353492231AA
:10F0F000897B0904084351492231C97B0906084329
:10F100004D4908644D487238C07F4C4956390979D9
:10F1100009020843494956394979090408434649CF
:10F12000486446481830F9F7D5F84349886468467A
:10F13000FFF7E6FC01990098039102906946487A2E
:10F14000897A090208433C4948653C482E30807D55
:10F150003A494431497809020843374988653748B4
:10F160002E30417D027D080210433349C865334883
:10F170002E30007E086631482E30407E48662F488B
:10F18000723880782D497239C978090208432B49B1
:10F1900072390979090408432849723949790906FD
:10F1A00008432549886725480E30807CC867234876
:10F1B0000E30C17C20488030016020487238417890
:10F1C0001D48803041601D482E30817E1A488030B5
:10F1D00081601A483030417F027F0802104316498F
:10F1E0008031486115484E3041780278080210435A
:10F1F0001149803188610AF0F5FC0F498031C861FE
:10F200000E482230017C763001717638417C7630B0
:10F2100041717638817C7630C1707638C17C763029
:10F2200081717638017D73380173090A4173733037
:10F23000417D7630C1711FBDFC2A0020122C0020B8
:10F24000050026F200200149087070477413002061
:10F250000020014908707047031400200020014974
:10F26000087070475414002030B589B004460D462C
:10F2700011488178684681750F48017968460176A2
:10F280000D484179684641760B48C17A6846C17796
:10F2900009488179684681760748C1796846C17610
:10F2A00006480088064901AA31C2009105A80FC886
:10F2B00000F008F809B030BD674500206613002053
:10F2C00067430020FFB581B00D9F0B9E0C9C00256D
:10F2D000FE20207060706820A0701020E07000BFD9
:10F2E00004E05848415D281D21546D1C072DF8DBB2
:10F2F00068468079E0726846C07B2073FB2E45DC4F
:10F30000301D60736846007AA0736846407AE073E7
:10F310006846807A20746846C07A60743246204617
:10F3200012300A99F8F796FF6846C07BC007C00FF5
:10F3300000280FD0627B444B21460E310020F9F7A4
:10F340000EFD607BC117090F09180911491C090737
:10F35000090E61730021607B0E302154022509E003
:10F36000607B0E30205C615D4018C1B2607B0E3066
:10F3700021546D1C607B0E30A842F1DC1621607BAD
:10F380000F302154607B1030388058E0301D81B23E
:10F39000009168460078607368464078A0736846BC
:10F3A000007AE0736846407A20746846807A607418
:10F3B0006846C07AA0743246204613300A99F8F79E
:10F3C00049FF6846C07BC007C00F002816D06946B9
:10F3D0000A881D4B21460F310120F9F7C0FC694610
:10F3E0000888C117090F09180911491C09050A0CD9
:10F3F00000926946487860730878A07300216846D7
:10F4000000880F30215402250BE0684600880F3039
:10F41000205C615D4018C1B2684600880F302154FD
:10F420006D1C684600880F30A842EEDC1621684645
:10F43000008810302154684600881130388005B0AB
:10F44000F0BD0000032C002053130020FFB581B055
:10F450000A9F0B9C00250026FE202070607068200B
:10F46000A0700220E070201D1BF048FE00BF06E0E7
:10F470002248415D284615302154681CC5B2062D2E
:10F48000F6DB6846407BE076684680792077684600
:10F49000C07A6077009768460078A0776846407821
:10F4A000E0773A46204620300499F8F7D3FE002151
:10F4B000684600882030215402260CE06846008807
:10F4C0002030205CA15D4018C1B268460088203021
:10F4D0002154701C86B2684600882030B042EDDCB2
:10F4E0001621684600882130215468460088223061
:10F4F00081B20C98018005B0F0BD0000032C002003
:10F500000148007870470000B40300201CB50721B3
:10F51000684616F043FA012168464170C1706A4698
:10F520000221C02006F04EF803220221C02006F07E
:10F530001FF8012203210846FDF7A4FD1CBD0000B1
:10F5400010B500F00FF91348F8F7C4FE12498842CD
:10F5500005D1002203210A20FDF794FD0AE00D48A1
:10F56000F8F7B8FE0D49884204D1002203210B2090
:10F57000FDF788FD0748F8F7ADFE03210161054856
:10F58000F8F7A8FE142101600021072012F05AFAB2
:10F5900010BD0000481C002000080040004800404A
:10F5A00010B500F025F81148F8F794FE00694021E5
:10F5B000884344180D48F8F78DFE04610B48F8F7AE
:10F5C00089FE00692021884344180848F8F782FE24
:10F5D00004610648F8F77EFE006904218843041D93
:10F5E0000248F8F777FE046110BD0000481C0020B7
:10F5F00038B580200EF0B4FC00F06AF80121072035
:10F6000012F020FA2F493048F8F77CFE2D48F8F721
:10F6100061FE00684021884304462A48F8F75AFEF4
:10F6200004602849091D0020F8F76CFE25490831BF
:10F630000420F8F767FE234910310220F8F762FE34
:10F640001021684601701F481030F8F743FEC1B220
:10F65000684641701B480830F8F73CFEC1B2684666
:10F66000C1701848001DF8F735FEC1B268468170B8
:10F670001448F8F72FFE0446694611F05DFB114867
:10F68000F8F728FE1149884205D1012203210A20FA
:10F69000FDF7F8FC0AE00B48F8F71CFE0A4988421F
:10F6A00004D1012203210B20FDF7ECFC0548F8F7FB
:10F6B00011FE00684021884344180248F8F70AFE0A
:10F6C000046038BD481C002000480040000800408D
:10F6D0001CB50721684616F061F9002168464170A3
:10F6E0006A46C02005F06EFF02220021C02005F00E
:10F6F000B7FF01220021C02005F0CAFF01211848F0
:10F7000011F034FB6A460121C02005F05BFF0222A4
:10F710000121C02005F0A4FF00220121C02005F036
:10F72000B7FF6A460421C02005F04CFF02220421E5
:10F73000C02005F095FF00220421C02005F0A8FF9D
:10F7400001216846417001716A460321C02005F01D
:10F7500039FF02220321C02005F082FF1CBD0000FA
:10F76000004800401CB50721684616F017F9002034
:10F77000694648706A460121C02005F023FF002237
:10F780000121C02005F06CFF00220121C02005F0FE
:10F790007FFF6A460421C02005F014FF00220421E7
:10F7A000C02005F05DFF00220421C02005F070FF9D
:10F7B0006A460321C02005F005FF00220321C02076
:10F7C00005F04EFF00220321C02005F061FF6A46CC
:10F7D0000021C02005F0F6FE00221146C02005F0F1
:10F7E0003FFF01220021C02005F052FF1CBD000098
:10F7F0000148007870470000BA0600200020014947
:10F8000008707047BA06002001200149087070474F
:10F81000BA06002070B504460025552C03D10EF021
:10F820005BFF054613E0012C04D1012005F0BAF975
:10F8300005460CE0022C04D1022005F0B3F9054680
:10F8400005E0032C03D1032005F0ACF9054628465A
:10F8500070BD000070B504460025112C12D13A4845
:10F860000EF01CFF00280BD0374800780004054339
:10F87000354840780002054333488078054361E00D
:10F88000324D5FE0222C12D131480EF007FF0028E4
:10F890000BD02F480079000405432D484079000221
:10F8A00005432B48807905434CE0284D4AE0012C64
:10F8B00004D10020FFF710F9054643E0022C04D1E3
:10F8C0000A20FFF709F905463CE0042C04D10B207F
:10F8D000FFF702F9054635E0032C04D10C20FFF7B1
:10F8E000FBF805462EE0052C04D106200EF0FCFAAC
:10F8F000054627E0062C04D107200EF0F5FA054650
:10F9000020E0072C04D108200EF0EEFA054619E09D
:10F91000082C04D109200EF0E7FA054612E0092C64
:10F9200004D10A200EF0E0FA05460BE00A2C04D1BF
:10F930002720FFF7D1F8054604E00B2C02D11CF07C
:10F9400079FF0546284670BDAC070020EEEEEE00BC
:10F95000B307002070B50646002423480578012E21
:10F9600027D108202840082801D1044303E00821BA
:10F9700020468843044604202840042801D104433B
:10F9800003E0042120468843044602202840022840
:10F9900001D1044303E0022120468843044640206D
:10F9A0002840402802D1012004431AE06408640082
:10F9B00017E0022E15D110202840102801D1044351
:10F9C00003E0102120468843044601200AF0B2FAE1
:10F9D000002802D08020044303E080212046884391
:10F9E0000446204670BD00009707002038B5044645
:10F9F0000025022C03D105F007FA054622E0012C70
:10FA000004D10C2005F000FA05461BE00A2C04D1B5
:10FA10000A2005F0F9F9054614E0042C04D104206D
:10FA200005F0F2F905460DE0072C04D1072005F09A
:10FA3000EBF9054606E00E2C04D112F0EDF900902A
:10FA4000009838BD2846FCE702461068C840C00749
:10FA5000C00F70470448807A0349C97A884201D0B0
:10FA6000012070470020FCE7C72E00200248C07A22
:10FA70000149085C70470000C72E0020024800784A
:10FA80000249096808707047820000206000002069
:10FA90000148007870470000A404002010B58020C1
:10FAA0000EF052FA04466006040E40200EF04CFAA6
:10FAB00004436006040E20200EF046FA044360065C
:10FAC000040E10200EF040FA04436006040E0820D5
:10FAD0000EF03AFA04436006040E04200EF034FAE5
:10FAE00004436006040E02200EF02EFA0443600662
:10FAF000040E01200EF028FA04436006040E20468E
:10FB000010BD00000148007870470000050F00207C
:10FB10000148007870470000700900200148407AD1
:10FB200070470000333A0020F7B582B00E46154604
:10FB300002981BF083FA0446002700200190A000E1
:10FB40002349085C1F281FD122480EF0A7FD214839
:10FB50000178214881701F4841781F48801C4170FE
:10FB60001C4881781C48801C81701A4801791A4809
:10FB7000801CC170174841791748801C01711548D5
:10FB800081791548801C4171FF2C1ED0A0001049BE
:10FB900040184078B04218D1A000401880780190F9
:10FBA000002709E00198411CC9B201910A49603956
:10FBB000085C28706D1C7F1CA00005494018407827
:10FBC000B842EFDC012005B0F0BD0020FBE70000EB
:10FBD000040A0020500A0020842A002003480078EC
:10FBE000002801D1012070470020FCE77513002098
:10FBF00003480078002801D1012070470020FCE76D
:10FC00007713002003480078002801D101207047B5
:10FC10000020FCE7721400200148007870470000C3
:10FC20007613002001480078704700007813002008
:10FC3000014800787047000073140020F0B591B0BF
:10FC400005460E461746012D7ED10020069006205F
:10FC500005F0DAF880B2B0490870000A487009204F
:10FC600005F0D2F880B2AC498870000AC87012F072
:10FC7000D3F8059000210598F8F7BCFE1BD2E907E0
:10FC8000059848400590A5490598F8F7ACFB04464F
:10FC9000F8F7EAFD81B2A0480171090A41710146F5
:10FCA0004879097900020843E90308439A49087131
:10FCB000000A487115E099490598F8F794FB044645
:10FCC000F8F7D2FD80B294490871000A487148796A
:10FCD0000979000208434104490C8F480171090A5F
:10FCE000417100208C498871C8710A2005F08CF898
:10FCF000044689490831F8F705FB87490C318848E3
:10FD0000F8F700FB8748F8F7E5FA87490390F8F71A
:10FD10006AFB0490F8F7A8FD04467F491031F8F714
:10FD2000F1FA804914394A7C0B7C110219430846C8
:10FD300079491431F8F7E6FA774918310020F8F7D5
:10FD4000E1FA09F057FF00E0DDE0001272490877A0
:10FD500009F050FFC1B270484177090A81770DF070
:10FD60006FF96D49C91C0877000A487706A80AF0A0
:10FD70004FFE6846008B404281B2674821300170D7
:10FD8000090A417006A80AF051FE68461821415E32
:10FD900000290EDA008B4042C1B25F482030C170AA
:10FDA000C0780121C9034018C1B25B482030C1703E
:10FDB00005E06846008BC1B257482030C1700AA8E0
:10FDC0000AF0C6FD544925310020F8F79BFA0024BB
:10FDD0004BE00AA8005D002846D04F482530F8F7D0
:10FDE00079FA00014C4925310490F8F78BFA0AA8FA
:10FDF000005D39280DDC48482530F8F76BFA0AA970
:10FE0000095D30390843444925310490F8F77AFAFE
:10FE10002AE00AA8005D662811DC0AA8005D6128B6
:10FE20000DDB3D482530F8F755FA0AA9095D573929
:10FE30000843394925310490F8F764FA14E00AA818
:10FE4000005D462810DC0AA8005D41280CDB324822
:10FE50002530F8F73FFA0AA9095D373908432E49DA
:10FE600025310490F8F74EFA641C0A2CB1DB0AF035
:10FE7000C3FD29492031487203A8FEF741FE0499C9
:10FE800003980991089008A80178234820308174CC
:10FE900008A8417820482030C17408A881781E48FD
:10FEA0002030017502214175022004F07BFE07908D
:10FEB0001D490798F8F797FA0490F8F7D5FC04461F
:10FEC00015493631F8F71EFA13493A310020F8F790
:10FED00019FA672108A8817531210176A12141769F
:10FEE0000321C177122181763421C1763E200A494F
:10FEF00001AAC1C200910DA80FC8FFF7E3F90120C4
:10FF00000A49087002E002200849087000200849E8
:10FF1000087011B0F0BD0000F44500200000C84298
:10FF200026F20000842C00200000204176130020DF
:10FF300075130020F0B591B004460D461646012C0D
:10FF40007ED1002071490870022004F02BFE0C9035
:10FF50006F490020F8F7D6F96E490C98F8F743FA84
:10FF60000490F8F781FC07466949091FF8F7CAF9B8
:10FF700002A814F0C9FA02A807C809AB07C369466A
:10FF8000888C0A21F8F7DCF86149091F08720DF026
:10FF900057F85F49091F4872000A88726846018D48
:10FFA0005B48001FC172090A01736846408D5849B9
:10FFB000091F48730FA80EF071FB10A84078544930
:10FFC000091F887310A801785148001FC17308A841
:10FFD000817F4F48001F017408A8417F4C48001FD3
:10FFE000417408A8017F4A48001F817403A8FEF7E6
:10FFF00087FD049903980E910D9008A8007D44494F
:020000040001F9
:10000000091FC87408A8417D4148001F017508A850
:10001000817D3F48001F41750221817509201BF039
:100020001FF83B49091F897D08433949091F887515
:100030000A20FEF751FD0002010E3548001F00E0C6
:100040002DE001760A20FEF747FD000E3049091F1A
:10005000C87511F0E1FE0746F8F706FC81B22C489E
:10006000001F4176090A81769A216846817502212E
:100070000176102141760321C177562181767821BE
:10008000C1761B202249091F01AA61C2009105A85F
:100090000FC8FFF717F901201F49087030E0032C43
:1000A00010D11A480078012808DA18480078401C56
:1000B0001649087001201849087021E002201649ED
:1000C00008701DE0F12C14D11448007D002808DDD3
:1000D0000AF0CCFC002804D00021012009F02EFFFA
:1000E00003E032210D488A30417002200A4908702D
:1000F00006E00021012009F021FF022006490870D6
:1001000000200749087011B0F0BD000079130020ED
:10011000364600200000204178130020202C0020CB
:10012000771300207CB504460D461646D248007869
:10013000042876D008DC00280DD0012858D00228E9
:1001400074D003286FD192E005286DD00A286CD0B6
:100150001528F7D14CE1012C08D10020C7490870BF
:10016000C74908700120C449087040E0022C1FD123
:10017000C2480078022804D1C24908700020BE4954
:100180000870BE480078032802D10A20BA490870D6
:10019000BA480078042805D10220BA490870002026
:1001A000B54908700020B649087011F005FD1EE041
:1001B000032C03D10F20B049087018E0F12C10D1A6
:1001C000FFF754FC002803D0FFF750FC032801D1AF
:1001D00011F0DAFC0220AB4908700020A649087033
:1001E00005E00220A74908700020A349087041E1FA
:1001F0001AF028FDA449087008460078002803D1A9
:1002000002209D4908700BE00020A04908700846B4
:1002100000781AF009FF9E4908700320964908707B
:1002200028E18AE002E021E19FE0C2E00220934958
:1002300008706620974988700020C8719648007839
:10024000401C9549087008460078924948729348C6
:1002500009F094FE924908803146284610F05CFF70
:1002600001208849087000208349087002E18B4909
:100270000A318748007809F04DFF8A49087008461E
:100280000078002858DD03207C4908707E480078FB
:10029000824908707D480078401C487000227C48E4
:1002A000017868460EF092FC69460878FBF70DFB72
:1002B0007A49887069464878FBF707FB7749C87028
:1002C00069468878FBF701FB74490871694608792B
:1002D000FBF7FBFA7149487169464879FBF7F5FA73
:1002E0006E49887169468879FBF7EFFA6B49C871E6
:1002F000062008726B48007848726A48007800014E
:100300000A30674908806620624988700020C871F9
:1003100061480078401C60490870084600785D49D3
:1003200048723146284610F0F7FE01205549087002
:1003300000205149087000BF9CE04520FEF7C2FB39
:1003400000280BD04520FEF7CFFB0020564908704F
:100350005649087005204849087005E002204949BF
:10036000087000204449087084E04D494B480AF069
:100370002FF94E48007801281AD167204549887026
:100380000020C87144480078401C43490870084662
:100390000078404948723146284610F0BDFE0420DE
:1003A000364908700120374908700020324908702A
:1003B00060E0374800780FF087F8002817D03348FE
:1003C0000078401C31490870084600782E490978A9
:1003D000884209DA2D4800781AF026FE2C49087068
:1003E00003202549087002E004202349087041E0F9
:1003F00023480078032820DA21480078401C20494F
:1004000008701E480078022802D11B4908702CE0B1
:100410001A480078032802D11749087025E01748C8
:100420000078042802D1144908701EE00220154902
:10043000087000201049087017E0FFF717FB00282C
:1004400003D0FFF713FB032809D10C4800780228DA
:1004500003D00A480078032801D111F095FB02204F
:100460000849087000200449087003E00020024990
:10047000087000BF00BF7CBD721400207014002003
:1004800071140020731400207514002076140020CD
:1004900077140020164C00206F140020864A00209C
:1004A0007A140020781400207C140020741400209A
:1004B00001200349087000200249087070470000BD
:1004C0007513002076130020002001490870704742
:1004D00072140020F0B589B0002400200890059027
:1004E000049000260027FA480078002802D001284E
:1004F0007ED129E000F0C4FEF64908600846006895
:10050000042820D006F0F2FB0A2814D1F248007823
:10051000401CF14908700321EF480078F7F710FEFE
:1005200000290DD10020EC49087011F01BFE0A20B3
:10053000EA49087004E011F015FE0A20E749087046
:100540000120E349087063E3E2480078C007C00F68
:1005500000287DD00020E249087100F0ABFE0020A9
:10056000E04908700B201AF0C9FE07A800F0BEFE93
:1005700006A804F0E1FA02A800F0A8FE03A804F01F
:10058000E7FA0024BDE2A00007990858A100D64A66
:100590005050A00006990858A100D44A5050082C89
:1005A0007EDAA00003990858A100D14A5050A0005B
:1005B00002990858A100CF4A5050A000CC49085CCD
:1005C0000006A100CA4A5158FF2212021140090236
:1005D0000843A100C64A5158FF2212041140090ADB
:1005E0000843A100C24A5158090E0843A10000E087
:1005F0000DE35050A000BF49085C0006A100BD4AB1
:100600005158FF221202114009020843A100B94AC1
:100610005158FF2212041140090A0843A100B54AAB
:100620005158090E0843A1005050A000B049085885
:10063000C00FC0070121C907884203D10020A100D3
:10064000AB4A5050A000AB490858C00FC00700E0AB
:1006500090E20121C907884203D10020A100A54AE8
:100660005050A000A249085800280DD0A0000858FA
:100670004B21C900884207D2A0009D49095805981E
:1006800008180590701CC6B2A0009A4908580028A6
:100690000FD0A00008584B21C900884209D200E0C1
:1006A00007E0A00093490958049808180490781CA2
:1006B000C7B2A0008C49085C0006A1008A4A5158C4
:1006C000FF221202114009020843A100864A515834
:1006D000FF2212041140090A0843A100824A51581E
:1006E000090E0843A1005050FBF71AFA012808D15F
:1006F0008148F7F7EFFDA1007B4A51584018A1004F
:100700005050A00079490858012109060840884244
:100710007DD1A00074490858C00FC0070121C90746
:10072000884212D1A0007049085840004008A1003A
:100730006D4A5050A00011460858C043401CA1000B
:1007400050500A201AF0DAFD02E017201AF0D6FD08
:10075000A00065490858002804D0A000085867493F
:1007600088420CD9A000604908580121C907884275
:1007700009D3A0005C4908586149884203D84D203C
:100780001AF0BCFD36E0A000574908585C49884281
:1007900009D9A000544908585A49884203D807206B
:1007A0001AF0ACFD26E0A0004F4908585549884290
:1007B00011D9A0004C490858534988420BD8A000D1
:1007C000494908584000400801218904081AA1003D
:1007D000454A50500EE0002C05D14348C06BA100A3
:1007E000414A505006E0601E80003F490858A10071
:1007F0003D4A5050A1003C4A505810F00DFB2120BA
:100800001AF07CFD16201AF079FD582000E00DE06A
:100810001AF074FD00203249487088700870C87062
:1008200000F03AFD012000F037FD15E1A0002F494E
:1008300008580121C9060840884238D12848407824
:10084000102804DB0020A100274A505013E0244860
:100850004078401C22494870002C05D12248C06BCA
:10086000A100214A505006E0601E80001E49085831
:10087000A1001D4A5050A1001B4A505810F0CCFA5C
:1008800002201AF03BFD17201AF038FD4D201AF017
:1008900035FD002012490870C87021201AF02EFD85
:1008A000002000F0F9FC012000F0F6FCD4E0A000EC
:1008B0000E490858012149060840884258D1084885
:1008C0008078102822DB0020A100074A505031E038
:1008D0001906002010060020D8060020500600202F
:1008E00051060020AA060020382000207820002091
:1008F0002823002048230020FE22002014AE0300FD
:1009000007010080EB51008000000480C24880781D
:10091000401CC1498870002C05D1C048C06BA100A3
:10092000BE4A505006E0601E8000BC490858A10035
:10093000BA4A5050A100B94A505810F06DFA082038
:100940001AF0DCFC21201AF0D9FC02201AF0D6FCA7
:1009500017201AF0D3FC4D201AF0D0FC0020AE492D
:100960000870C87000F098FC012000F095FC73E05E
:10097000A000AB49085801218906084088421DD1D2
:10098000A5480078401CA449087008460078032850
:100990000EDC002C05D1A148C06BA1009F4A50502D
:1009A00006E0601E80009D490858A1009B4A5050F7
:1009B000A1009A4A505810F02FFA4DE0A000984933
:1009C0000858012149070840884204D0A0009449F2
:1009D0000858002829D103201AF090FC8E48C078CE
:1009E000401C8D49C870002C05D18C48C06BA100FB
:1009F0008A4A505006E0601E800088490858A100CD
:100A0000864A50508448C078102808DB002082496C
:100A1000C870FDF791FA012801D100F06DFCA1002A
:100A20007E4A505810F0F8F916E021201AF066FCC2
:100A3000002C05D17948C06BA100784A505006E0DF
:100A4000601E800075490858A100744A5050A100EA
:100A5000724A505810F0E0F9A0007149085801217D
:100A600009070840884247D109201AF047FC089836
:100A7000401CC0B208900898102809D1002405E055
:100A80000120A100654A5050601CC4B2102CF7DB55
:100A9000002C15D16148C06B0121C90788420AD8D2
:100AA0005E48C06B5F49884205D35C48C06BA100BB
:100AB0005A4A505023E00120A100584A50501EE0ED
:100AC000601E8000554908580121C90788420ED888
:100AD000601E8000514908585249884207D3601E61
:100AE00080004E490858A1004C4A505007E00120B0
:100AF000A1004A4A505002E063201AF0FFFB601C3C
:100B0000C4B2102C00DA3EE5002F08D03946049814
:100B1000F7F700FB44490190F7F7F4FB03E0424983
:100B20000020F7F7EFFB002E09D031460598F7F7C4
:100B3000F1FA3D490C390190F7F7E4FB04E03A493A
:100B40000C390020F7F7DEFBFEF75EFE36480C3866
:100B5000F7F7C0FB35490190F7F7D4FB3248F7F7B8
:100B6000B9FB32490C310190F7F7CCFB002030493A
:100B700008704BE02F48006802210840022845D148
:100B800025480079401C2449087100F093FB00F0CF
:100B900071FB05462048007905280BDB05201E491E
:100BA000087140211D48F7F76EFB40211C48F7F7FC
:100BB0006AFB19E0002410E0002C05D11748C06B37
:100BC000A100164A505006E0601E800013490858E4
:100BD000A100124A5050601CC4B2102CECDBA100E2
:100BE0000E4A505810F018F9E807C00F002803D03B
:100BF00001201AF083FB06E002202840022802D1DF
:100C000001201AF07BFB00200949087000E000BFBA
:100C100000BF09B0F0BD00005106002038200020C0
:100C20007820002066660000542200200022002068
:100C3000190600201006002010B53448007800285E
:100C400002D001285FD14CE00120FDF73BFF0128D5
:100C500046D1FDF749FF002405E00020A1002C4A01
:100C60005050601CC4B2102CF7DB2A4A0020014609
:100C7000F7F751FB28490020F7F744FB2649091DE7
:100C80000020F7F73FFB25490020F7F73BFB2349FE
:100C9000091D0020F7F736FB21490020F7F732FB4A
:100CA0000020204908602049086020490860204948
:100CB000086000F043F8FBF7C5FE00280DD01D4B7F
:100CC0001622FF2101311C48FCF720F900200F49B2
:100CD0000870FF201AF012FB02E001200B49087097
:100CE00012E0FBF7AFFE00280CD0124B1622FF21BA
:100CF00001311148FCF70AF9002004490870FF206F
:100D00001AF0FCFA00E000BF00BF10BD9106002001
:100D1000382000207D060020EC2100203422002015
:100D20005E060020007F0020047F0020087F002056
:100D30000C7F0020D9060020E022002010B577208B
:100D40001D490870882048701C480DF0A7FC1B48FE
:100D5000007819498870194841781748C1701748B8
:100D6000817815480171154801791348417114487B
:100D7000F7F7B0FA04461049891DF7F7C3FA10488F
:100D8000001DF7F7A7FA04460B490A31F7F7BAFA3C
:100D90000B482830F7F79EFA044607490E31F7F75B
:100DA000B1FA07482C30F7F795FA04460249123198
:100DB000F7F7A8FA10BD0000E0220020BB060020D3
:100DC000EC210020F8B5B2480078030013F0E7FEEC
:100DD000090627F9F3F2F1F0EFEEF200FBF732FE2D
:100DE00000281BD000240DE0A000AA4A8118002092
:100DF000F7F788FAA000A84A81180020F7F782FACE
:100E0000601CC4B2122CEFDBA44B1622A449FF20B5
:100E10000130FCF735F801209D49087035E19F4805
:100E20000078FBF701FE01287ED1FBF70BFE0128BD
:100E3000FAD19B480078772877D19948407888285C
:100E4000FAD1984800689849884229D104219748E6
:100E50000CF090FF012806D19148801DF7F73AFA6F
:100E60009249086005E08E49891D90480068F7F7AF
:100E700049FA04218E480CF07DFF012806D18848EC
:100E80000A30F7F727FA8A49086005E084490A31F1
:100E900087480068F7F736FA05207D49087002E0B8
:100EA00007207B4908707E480E30F7F713FA054695
:100EB0008121C905F7F7A8FD1BD379481230F7F750
:100EC00009FA05468121C905F7F79EFD11D374483B
:100ED0000E30F7F7FFF905467649F7F78BFD08D393
:100EE0006F481230F7F7F6F905467249F7F782FDB9
:100EF0000CD26B490E310020F7F704FA6849123121
:100F00000020F7F7FFF90520614908706448801D4B
:100F1000F7F7E0F905465F49091DF7F7F3F960486F
:100F20000A30F7F7D7F901E04AE02AE005465949C7
:100F30000831F7F7E7F95A48801DF7F7CBF905466E
:100F40005D49F7F7DFF956480E30F7F7C3F9054664
:100F500050492C31F7F7D6F951481230F7F7BAF962
:100F600005464C493031F7F7CDF94A48001DF7F7EF
:100F7000B1F90746F7F7E6FC0546504AF7F7CBF913
:100F80001EE04D490020F7F7BDF9FBF75BFD002897
:100F900013D0FFF7D3FE414B1622FF210131404809
:100FA000FBF7B4FF03203A49087009E056E040E03F
:100FB00036E025E068E015E003E0022034490870DF
:100FC00063E0FBF73FFD00280BD0FFF7B7FE334B84
:100FD0001622FF2101313248FBF798FF03202C49EC
:100FE000087052E02D480078FBF71EFD012806D15D
:100FF000FBF728FD012802D107202549087044E0AD
:10100000FBF720FD00280AD0244B1022FF210731D6
:101010002348801DFBF77AFF03201D49087034E048
:101020001520FDF759FD2649086001202549087063
:101030002BE01A480078FBF7F7FC01280DD1FBF7ED
:1010400001FD012809D1154B0C221F49FF20513009
:10105000FBF716FF08200E49087016E00F480078CD
:10106000FBF7E2FC01280ED1FBF7ECFC01280AD1CA
:10107000FAF756FD002803D113490831F7F742F972
:1010800006200349087000E000BF00BFF8BD000063
:10109000A5060020E821002030220020C206002002
:1010A000E0220020147F00206D5C4B3A007F00207E
:1010B000047F0020000080C0150600207D0600206F
:1010C00070060020A6060020F622002070B55548C4
:1010D0000078002804D001280BD006287AD17AE0C5
:1010E000E121090103200DF04FFC01204D4908705A
:1010F00095E003200DF0A2FA002814D00CF054F86B
:10110000012810D00320FDF7DDFC01280BD0464854
:101110000078002807D1FAF7FDFC012803D013F06E
:10112000ADFB012855D1FBF78DFC002851D00320E1
:101130000DF084FA00282ED13C48F7F7CBF805468D
:101140003B48F7F7C7F806462946F7F744F904463F
:101150007F21C9052046F7F757FC04D335492046BF
:10116000F7F748FC13D23248F7F7B4F805462F4991
:10117000F7F7C8F8FFF7E2FD2F4B1622FF210131E8
:101180002E48FBF7C3FE06202649087021E0002008
:10119000244908701DE0FAF7BDFC01280AD100209F
:1011A00027490870274B0422FF2159312648FBF7B5
:1011B000ADFE0EE000201C490870FFF7BFFD1E4B7E
:1011C0001622FF2101311D48FBF7A0FE062015491C
:1011D000087024E022E0FBF735FC00281DD0FF203A
:1011E0001AF08CF80320FDF76DFC012805D10320CF
:1011F000FDF77AFC0120154908700BF0D5FF012896
:1012000003D013F03BFB012804D1012008F002FDBC
:1012100013F010FD00200349087000E000BF00BF7C
:1012200070BD0000A4060020900600204C0600209F
:10123000EC210020000080BFDA060020E022002020
:10124000A80600207C060020FE220020A706002021
:1012500010B5074800780A2807DA05480078401CCE
:101260000349087000F048F801E004F087F810BD69
:10127000AA0600200148007870470000BA03002049
:101280000148007870470000B90300200148007849
:1012900070470000BC030020072800DD70470121D3
:1012A0008140034A12788A4301490A7000BFF5E77A
:1012B000BA0300200420014908707047B9030020D8
:1012C0000020014908707047BC0300200549C97817
:1012D000C900054A8A180349C9784910890051187C
:1012E00001607047CA0100207C1C00200149016098
:1012F000704700007C1C002010B5FEF707F9FEF7D0
:1013000077F900200F4908600F4908600F490870FD
:101310000F4908700F4908700F4908700F4908708D
:101320000F4908700F4908700F4908700F4908608D
:101330000F4908600F49086010F04CFF0B49086026
:1013400010BD0000AC030020B0030020B403002057
:10135000B5030020B6030020B7030020B803002027
:10136000BD030020BB030020BC030020C8030020F5
:10137000C0030020C4030020F8B50446002C0AD0A6
:1013800001204005844202D31748844203D9062035
:1013900019F0B4FF02E0422019F0B0FF002C07D092
:1013A00001200005844203D2042019F0A7FF02E0C7
:1013B0002C2019F0A3FF10F02FFD07460B493846EB
:1013C000F7F722FB08D33846F7F7BCFA05460022A8
:1013D000074BF7F7CBFA03D2052019F08FFF02E095
:1013E000372019F08BFFF8BD0000B04F00005C42C1
:1013F0000000E0BFF0B589B00025002700261720C7
:10140000FDF76AFBFE4908600846006803F05FFDCF
:10141000FC490860084601680020F6F7DCFFFA493D
:10142000086000242DE0A000F84908580121C907F0
:1014300088421CD3A000F549085840004008A1008C
:10144000F24A5050A100505803F041FD002107908E
:10145000F6F7C5FFA100EE4A5050A000EB4908582E
:101460000121C9070843A100E84A505007E0A10044
:10147000E64A505803F02BFDA100E54A5050601C8D
:10148000C4B2102CCFDB05F031FC0A2873D1002048
:10149000E04908701021DE48FBF75EFF0646DE4893
:1014A000066000213046F7F7A5FA08D20A20DB498A
:1014B000087031460020F6F78EFF064602E0012054
:1014C000D64908703046FDF741FA0890089800F0B8
:1014D000B3FA07463846FDF739FAD1490690F6F7D0
:1014E00011FFCF48F6F7F6FECE490690F6F70AFF51
:1014F000CB48F6F7EFFE0690FFF73EFFCA4840796B
:1015000001280BD1C9480078401CC849087008461A
:101510000078F02805DB0020087002E00020C349B5
:101520000870C048F6F7D6FE002805D0162019F03E
:10153000E5FE582019F0E2FE384608F09FFB07460A
:10154000384601F0A3FE39460020F7F753FA7DD064
:10155000B748007800280FD1B6480068F7F75BF964
:10156000432109060590F6F77BFF39460690F6F70A
:101570003AFF054612E08EE1AF493846F6F733FFF1
:101580000746AC480068F7F746F939460590F6F784
:101590002AFFAA490690F6F763FF0546A8492846A0
:1015A000F6F721FFA7490690F6F75AFF0546A64928
:1015B0002846F6F755FF054698480078012813D1CC
:1015C000A248F6F791FE039102902846F7F7BAF980
:1015D00001910090039B029AF6F780FF9B4A0591C8
:1015E0000490F6F798FEE0E01620FDF775FA9849AA
:1015F00088423BD19548F6F777FE0591049028463E
:10160000F7F7A0F903910290059B049AF7F7C2F946
:1016100005D88E4A00200146F6F77DFE12E08B4881
:10162000F6F762FE039102902846F7F78BF90191D5
:101630000090039B029AF6F7FBFF844A0591049001
:10164000F6F769FE8148F6F74FFE00E0A7E0059146
:101650000490F7F7B3F9734908390690F6F752FE8C
:1016600070480838F6F736FE7A4908606D48001F62
:10167000F6F730FE78490690F7F7C6F921D22946E9
:1016800076480068F6F756FE744908606C4973485E
:101690000068F7F7B9F97BD2694970480068F6F736
:1016A0009AFE6E4908605F48001FF6F713FE644912
:1016B0000590F6F73FFE5B49091F0690F6F722FEFC
:1016C00066E05848001FF6F705FE65490690F7F7F3
:1016D0009BF921D2294661480068F6F72BFE5F4945
:1016E000086060495D480068F7F78EF950D25D499F
:1016F0005A480068F6F76FFE584908604948001FCD
:10170000F6F7E8FD57490590F6F714FE4549091F1D
:101710000690F6F7F7FD3BE04248001FF6F7DAFDCA
:101720004649A0390690F7F76FF924D229464B486D
:101730000068F6F7FFFD494908607F21C905474861
:101740000068F7F761F923D27F21C9054348006893
:10175000F6F741FE414908603248001FF6F7BAFD2E
:101760007F21C9050590F6F7E5FD2E49091F069072
:10177000F6F7C8FD0CE02B48001FF6F7ABFD294635
:101780000590F6F7D7FD2749091F0690F6F7BAFD31
:101790002448001FF6F79EFD3349086005E0214804
:1017A000001FF6F797FD304908603A461B4801785C
:1017B000284613F09BF80790012189070798F7F74F
:1017C00023F905D3032189070798F7F713F901D205
:1017D000002007901D48F6F787FD039102900798B7
:1017E000F7F7B0F801910090039B029AF6F776FEA6
:1017F000164A05910490F6F78EFD144836E0000075
:10180000380600203C06002040060020382000203A
:10181000A02200205006002094060020850600200B
:101820003C220020F42100208C220020AB06002066
:10183000A0060020B4060020643B7F3F00247449CA
:101840000000C8420000614500007A447D06002087
:101850003C4D0000007F0020A3BBBE4C880600204A
:101860007696184B00002041047F0020F6F73CFDDF
:1018700005910490F7F7A2F85C490690F6F742FD4F
:101880005A48F6F727FD5A4908605A4805605A48F1
:101890005A490860A7E05A480078012804D100207E
:1018A000574908701AF082FF10215648FBF754FD83
:1018B00006465548066000213046F7F79BF800D2EF
:1018C00000263046FDF742F80890089800F0B4F87A
:1018D00007463846FDF73AF84C4908604C484079CD
:1018E00001280BD14B480078401C4A490870084633
:1018F00000780F2805DB0020087002E00020454931
:101900000870384608F0BAF907463846FAF7A8FED4
:10191000384601F0BBFC39460020F7F76BF851D090
:10192000162019F0EBFC582019F0E8FC3A48006842
:10193000F6F771FF432109060590F6F791FD394648
:101940000690F6F750FD35490790F6F789FD0546F4
:101950003348F6F7BFFC29460690F6F7EBFC304912
:101960000790F6F7CFFC2F48F6F7BEFC05910490E0
:101970002D492846F6F774FD0190F6F7E3FF039131
:101980000290059B049AF6F7A9FD264A0791069056
:10199000F6F7C1FC2348F6F7A7FC05910490F7F78A
:1019A0000DF812490790F6F7ADFC1D48F6F792FCCA
:1019B0001E4908601E4805600C48F6F78BFC0C4970
:1019C00008600DE00948F6F785FC094908600748FA
:1019D000001DF6F77FFC17490860002014490860D5
:1019E00005480649086009B0F0BD0000EC21002060
:1019F000007F0020187F00206D5C4B3A147F002090
:101A000025060020A0220020940600201C060020AD
:101A10008C220020AB060020B406002000001042FB
:101A2000342200207D06002000007A44087F002038
:101A30000C7F0020047F002001B59CB000201B908B
:101A40001A90199005200CF0EFFD002811D0052008
:101A50000CF01AFEFE480068FE49884203D90120B6
:101A6000FD49087002E00020FB4908700020F84999
:101A70000860FA491C980968884204D30121890446
:101A80001C98884202D300201B90F6E3F0480068BF
:101A9000401CEF4908601C9803F019FA1A90F049AD
:101AA0001A98F6F7A0FC1A90FAF73AF801281AD11A
:101AB000EC480068401CEB49086004200CF0B4FDC1
:101AC000002813D004200CF0DFFDE6480068E1494F
:101AD000884204D903F006FA0120E3490870002087
:101AE000E049086002E00020DE490860DF48007835
:101AF000002803D0DE480068199002E010F08CF94D
:101B000019901998F6F71EFF0022DA4B17911690DC
:101B1000F6F72CFF0CD2D848F6F7DCFB5F2807D984
:101B2000D5480C30F6F7D6FB5F2801D9D348199079
:101B30000CF0D2F9D2490860D2481A99F6F753FC52
:101B400015901A99F6F74FFC1790CF481999F6F7A8
:101B50004AFC13901A99F6F746FC1590CB48199950
:101B6000F6F741FC11901999F6F73DFC1390C8481F
:101B70001A99F6F738FC1190C6481999F6F733FC14
:101B8000C5490F90F6F7D6FB10901199F6F7D2FBE6
:101B900012901399F6F71FFC14901599F6F7CAFBEB
:101BA00016901799F6F7C6FB1890BC491898F6F7E7
:101BB00021FF7DD800211998F6F71CFF04D3B849FE
:101BC0001998F6F721FF03D2B648006D179028E068
:101BD0001998F6F749FEC0B215901598F6F71BFE56
:101BE0000D901999F6F7FBFB149015988000AD49FC
:101BF00008580B901598401C800008580A900B99C3
:101C0000F6F7E9FB0C901499F6F7EDFB0D9015989B
:101C10008000A449085801460C900D98F6F78AFBFD
:101C2000179017990846F6F7DEFB0C901A99F6F70D
:101C3000DAFB9D490D90F6F7D6FB13901998129098
:101C400000211998F6F7D6FE02D20020129006E085
:101C500096491998F6F7D8FE01D294481290944804
:101C60001299F6F7C0FB0C9092481299F6F7BBFB5D
:101C700008901299F6F7B7FB0A908F481299F6F779
:101C8000B2FB07901299F6F7AEFB08901299F6F79F
:101C9000AAFB09900A99F6F74DFB0B900C99F6F701
:101CA0009AFB86490D90F6F745FB1190844800E0B9
:101CB000ECE11299F6F797FB0B9082481299F6F730
:101CC00092FB09901299F6F78EFB0A900B99F6F7A2
:101CD00031FB7D490C90F6F72DFB7C490D90F6F712
:101CE00082FB109079481099F6F77DFB0B901399C1
:101CF000F6F779FB76490C90F6F775FB0D90119984
:101D0000F6F7AEFB0F9073491398F6F76CFB1B9038
:101D10006E490F98F6F7A4FB0E906F490E98F6F7F0
:101D200069FE55D26D480E99F6F75DFB0C906C4834
:101D30000E99F6F758FB08900E99F6F754FB0A90A7
:101D400068480E99F6F74FFB05900E99F6F74BFB96
:101D500006900E99F6F747FB089063480E99F6F740
:101D600042FB02900E99F6F73EFB03900E99F6F7B0
:101D70003AFB04900E99F6F736FB06905B480E99F5
:101D8000F6F731FB01900E99F6F72DFB02900E99B4
:101D9000F6F729FB03900E99F6F725FB04900E99B0
:101DA000F6F721FB05900699F6F715FB07900899C1
:101DB000F6F7C0FA09900A99F6F70DFB0B900C990B
:101DC000F6F7B8FA4A490D90F6F7B4FA169052E1D0
:101DD00048490E98F6F70EFE38D247480E99F6F7A6
:101DE00002FB0C9045480E99F6F7FDFA08900E9903
:101DF000F6F7F9FA0A9042480E99F6F7F4FA0590C8
:101E00000E99F6F7F0FA06900E99F6F7ECFA0890AC
:101E10003C480E99F6F7E7FA02900E99F6F7E3FAC6
:101E200003900E99F6F7DFFA04900E99F6F7DBFAB5
:101E3000069035480E99F6F7D6FA01900E99F6F706
:101E4000D2FA02900E99F6F7CEFA5FE07CE000003D
:101E5000D0060020B8A10000A90600203806002006
:101E600000007A43CC060020A8060020320600209D
:101E7000340600200000E0BF002200200000A04146
:101E8000AC0600204DA0083C423EE83D8126C23C05
:101E90003D0ABB41C1CAC13FEC51E8C100C0284561
:101EA0000000C84238D80200B91DCA3100005C42A7
:101EB00023DB5C421A516A3FA69BC4BB6606DF4423
:101EC0003B4A5B372684B3B64703803F00007A4421
:101ED0000000D04162E1F144CDCCAC404B75013DF6
:101EE00061E28F3C1A53B03B3EF4553AE93A493827
:101EF000C009653F00004842643B043B5762D83844
:101F0000451E4D3632CE46330689982F03900E99E2
:101F1000F6F769FA04900E99F6F765FA05900699B6
:101F2000F6F759FA07900899F6F704FA09900A9912
:101F3000F6F751FA0B900C99F6F7FCF9FE490D9063
:101F4000F6F7F8F9169096E0FC490E98F6F752FD70
:101F500055D2FB480E99F6F746FA0C90F9480E99BF
:101F6000F6F741FA08900E99F6F73DFA0A90F6480E
:101F70000E99F6F738FA05900E99F6F734FA0690AE
:101F80000E99F6F730FA0890F0480E99F6F72BFA0A
:101F900002900E99F6F727FA03900E99F6F723FAB6
:101FA00004900E99F6F71FFA0690E9480E99F6F795
:101FB0001AFA01900E99F6F716FA02900E99F6F7B2
:101FC00012FA03900E99F6F70EFA04900E99F6F7AE
:101FD0000AFA05900699F6F7FEF907900899F6F7C0
:101FE000A9F909900A99F6F7F6F90B900C99F6F70A
:101FF000A1F9D8490D90F6F79DF916903BE0D64827
:102000000E99F6F7F0F90C90D4480E99F6F7EBF923
:1020100008900E99F6F7E7F90A90D1480E99F6F76D
:10202000E2F905900E99F6F7DEF906900E99F6F7AB
:10203000DAF90890CB480E99F6F7D5F904900E9985
:10204000F6F7D1F905900E99F6F7CDF906900E99AD
:10205000F6F7C9F907900899F6F76CF909900A990B
:10206000F6F7B9F90B900C99F6F764F9BE490D90A3
:10207000F6F760F9169016991B98F6F7B4F91B90CD
:1020800019A807C8FBF736F81B90EEE3B749199873
:10209000F6F7BAFC7ED2B6491898F6F7ABFC7AD2BE
:1020A000B4480068014613901A98F6F743F9159062
:1020B000B0480068014611901A98F6F73BF9139062
:1020C000AC480068014610901A98F6F733F9119061
:1020D000A848806A014610901198F6F784F912908A
:1020E0001399F6F780F914901599F6F77CF9179083
:1020F000A0480068014610901A98F6F71BF9129054
:102100009C48006801460F901A98F6F713F9109052
:102110009848406A01460F901098F6F764F91190BC
:102120001299F6F760F913901999F6F75CF9159082
:102130009048006801460E901A98F6F7FBF80F9049
:102140008C48006A01460E900F98F6F74CF91090F3
:102150001999F6F748F911901999F6F744F913907F
:102160008448C0690D901999F6F73DF90E901999B8
:10217000F6F739F90F901999F6F735F911907D486E
:10218000006801460B901A98F6F7D4F80D9079483C
:10219000006801E07DE171E001460A901A98F6F7C7
:1021A000C9F80B907348806901460A900B98F6F7BE
:1021B0001AF90C900D99F6F716F90F906D48006812
:1021C000014609901A98F6F7B5F80A9069484069EF
:1021D000014609900A98F6F706F90B901999F6F757
:1021E00002F90D906348006908901999F6F7FBF819
:1021F00009901999F6F7F7F80B905E4800680146C8
:1022000006901A98F6F796F807905A48C068014663
:1022100006900798F6F7E7F8099056488068069008
:102220001999F6F7E0F80790524840680146069081
:102230000798F6F77FF808900999F6F77BF80A9067
:102240000B99F6F777F80C900D99F6F773F80E9056
:102250000F99F6F76FF810901199F6F76BF8129046
:102260001399F6F767F814901599F6F763F8169036
:102270001799F6F75FF81B90F7E2FAE33D48C06A5A
:10228000014613901A98F6F755F815903948C06A28
:10229000014611901A98F6F74DF813903548C06A28
:1022A000014610901A98F6F745F811903148406DA4
:1022B000014610901198F6F796F812901399F6F7D8
:1022C00092F814901599F6F78EF817902948C06A7D
:1022D000014610901A98F6F72DF812902548C06A1A
:1022E00001460F901A98F6F725F810902148006DD6
:1022F00001460F901098F6F776F811901299F6F7BC
:1023000072F813901999F6F76EF815901948C06A8B
:1023100001460E901A98F6F70DF80F901548C06C0C
:1023200001460E900F98F6F75EF810901999F6F79F
:102330005AF8119019991FE070256B3F0000C843AF
:10234000CB694B39C66FA7350D4FA03168681D2D7D
:10235000F82DF527CB106F3F574FED37D96F12335C
:10236000D9FBC82D6F73E1A74AA1713F00000C4251
:1023700000008C43140F0020F6F735F81390FE4848
:10238000806C0D901999F6F72EF80E901999F6F7C2
:102390002AF80F901999F6F726F81190F648C06AB6
:1023A00001460B901A98F5F7C5FF0D90F248C06AE8
:1023B00001460A901A98F5F7BDFF0B90EE48406C65
:1023C00001460A900B98F6F70EF80C900D99F6F767
:1023D0000AF80F90E848C06A014609901A98F5F784
:1023E000A9FF0A90E448006C014609900A98F5F7A5
:1023F000FAFF0B901999F5F7F6FF0D90DE48C06BC8
:1024000008901999F5F7EFFF09901999F5F7EBFF87
:102410000B90D948C06A014606901A98F5F78AFFD2
:102420000790D548806B014606900798F5F7DBFFCB
:102430000990D148406B06901999F5F7D4FF0790A1
:10244000CD48006B014606900798F5F773FF08909A
:102450000999F5F76FFF0A900B99F5F76BFF0C9050
:102460000D99F5F767FF0E900F99F5F763FF109040
:102470001199F5F75FFF12901399F5F75BFF149030
:102480001599F5F757FF16901799F5F753FF1B901D
:10249000EBE1BA491898F6F7ADFA7DD2B648806DEF
:1024A000014613901A98F5F745FF1590B248806DD4
:1024B000014611901A98F5F73DFF1390AE48806DD4
:1024C000014610901A98F5F735FF1190AA48803010
:1024D0000068014610901198F5F785FF1290139946
:1024E000F5F781FF14901599F5F77DFF1790A24835
:1024F000806D014610901A98F5F71CFF12909E48C7
:10250000806D01460F901A98F5F714FF10909A48C5
:10251000C06F01460F901098F5F765FF1190129962
:10252000F5F761FF13901999F5F75DFF1590924843
:10253000806D01460E901A98F5F7FCFE0F908E48BC
:10254000806F01460E900F98F5F74DFF1090199986
:10255000F5F749FF11901999F5F745FF1390864853
:10256000406F0D901999F5F73EFF0E901999F5F708
:102570003AFF0F901999F5F736FF11907E48806D5C
:1025800001460B901A98F5F7D5FE0D907A48806DAC
:1025900001460A901A9800E06DE0F5F7CBFE0B902B
:1025A0007548006F01460A900B98F5F71CFF0C90D8
:1025B0000D99F5F718FF0F906F48806D014609904F
:1025C0001A98F5F7B7FE0A906B48C06E014609905D
:1025D0000A98F5F708FF0B901999F5F704FF0D908D
:1025E0006548806E08901999F5F7FDFE09901999D4
:1025F000F5F7F9FE0B906048806D014606901A9839
:10260000F5F798FE07905C48406E014606900798E3
:10261000F5F7E9FE09905848006E06901999F5F70C
:10262000E2FE07905448C06D014606900798F5F702
:1026300081FE08900999F5F77DFE0A900B99F5F750
:1026400079FE0C900D99F5F775FE0E900F99F5F740
:1026500071FE10901199F5F76DFE12901399F5F730
:1026600069FE14901599F5F765FE16901799F5F720
:1026700061FE1B90F9E040488030406801461390AD
:102680001A98F5F757FE15903B4880304068014690
:1026900011901A98F5F74EFE139037488030406835
:1026A000014610901A98F5F745FE11903248803097
:1026B000C06A014610901198F5F795FE1290139993
:1026C000F5F791FE14901599F5F78DFE17902A48AD
:1026D00080304068014610901A98F5F72BFE129052
:1026E00025488030406801460F901A98F5F722FE81
:1026F000109021488030806A01460F901098F5F7BD
:1027000072FE11901299F5F76EFE13901999F5F774
:102710006AFE159018488030406801460E901A985D
:10272000F5F708FE0F9014488030406A01460E907D
:102730000F98F5F758FE10901999F5F754FE11907F
:102740001999F5F750FE13900B488030006A0D90F0
:102750001999F5F748FE0E901999F5F744FE0F9078
:102760001999F5F740FE1190034880304068014602
:102770000B901A9804E00000140F002000008C4316
:10278000F5F7D8FD0D90F948406801460A901A986F
:10279000F5F7D0FD0B90F548C06901460A900B98FB
:1027A000F5F721FE0C900D99F5F71DFE0F90EF48FF
:1027B0004068014609901A98F5F7BCFD0A90EB486D
:1027C0008069014609900A98F5F70DFE0B9019995A
:1027D000F5F709FE0D90E548406908901999F5F75D
:1027E00002FE09901999F5F7FEFD0B90DF4840684D
:1027F000014606901A98F5F79DFD0790DB480069A1
:10280000014606900798F5F7EEFD0990D748C06895
:1028100006901999F5F7E7FD0790D44880680146BE
:1028200006900798F5F786FD08900999F5F782FD5F
:102830000A900B99F5F77EFD0C900D99F5F77AFD4E
:102840000E900F99F5F776FD10901199F5F772FD3E
:1028500012901399F5F76EFD14901599F5F76AFD2E
:1028600016901799F5F766FD1B90C1491898F6F771
:10287000C1F818D8BF4800688830F5F72BFD1690CE
:10288000BC4800689030F5F725FD14901B99F5F7CA
:10289000AAFD15901699F5F74DFD17901B99F5F7C0
:1028A000A2FD1B9053E0B4491898F6F7A3F818D886
:1028B000B04800685C30F5F70DFD1690AD48006833
:1028C0006430F5F707FD14901B99F5F78CFD159012
:1028D0001699F5F72FFD17901B99F5F784FD1B90BE
:1028E00035E0A6491898F6F785F818D8A148006889
:1028F0003030F5F7EFFC16909E4800683830F5F759
:10290000E9FC14901B99F5F76EFD15901699F5F7F3
:1029100011FD17901B99F5F766FD1B9017E0954880
:102920000068001DF5F7D6FC1690924800680C3040
:10293000F5F7D0FC14901B99F5F755FD15901699F5
:10294000F5F7F8FC17901B99F5F74DFD1B908C4996
:102950001998F6F74FF807D200201999F6F74AF8B8
:1029600002D000201DB000BDF9F7DAF8012806D129
:1029700084491B98F6F73EF801D80020F2E7824818
:10298000F5F7A8FC1590F5F761FF00227F4B179132
:102990001690F5F7EBFF0DD37B480C30F5F79AFC5A
:1029A0001590F5F753FF0022784B17911690F5F725
:1029B000DDFF07D2212149061B98F6F71BF801D845
:1029C0000020CFE700211B98F6F714F801D2002071
:1029D0001B906F491998F6F70DF856D26D491B9860
:1029E000F6F708F805D26C491B98F5F7FCFC1B902C
:1029F00002E268491B98F6F707F812D867491B9856
:102A0000F5F7F8FF0DD266481B99F5F7ECFC654920
:102A10001690F5F78FFC17901B99F5F7E4FC1B90C7
:102A2000F4E35E491B98F5F7EFFF12D85E491B9857
:102A3000F5F7E0FF0DD25D481B99F5F7D4FC5C4932
:102A40001690F5F777FC17901B99F5F7CCFC1B90C7
:102A5000DCE355491B98F5F7D7FF0BD855491B9870
:102A6000F5F7C8FF06D254491B98F5F7BCFC1B903C
:102A7000CCE3D0E351491B98F5F7C6FFB8D85049CD
:102A80001B98F5F7B0FC1B90C0E34E491998F5F779
:102A9000B1FF6AD23F491B98F5F7ACFF05D23E491A
:102AA0001B98F5F7A0FC1B90B0E33A491B98F5F78B
:102AB000ABFF12D839491B98F5F79CFF0DD2384867
:102AC0001B99F5F790FC37491690F5F733FC1790F2
:102AD0001B99F5F788FC1B9098E330491B98F5F794
:102AE00093FF12D830491B98F5F784FF0DD22F4879
:102AF0001B99F5F778FC2E491690F5F71BFC1790FB
:102B00001B99F5F770FC1B9080E327491B98F5F79C
:102B10007BFF0AD827491B98F5F76CFF05D22A4995
:102B20001B98F5F760FC1B9070E322491B98F5F7A2
:102B30006BFF0AD825491B98F5F75CFF05D21E49A3
:102B40001B98F5F750FC1B9060E321491B98F5F7A3
:102B50005BFF41D81F491B98F5F74CFF3CD2184941
:102B60001B98F5F740FC1B9050E358E0940F0020B1
:102B700000009842AC0600200080044400C02845B4
:102B8000CDCCCC3D00001042002200200000694066
:102B900014AE3F4100000C42D7A3803F00007042BA
:102BA00082A8FBB8772D813F00008C4252491DBAA4
:102BB0002FDD843F0000AA42DBF97E3F000016446F
:102BC0001283803F00008441B6F37D3F0000F04255
:102BD000000048430000A043FE491B98F5F714FF8E
:102BE00012D8FD491B98F5F705FF0DD2FB481B993C
:102BF000F5F7F9FBFA491690F5F79CFB17901B992E
:102C0000F5F7F1FB1B9001E3F6491B98F5F7FCFE85
:102C10008AD8F5491B98F5F7E6FB1B90F6E2F349D5
:102C20001998F5F7E7FE73D2F1491B98F5F7E2FE24
:102C300005D2ED491B98F5F7D6FB1B90E6E2ED496E
:102C40001B98F5F7E1FE0AD8EB491B98F5F7D2FE81
:102C500005D2EA491B98F5F7C6FB1B90D6E2E64978
:102C60001B98F5F7D1FE12D8E5491B98F5F7C2FE7F
:102C70000DD2E4481999F5F7B6FBE3491690F5F73C
:102C800059FB17901B99F5F7AEFB1B90BEE2DC4990
:102C90001B98F5F7B9FE12D8DC491B98F5F7AAFE88
:102CA0000DD2DB481999F5F79EFBDA491690F5F736
:102CB00041FB17901B99F5F796FB1B90A6E2D349B1
:102CC0001B98F5F7A1FE0AD8C2491B98F5F792FEAA
:102CD00005D2C5491B98F5F786FB1B9096E2BD49C6
:102CE0001B98F5F791FE8ED8BB491B98F5F782FE2D
:102CF00089D2C9481B99F5F776FBC8491690F5F7B4
:102D000019FB17901B99F5F76EFB1B907EE2FFE70E
:102D1000C3491998F5F76EFE3FD2C2491B98F5F7E3
:102D200073FE12D8B4491B98F5F764FE0DD2BE4865
:102D30001B99F5F758FBBD491690F5F7FBFA17906C
:102D40001B99F5F750FB1B9060E2AB491B98F5F718
:102D50005BFE0AD8B6491B98F5F74CFE05D2B5497B
:102D60001B98F5F740FB1B9050E2B1491B98F5F713
:102D70004BFE8BD898491B98F5F73CFE86D2AE489F
:102D80001B99F5F730FBAD491690F5F7D3FA17907C
:102D90001B99F5F728FB1B9038E2A9491998F5F71C
:102DA00029FE7BD292491B98F5F724FE0DD2A54847
:102DB0001999F5F718FBA4491690F5F7BBFA179087
:102DC0001B99F5F710FB1B9020E289491B98F5F73A
:102DD0001BFE12D887491B98F5F70CFE0DD29B48B5
:102DE0001B99F5F700FB9A491690F5F7A3FA17908F
:102DF0001B99F5F7F8FA1B9008E27E491B98F5F746
:102E000003FE12D87C491B98F5F7F4FD0DD29148CA
:102E10001B99F5F7E8FA90491690F5F78BFA179099
:102E20001B99F5F7E0FA1B90F0E173491B98F5F751
:102E3000EBFD0AD87E491B98F5F7DCFD05D28749E2
:102E40001B98F5F7D0FA1B90E0E179491B98F5F74C
:102E5000DBFD0AD85F491B98F5F7CCFD05D2754913
:102E60001B98F5F7C0FA1B90D0E15A491B98F5F76B
:102E7000CBFD91D858491B98F5F7BCFD8CD278480A
:102E80001B99F5F7B0FA77491690F5F753FA1790B2
:102E90001B99F5F7A8FA1B90B8E1FFE7724919985A
:102EA000F5F7A8FD73D252491B98F5F7A3FD05D29B
:102EB0006E491B98F5F797FA1B90A7E14C491B98B0
:102EC000F5F7A2FD12D84B491B98F5F793FD0DD2EB
:102ED0005E481B99F5F787FA5D491690F5F72AFACF
:102EE00017901B99F5F77FFA1B908FE141491B98CA
:102EF000F5F78AFD12D840491B98F5F77BFD0DD2F6
:102F000049481B99F5F76FFA59491690F5F712FAE7
:102F100017901B99F5F767FA1B9077E136491B98D4
:102F2000F5F772FD0AD842491B98F5F763FD05D203
:102F30004A491B98F5F757FA1B9067E13C491B98E3
:102F4000F5F762FD0AD823491B98F5F753FD05D222
:102F500038491B98F5F747FA1B9057E11D491B9814
:102F6000F5F752FD98D81C491B98F5F743FD0CD294
:102F700029481B99F5F737FA28491690F5F7DAF939
:102F800017901B99F5F72FFA1B903FE1FFE739499E
:102F90001998F5F72FFD71D215491B98F5F72AFD01
:102FA00005D232491B98F5F71EFA1B902EE1104905
:102FB0001B98F5F729FD68D80F491B98F5F71AFDFE
:102FC00063D224481B99F5F70EFA2B491690F5F7B2
:102FD000B1F954E00000A0430000AF43EA750BB91B
:102FE0002FF9853F000016441283803FEC51A44125
:102FF0000000704200008C420000AA42643B7F3F08
:103000000000F042A69B443B986E723F000048438C
:103010006F12833AC3D37B3F22FC8BB956F28B3FAE
:103020000000DC410000964252499D39713D7A3FD3
:1030300000008C432506813FD6E594B83333833FA7
:10304000713D0642A69BC43AD42B753F17B7D139C0
:1030500048E17A3F17B751392DB27D3F3789813F1B
:1030600017B751B9C3F5883FE17A1E42E926813F7F
:10307000C4427D3F14AE2E4252B87E3F60E01790AE
:103080001B99F5F7B0F91B90C0E068491B98F5F75C
:10309000BBFC0AD866491B98F5F7ACFC05D265491C
:1030A0001B98F5F7A0F91B90B0E061491B98F5F764
:1030B000ABFC0AD860491B98F5F79CFC05D25F4928
:1030C0001B98F5F790F91B90A0E05B491B98F5F76A
:1030D0009BFC12D85A491B98F5F78CFC0DD2594825
:1030E0001999F5F780F958491690F5F723F91790D3
:1030F0001B99F5F778F91B9088E051491B98F5F773
:1031000083FC12D851491B98F5F774FC0DD2504836
:103110001B99F5F768F94F491690F5F70BF91790D9
:103120001B99F5F760F91B9070E048491B98F5F77B
:103130006BFC6BD248491B98F5F755F91B9065E07D
:1031400046491998F5F760FC60D845491B98F5F792
:1031500051FC04D243491B98F5F745F91B904049AF
:103160001B98F5F751FC12D83F491B98F5F742FC24
:103170000DD23E481B99F5F736F93D491690F5F703
:10318000D9F817901B99F5F72EF91B903EE03649B8
:103190001B98F5F739FC12D824491B98F5F72AFC3F
:1031A0000DD234481B99F5F71EF933491690F5F7FF
:1031B000C1F817901B99F5F716F91B9026E01B49EB
:1031C0001B98F5F721FC0AD819491B98F5F712FC52
:1031D00005D22A491B98F5F706F91B9016E0144909
:1031E0001B98F5F711FC11D815491B98F5F702FC4F
:1031F0000CD223481B99F5F7F6F822491690F5F7FB
:1032000099F817901B99F5F7EEF81B901B9818F09A
:10321000A7FD1B9000BF1C491B98F5F7F5FB01D2D9
:1032200019481B901B98FFF79DFB00000000AA4265
:1032300000005C433789813F00008C4360E5803F9C
:103240000000A04352491DBA9CA2833F0000AF4337
:10325000B91C2FB92715873F643B7F3F14AE2E4220
:1032600000000C42D7A3803F0000704217B75139CD
:10327000AED87F3F62BEBC39A3017C3F85EB813F66
:1032800017B7D1B89318843F0060EA46F0B585B00F
:10329000044600270020039002900190FAF74CFEAC
:1032A000002802D10120974908709748007800282B
:1032B00006D0012823D002282AD0032871D111E199
:1032C00000212046F5F796FB18D003F00FFD0A28E1
:1032D00005D18E48F4F7FEFF8D49086004E08D4863
:1032E000F4F7F8FF8A49086003210C200BF04CFB2F
:1032F000002084490870012083490870FFE00C20F9
:103300000BF09CF9002802D102207F490870F6E0FA
:1033100000212046F5F76EFB7ED103F0E7FC0A287A
:103320007BD17A48F4F7D6FF0546794801682846EC
:10333000F5F751F807463F2109063846F5F74BF8EF
:1033400003907F21C9053846F5F745F80290724988
:103350003846F5F740F8019070490298F5F754FBAC
:1033600020D86F490298F5F745FB1BD86748F4F75A
:10337000B1FF06466B490298F5F735F831460090E3
:10338000F5F72DF805466149F4F7BCFF5F48F4F7FF
:10339000A1FF0090F5F7D6FA0546634AF4F7BBFFA4
:1033A0009AE0A8E061490398F5F72EFB1FD8604921
:1033B0000398F5F71FFB1AD85448F4F78BFF06461D
:1033C00058490398F5F70FF831460090F5F707F8DC
:1033D00005464E49F4F796FF4C48F4F77BFF009002
:1033E000F5F7B0FA0546504AF4F795FF74E05149F5
:1033F0000198F5F709FB6FD84F490198F5F7FAFAEC
:103400006AD840480078012866D14048F4F762FF46
:1034100006464A49019801E063E014E0F4F7E3FF4F
:1034200031460090F4F7DBFF05463849F4F76AFFB0
:103430003648F4F74FFF0090F5F784FA05463A4A0C
:10344000F4F769FF48E03348F4F744FF0546304895
:1034500001682846F4F7BFFF074639493846F4F7B4
:10346000BAFF039037493846F4F7B5FF0290364962
:103470000298F5F7C9FA15D834490298F5F7BAFA5F
:1034800010D82448F4F726FF064626490298F4F798
:10349000AAFF31460090F4F7A2FF05461D49F4F754
:1034A00031FF19E02A490398F5F7AEFA14D82949F3
:1034B0000398F5F79FFA0FD81648F4F70BFF064666
:1034C00018490398F4F78FFF31460090F4F787FF0F
:1034D00005461049F4F716FF00200A4908700A490A
:1034E00008700CE000212046F5F784FA02D1002094
:1034F0000549087003E000200349087000BF00BFC1
:1035000005B0F0BDC8060020C3060020EC21002055
:10351000C40600203422002000002041295C0FBD99
:10352000295C0F3DCDCC4C3E7D060020295C8FBC34
:10353000295C8F3CCDCC4CBFCDCC4C3F9A99593FA8
:103540000000FA4300007A4400000CC200000C4264
:1035500000008CC100008C4103480078012800D194
:1035600070470020FCE70000BD03002010B5FBF70A
:10357000CDFFFCF73DF800201549086015490860AB
:1035800015490870154908701549087015490870E3
:103590001549087015490870042015490870002065
:1035A00014490870144908701449087014490860D7
:1035B00014490860144908600EF00CFE10490860B8
:1035C0001920FBF789FAC1B21048C17010BD000084
:1035D000AC030020B0030020B4030020B50300209A
:1035E000B6030020B7030020B8030020BD0300206D
:1035F000B9030020BA030020BB030020BC03002055
:10360000C8030020C0030020C4030020CA0100201A
:10361000F8B500260024FE480078232801D301F0E5
:1036200000F843007B449B885B009F4422005100CC
:10363000A100F60012012F015603D803FA0341043A
:103640005E047E04CB042706DF060607AF07FA07F1
:10365000C407E2074E016A018A01DA01FA07DD00B8
:10366000E70407055705B7050A06D4021D037506CA
:103670009506E84901200006F4F744FEE5481C38A9
:10368000C078102803DD1021E2481C38C170E248E0
:103690000078012802D10020DF4908700EF09AFD61
:1036A000DE4908600120DA490870DD490870002011
:1036B000DC490870DC4908700120DC490860002002
:1036C000DB490860DB48DC490860FBF769FFC4E3BD
:1036D0004E20FBF7F7F900282AD00EF07BFDCF49EA
:1036E0000968401AD549884241D94E20FBF7FCF9B8
:1036F000CC48007801283AD10EF06CFDC74908602B
:103700000020C84908700220C14908700120C4493E
:1037100008700220C54908600420C5490860C848EF
:10372000C5490860C748C8490860FBF739FF1EE073
:10373000BC48007801281AD10EF04CFDB74908604A
:103740000020B84908700220B14908700120B4492E
:1037500008700220B54908600420B5490860B848DF
:10376000B5490860B748B8490860FBF719FFAEE7EC
:10377000AD480078012836D10020AB490870B14827
:10378000C078B249487008464078042108400428AF
:103790000AD10020AE4908600EF01CFD9F49086068
:1037A00019209B4908701EE0A9480068401CA849E0
:1037B000086008460068FF212D3188420ED900209C
:1037C000A34908600220A3490870A348007801219A
:1037D0000843A1490870FDF73BFD04E00120914931
:1037E00008708B49087072E700208E49087003202A
:1037F0008749087001208A4908700EF0EBFC874960
:1038000008600620894908600020894908609348BB
:1038100089490860FBF7C4FE59E78248007801280F
:1038200016D100207F4908700EF0D4FC7B49086057
:103830000420774908700120794908707B490860A5
:1038400000207B49086086487B490860FBF7A8FE9A
:103850003DE774480078012817D10EF0BBFC6F4992
:10386000086000206F490870052069490870012030
:103870006B49087006206D49086000206C4908609B
:1038800078486D490860FBF78BFE20E765480078B3
:10389000012819D10EF09EFC6049086000206149A2
:1038A000087014205A49087001205D4908700620EC
:1038B0005E49086000205E4908606B4908706B48EB
:1038C0005D490860FBF76CFE01E756480078012867
:1038D00016D100205349087015204D4908700EF08C
:1038E00079FC4E49086001204D4908704F49086035
:1038F00000204F4908605E484F490860FBF750FEC2
:10390000E5E64848007801281AD10EF063FC4349E7
:10391000086000204349087016203D4908700120C6
:103920003F4908700220414908600420404908606E
:10393000434841490860434843490860FBF730FE6B
:10394000C5E63948007801284AD100203649087078
:103950003C48C0783D49C8700846C07808210840F6
:1039600008281DD100203A4908602E4908700EF041
:1039700031FC2A4908601720254908700120284990
:103980000870022029490860042029490860394844
:10399000294908602B482C490860FBF701FE1FE00D
:1039A0002B480068401C2A49086008460068FF212F
:1039B0002D3188420ED90020254908600220254972
:1039C0000870254800780121084323490870FDF755
:1039D0003FFC05E001201349087015200C490870D0
:1039E00075E61148007801287DD100200E49087045
:1039F0000C4908700EF0EEFB084908601148007889
:103A00001249C8700F48407888700E48807833E0BB
:103A1000B5030020E6010020BB030020C8030020FE
:103A2000B6030020B8030020B7030020B003002035
:103A3000AC03002080D102009403002050C300009A
:103A400052D102009C030020980300208C0100202A
:103A5000C0030020B9030020BA0300203AD10200BD
:103A600081D1020040D10200A803002046D102000B
:103A700084D102006ED102004870F848C078087006
:103A800000201AE0014609318900F54A525C0146DE
:103A900009318900F24BC918497852180146093199
:103AA0008900C91889785218014609318900C91856
:103AB000C97851180C19411CC8B21028E2DB210644
:103AC000FF221202224012021143FF22120422405E
:103AD000120A1143220E11430846E249F4F712FC80
:103AE000002400201BE075E001464F318900DC4ACC
:103AF000525C01464F318900D94BC9184978521898
:103B000001464F318900C9188978521801464F3152
:103B10008900C918C97851180C19411CC8B22E283F
:103B2000E2DB2106FF221202224012021143FF2291
:103B300012042240120A1143220E11430846C949B9
:103B4000091DF4F7DFFB002004E0C749095C8E196A
:103B5000411C88B20D2189018842F6D33106FF222B
:103B60001202324012021143FF2212043240120AA2
:103B70001143320E11430846BA490831F4F7C2FB2B
:103B8000BA48F4F7A7FBB04210D00620B849087035
:103B90000120B8490870B84908600020B74908609A
:103BA000B748B8490860FBF7FBFC13E01F20B04999
:103BB00008700120AF4908700220AF490860042056
:103BC000AE490860B048AF490860A448AF490860F2
:103BD000FBF7E6FC7BE5AE480078012843D10020E6
:103BE000AB490870AB4908700EF0F4FAAA490860B6
:103BF0009A4800789D4908709848407848709748DE
:103C0000807888709548C078C8709648F4F762FB51
:103C100005469648F4F75EFB854210D0072094498C
:103C20000870012093490870934908600020934967
:103C30000860934893490860FBF7B2FC13E020202A
:103C40008B49087001208B49087002208A4908605E
:103C500004208A49086091488A4908607F488B4956
:103C60000860FBF79DFC32E589480078012833D1D4
:103C7000002087490870874908700EF0ABFA864922
:103C80000860764800787949087074484078487030
:103C90007248807888707148C078C8707148001D7B
:103CA000F4F718FB05467148F4F714FB854203D07E
:103CB00007206F49087002E01E206D49087001203E
:103CC0006C4908706C49086000206C4908606C48B9
:103CD0006C490860FBF764FCF9E46E480078012841
:103CE0007CD1002500206B4908700EF073FA6A49F8
:103CF00008606B480068401E6A490978884235D9D7
:103D00005C206949087067490878C10F0918491093
:103D1000654A517063490878C10F09184910490074
:103D2000411AC907090E917000BF09E05D4800788B
:103D3000C00140194C49095CE81C5B4A11546D1CD8
:103D4000802DF3D301204B49087083204A49086035
:103D500000204A49086054484A490860FBF720FCA3
:103D600050480078401C4F49087036E05C204E49AE
:103D700008704C490878C10F091849104A4A517017
:103D800048490878C10F091849104900411AC90764
:103D9000090E9170002509E042480078C0014019E1
:103DA0003149095CE81C404A11546D1C3F480068C9
:103DB0008542F1D301202F4908703C480068C01C9F
:103DC0002D49086000202D49086037482D490860BA
:103DD000FBF7E6FB07202649087000BF77E42D4873
:103DE000007801281CD10EF0F5F92B49086000205D
:103DF0002849087008201E49087001201D490870D4
:103E0000FF20FF301C49086000201C490860012089
:103E1000184908701248801C1A490860FBF7C0FB5B
:103E200055E41C480078012816D10EF0D3F91A4940
:103E3000086000201749087009200D49087001200A
:103E40000C4908700C49086000200C4908600C48B7
:103E50000C490860FBF7A4FBE4E30EE29C0300209E
:103E6000920100208603002085D102008C010020F1
:103E7000B5030020B6030020B0030020AC030020EF
:103E800082D102009403002070D102009803002028
:103E9000B7030020B8030020C803002072D102003D
:103EA000A0030020A80300203C1D0020A403002044
:103EB000FE480078012817D10EF08CF9FC49086003
:103EC0000020FA4908700A20FA4908700120FA49CE
:103ED00008700620F94908600020F9490860F9488F
:103EE000F9490860FBF75CFB9CE3F0480078012887
:103EF0001AD10EF06FF9EE4908600020EB49087006
:103F00000B20EC4908700120EB4908700220EB49B6
:103F100008600420EA490860EC48EB490860EC4876
:103F2000EC490860FBF73CFB7CE3EB480078012898
:103F300047D10020E8490870E548C078E749C870D3
:103F40000846C0780221084002281AD10020E4491E
:103F500008600EF03FF9D64908600020D349087088
:103F60000C20D44908700120D3490870D349086057
:103F70000020D3490860DB48D3490860FBF710FBF9
:103F80001FE0D7480068401CD54908600846006813
:103F9000FF212D3188420ED90020D149086002202E
:103FA000D1490870D148007801210843CF490870F1
:103FB000FDF74EF905E00120BC4908700A20BD4913
:103FC00008702FE3B9480078012816D10EF002F9E5
:103FD000B74908600020B54908701A20B549087033
:103FE0000120B5490870B54908600020B44908604F
:103FF000BF48B5490860FBF7D3FA13E3AB48007834
:1040000001281AD10EF0E6F8A94908600020A74956
:1040100008701B20A74908700120A74908700220DA
:10402000A64908600420A6490860A848A649086077
:10403000A748A8490860FBF7B3FAF3E2A64800785E
:1040400001284AD10020A4490870A148C078A3499A
:10405000C8700846C0780821084008281DD10020F3
:104060009F490860914908700EF0B4F890490860C3
:104070001C209049087001208F49087002208F4948
:10408000086004208E4908609A488F49086090486B
:1040900090490860FBF784FA1FE091480068401CD3
:1040A0008F49086008460068FF212D3188420ED9EB
:1040B00000208B49086002208B4908708B480078EB
:1040C0000121084389490870FDF7C2F805E0012085
:1040D000764908701A2077490870A3E27E48007874
:1040E00001285AD100207C490870704908700EF0F0
:1040F00071F86F490860764800787849087074480C
:10410000407848707248807888707148C078C8706C
:104110007948F4F7DFF805467048F4F7DBF8854294
:1041200027D076480068401C74490860084600683B
:1041300003280DD90020086002206B4908706B48E5
:1041400000780121084369490870FDF781F824E0EF
:1041500007205849087001205749087057490860DE
:104160000020574908605F4857490860FBF718FA74
:1041700013E01D204F49087001204F4908700220AC
:104180004E49086004204E4908605D484E49086069
:104190004F4850490860FBF703FA43E24E48007865
:1041A00001284DD100204C490870404908700EF09C
:1041B00011F83F490860464800784849087044486B
:1041C000407848704248807888704148C078C8700C
:1041D0004948001DF4F77EF805464048F4F77AF8A0
:1041E00085421AD045480068401C4449086008468A
:1041F000006803280DD90020086002203A490870A1
:104200003A4800780121084338490870FDF720F842
:1042100009E007202749087005E0002037490860B9
:104220001E20244908700120234908702349086092
:104230000020234908602B4823490860FBF7B0F9A8
:10424000F0E11A480078012817D10DF0C3FF184992
:1042500008600020154908700D20164908700120DB
:1042600015490870062015490860002014490860A7
:10427000244815490860FBF793F9D3E10B4800780F
:10428000012848D10DF0A6FF094908600020074920
:104290000870012008490870084908600020084992
:1042A000086019480849086030E00000B8030020A1
:1042B000C8030020B5030020B6030020B00300208F
:1042C000AC03002054D102009403002052D102001C
:1042D0009C03002098030020B70300208C010020DD
:1042E000C003002082D10200B9030020BA030020DD
:1042F00084D1020070D1020086030020C403002094
:1043000072D102005AD1020080D10200FBF748F9B5
:104310002120D549087085E1D448007801281AD1B8
:104320000DF058FFD24908600020D04908702220C3
:10433000CD4908700120CF4908700220CE4908609D
:104340000420CE490860CE48CE490860CE48CF4907
:104350000860FBF725F965E1CD480078012844D1D4
:104360000020CB490870C848C078CA494870084640
:10437000407804210840042817D10020C64908606D
:104380000DF028FFBA4908600120BA490870BA49FF
:1043900008600020B9490860C048BA490860FBF7C6
:1043A000FFF80E20B04908701FE0BB480068401CB1
:1043B000B949086008460068FF212D3188420ED9AE
:1043C0000020B54908600220B5490870B54800785A
:1043D00001210843B3490870FCF73AFF05E00120CA
:1043E000A24908702120A04908701BE19F4800786D
:1043F000012821D10020AC4908709C4908700DF0BB
:10440000E9FE9B490860A948C078A8491431C978D9
:1044100048437D214843C117490E0918C8117D2121
:10442000C900F3F78DFEC01C87B2394608200AF098
:10443000ABFA0F208C490870F4E008200AF0FEF86F
:1044400000280BD102209649087096480078012177
:10445000084394490870FCF7FBFE96E09248007808
:1044600001283ED192480088FF210131084390493C
:10447000088000208F4908708B4908708B48C078ED
:104480008A491431C97848437D214843C117490EF0
:104490000918C8117D21C900F3F752FEC01C87B26C
:1044A000394608200AF070FA0DF094FE7049086051
:1044B00012206D49087001206E49087002206E4973
:1044C00008607A481430C0780C2148436B49086072
:1044D00079486C49086079486C490860FBF760F8D6
:1044E00053E07748007801280BD1F8F7ABFA0128A0
:1044F00007D100206F490870714908705A49087047
:1045000043E0FCF7C3FE01281AD1FCF7D9FE0020D6
:10451000684908700DF05EFE554908601020524948
:104520000870012053490870062053490860002094
:1045300052490860634853490860FBF731F824E0AA
:10454000FCF7A4FE02281AD1FCF7BAFE0020594954
:1045500008700DF03FFE464908601020424908707F
:10456000012044490870062043490860002043495F
:104570000860554843490860FBF712F805E0012040
:104580004C4908700F20384908704BE037480078D4
:1045900001280CD100203E49087034490870364982
:1045A0000860364908600F202F49087002E010208B
:1045B0002D49087036E036480078012815D10020D2
:1045C00033490870294908701320274908700120D1
:1045D00028490870284908600020284908602F48A9
:1045E00028490860FAF7DCFF02E012201E49087033
:1045F00018E01E48007801280FD1002024490870D7
:104600001A4908701C4908601C49086001202449A7
:1046100008700F201449087002E013201249087036
:1046200000E000BF00BF104800780F281BD00E48E4
:104630000078002817D00DF0CDFD0D490968401A0B
:10464000224988420FD317480078022108431549B0
:1046500008700220124908700020084908600649C5
:104660000860FCF7F5FDF8BDB5030020B803002095
:10467000C8030020B6030020B0030020AC030020D4
:1046800052D10200940300209C03002098030020D4
:10469000B70300208C010020C003002082D102005B
:1046A000B9030020BA030020B4030020B6010020A3
:1046B00020090020BD03002060D102007C1C0020E6
:1046C000BB0300207AD1020074D10200B0AD01001A
:1046D0007047000010B525480078002804D0012854
:1046E00012D002283ED12AE002F000FB0A2805D1B0
:1046F00007F0CEFE02201D49087004E000F0B0F87B
:1047000001201A4908702EE002F0F0FA0A2815D1AB
:10471000002002F0EFF9002015490870082000F091
:104720008DF8002013490860134908601349086098
:1047300013481449086002200C49087013E002F085
:10474000D5FA01280DD100200F49088000F088F823
:10475000102000F073F80D480A4908600120034951
:10476000087000E000BF00BF10BD00005C06002024
:1047700032060020087F00200C7F0020187F0020D8
:104780005A6B7C8D107F00201C7F00208D7C6B5A23
:10479000F8B525480078002802D0012840D107E06C
:1047A0003C2105200AF0F0F801201F49087038E08C
:1047B000052009F043FF002831D1022000F0F2F972
:1047C00000901220FAF77EF900281ED11748F3F75F
:1047D00081FD054629460098F3F7FDFD044614497E
:1047E000F4F712F911D21148F3F774FD0446114998
:1047F000F3F788FD0F48F3F76DFD0646F4F7A2F8CE
:1048000004460D4AF3F787FD06E01220FAF76CF92B
:1048100006490098F3F776FD00200349087000E090
:1048200000BF00BFF8BD00001406002015060020E0
:1048300000001643EC2100207D060020082803D14B
:104840000121064A117008E0102803D10221034A11
:10485000117002E00021014A11707047BC03002072
:10486000F0B585B009F0AAFA0546802102F006F9F4
:104870000DF0B0FC964908600421964809F07AFAD8
:10488000012817D00421944809F074FA012811D0A6
:10489000002190480068F4F7ADF80BD38F498D489C
:1048A0000068F4F7B1F805D300218B480068F4F7ED
:1048B000A1F804D2002087490860874908600221D6
:1048C000874809F057FA012802D10020844908805E
:1048D0004D20FAF7F7F8002843D04D20FAF704F9F5
:1048E0007F480088F3F797FF432109060290F3F70A
:1048F000B7FD7C490390F3F71DFD07467548016835
:104900003846F3F770FD0646734801683046F3F702
:1049100011FD05467449F3F7F5FC7448F3F7DAFC2A
:1049200003906F480088F3F776FF43210906009053
:10493000F3F796FD6B490190F3F7FCFC0290654894
:1049400001680298F3F74FFD07466949F3F788FDC0
:1049500006460399F3F7EEFC05466449F3F7D2FCEB
:104960003FE05F480088F3F756FF432109060290B5
:10497000F3F776FD07465F49F3F7DCFC03905548F3
:1049800001680398F3F72FFD064653480168304647
:10499000F3F7D0FC05465449F3F7B4FC5348F3F75A
:1049A00099FC03904E480088F3F735FF4321090630
:1049B0000090F3F755FD07464E49F3F7BBFC019015
:1049C000444801680198F3F70EFD49490290F3F756
:1049D00047FD06460399F3F7ADFC05464349F3F757
:1049E00091FC4248F3F776FC0746F3F7ABFF054628
:1049F000414AF3F790FC00204049086001204049FB
:104A0000087000203F4908703749091DF3F77AFC08
:104A1000354908310020F3F775FC3449083100208E
:104A2000F3F770FC304930310020F3F76BFC2E496E
:104A300034310020F3F766FC2B4938310020F3F7BE
:104A400061FC29493C310020F3F75CFC26494031E8
:104A50000020F3F757FC002405E00020A1002A4ABB
:104A60005050601C84B2102CF7DB40212748F3F72C
:104A70000AFC002405E00020A100254A5050601CDB
:104A800084B2102CF7DB002405E00020A100214AAD
:104A90005050601C84B2142CF7DB002405E0002089
:104AA000A1001D4A5050601C84B21E2CF7DB002070
:104AB0001A4908801A4908701A4908801A4908805A
:104AC0001A4908701A4908601A49087005B0F0BD03
:104AD000440600200C7F0020087F00200080BB449B
:104AE0001C7F00206666164034220020EC21002046
:104AF00000007A443333B33E7D060020187F002047
:104B00005D0600203206002038200020782000209A
:104B1000B8200020F8200020482100202C0600208A
:104B20002E06002020060020220600202406002059
:104B300058060020250600200349C9788900034A49
:104B40008918016070470000CA0100207C1C002009
:104B50000349C978C900034A8918016070470000F9
:104B6000CA0100207C1C002010B50221C02000F0EA
:104B70001DFD012805D1034908700221C02000F065
:104B8000E9FC10BDB403002005480078002804D0DB
:104B9000002003490870012070470020FCE7000056
:104BA000A7060020F8B5044623000FF0F8FF0D6AB1
:104BB000080C2A3D42474C51565B60656A003248FA
:104BC000F3F788FBF8BD30480838F3F783FB054658
:104BD0000021F3F70FFF0FD22B4908390020F3F71C
:104BE00091FB29480838F3F775FB0746F3F7AAFE4F
:104BF0000546264AF3F78FFB23480838F3F76AFB8C
:104C0000E0E72148001FF3F765FB05460021F3F7B5
:104C1000F1FE04D21C49091F0020F3F773FB1A4868
:104C2000001FF3F757FBCDE71748001DF3F752FBC2
:104C3000C8E715480830F3F74DFBC3E712480C30BE
:104C4000F3F748FBBEE710481030F3F743FBB9E732
:104C50000D481430F3F73EFBB4E70B481830F3F778
:104C600039FBAFE708481C30F3F734FBAAE70648E6
:104C70002030F3F72FFBA5E703482430F3F72AFB96
:104C8000A0E70020C0439DE7F42100207D0600201E
:104C9000002014490979134AD27852001143114A6D
:104CA0005279920011430F4A5278D20011430D4AB3
:104CB000127A120111430B4A927852011143094AA8
:104CC000D27992011143074A1278D2011143054A61
:104CD000927912021143034A527A5202114388B266
:104CE000704700008C22002038B50024002000907E
:104CF000FFF7CEFF0446E007C00F002816D0640877
:104D000064003D480078401C3B4908706A46012118
:104D10000220FAF709FF00280BD0374800786946CF
:104D20000978884205DD0120044302E00020324971
:104D3000087004202040002818D004212046884311
:104D400004462E480078401C2C4908706A46012110
:104D50000420FAF7E9FE00280BD0284800786946BD
:104D60000978884205DD0420044302E0002023493D
:104D7000087020202040002818D020212046884399
:104D800004461F480078401C1D4908706A460121EE
:104D90000520FAF7C9FE00280BD0194800786946AB
:104DA0000978884205DD2020044302E000201449F0
:104DB000087008202040002818D008212046884389
:104DC000044610480078401C0E4908706A460121CC
:104DD0000720FAF7A9FE00280BD00A480078694698
:104DE0000978884205DD0820044302E000200549D7
:104DF0000870204638BD0000A10A0020A20A002049
:104E0000A30A0020A40A002010B5044623000FF0D6
:104E1000C6FE0D3C080C11161B20252A2F343C39E8
:104E20003C001B48F3F756FA10BD19480838F3F751
:104E300051FAF9E71648001FF3F74CFAF4E7144863
:104E4000001DF3F747FAEFE711480830F3F742FA8D
:104E5000EAE70F480C30F3F73DFAE5E70C4810306D
:104E6000F3F738FAE0E70A481430F3F733FADBE7F0
:104E700007481830F3F72EFAD6E705481C30F3F749
:104E800029FAD1E703480068CEE70020C043CBE70A
:104E90003C2200201C060020FEB505460C46284694
:104EA000F3F7B9FC07468F21C905F3F7D9FA06468F
:104EB0002046F3F7B0FC31460090F3F794FA07462A
:104EC000F3F7D2FC0190019800F018FDFEBD70B51B
:104ED00004462046F3F79FFC05468F21C905F3F7EA
:104EE000BFFA70BD70B50024F6F71AFE012827D16D
:104EF0002948F3F7EFF9C00FC0070121C90788421D
:104F000010D12548F3F7E6F9C043461C3046FFF7B9
:104F1000DEFF0546214801682846F3F70BFA1F49D2
:104F200008600DE01C48F3F7D5F90646FFF7CFFF00
:104F300005461A4801682846F3F751FA17490860F0
:104F4000164800680121C907484004461449204614
:104F5000F3F750FD04D313492046F3F755FD00D273
:104F600070BD00212046F3F745FD0CD20120C0079B
:104F700044402046F9F7EAFC401EC543064928464E
:104F8000F3F7C0F906E02046F9F7E0FC05460249D0
:104F9000F3F7B8F900BFE3E7FE22002094060020F3
:104FA0000AD723BD0AD7233D014800687047000097
:104FB000107F002010B50D480078002813D10C4850
:104FC000007800280FD10B48007801280BD10A483F
:104FD0000078002807D1FCF753F904210840042881
:104FE00001D1012010BD0020FCE700009806002040
:104FF00091060020A40600201906002010B500200C
:10500000284988704870C870087027490870274977
:10501000087027490870274908702749087005E07B
:10502000F7F788FDF9F7CEFEFBF7CCFE23480078B2
:105030000028F5D00421224808F09CFE01280BD05E
:1050400000211F480068F3F7D5FC05D31D491C4813
:105050000068F3F7D9FC02D21B48194908601B48C5
:1050600000681B4988420AD01848006819498842DC
:1050700005D01748154908601348114908601348BE
:1050800000681449884206D11020FFF7D7FB0020A2
:10509000F9F79EFE04E000200F4908600F49086000
:1050A00010BD00008C2200205C06002019060020A4
:1050B00091060020A406002014060020A606002069
:1050C000387F0020000070420000A041107F0020C7
:1050D0005A6B7C8D8D7C6B5A087F00200C7F0020E2
:1050E000F8B507460C463846F3F795FB05461549D3
:1050F000F3F708F91348F3F7EDF80090F3F722FC03
:105100000546114AF3F707F90E48F3F7E3F80546A9
:105110000E49F3F7F7F80B48F3F7DCF80C49086091
:105120002046F3F778FB05460649091DF3F7EAF830
:105130000448001DF3F7CEF806490860012006492F
:105140000870F8BDEC2100207D0600205E060020DE
:10515000007F0020047F002090060020FEB5FFF7AE
:10516000B9FAFBF7B7F908F0C9FE01F0BFFD0A284C
:1051700056D171480078002802D001284FD122E092
:1051800009F04CFA0821084008281BD1FAF730FB37
:10519000012817D1032009F069FAFAF72FFBF9F774
:1051A000E9FB0DF017F86549086065480078FCF7E1
:1051B00021F9F8F7C1FE002804D1012061490870E7
:1051C0005D4908702BE0FAF713FB012826D1032074
:1051D00009F04CFAFAF712FBF9F7CCFB0CF0FAFFE6
:1051E00056490968401A584908600CF0F3FF5349C2
:1051F0000860554800685549884202D954485249C8
:1052000008604F480078FCF7F5F8F8F795FE01289C
:1052100004D10020484908704A49087000BF84E062
:1052200001F064FD012819D1FAF732FC012815D1EB
:105230000CF0D0FF47490860FAF7DAFA012874D178
:10524000FAF7DCFAF6F706FDF9F794FB3C4800782C
:10525000FCF7D0F82220F9F747FC66E001F046FDA4
:10526000012862D10CF0B6FF3A490968401A3A4960
:1052700088425AD32220F9F725FC002852D1F8F7AA
:105280005BFE012851D135480088F3F7C4FA432169
:1052900009060290F3F7E4F807463149F3F74AF8B4
:1052A0000646304801683046F3F79DF805462E481B
:1052B00001682846F3F73EF804462C49F3F722F834
:1052C0002B48F3F707F8029024480088F3F7A3FA75
:1052D000432109060090F3F7C3F821490190F3F741
:1052E00029F807461F4801683846F3F77CF8064658
:1052F0002049F3F7B5F805460299F3F71BF8044681
:105300001B49F2F7FFFF1A48F2F7E4FF0646F3F7EE
:1053100019FB0446184AF2F7FEFF022004F07AFC5B
:105320000FF088FC2220F9F7DFFBFBF785FCFBF789
:10533000CDFEFFF72DFAFEBD980600209C0600204A
:1053400050060020A0060020B40600208096980099
:1053500080841E0044060020E0C810001C7F00204E
:105360003333B33E0C7F0020087F0020342200201E
:10537000EC21002000007A447D0600200120034932
:10538000087000200249087070470000BD0300202B
:10539000B5030020FEB505465B48066807685B4814
:1053A00005705B480570002D60D0002405E00020EA
:1053B000A100584A5050601C84B2102CF7DB002426
:1053C00005E00020A100544A5050601C84B2142C07
:1053D000F7DB002405E00020A100504A5050601C7B
:1053E00084B21E2CF7DB00204D4908704D4908801F
:1053F0004D4908804D4908804D4908704D49086065
:105400004D4908704D49F2F77DFF4D490020F2F7F4
:1054100079FF4B4928310020F2F774FF48492C31BD
:105420000020F2F76FFF464930310020F2F76AFFA3
:10543000424934310020F2F765FF404938310020FD
:10544000F2F760FF002405E00020A1002E4A505032
:10545000601C84B20A2CF7DB00203A4908703A49F4
:1054600008703A4908703A4908604BE036480078BD
:10547000032840DD00241EE0A100234A5058314695
:10548000F3F7C2FA02D8A0001F490E58A1001E4A25
:1054900050583946F3F7AEFA02D8A0001A490F580F
:1054A000A000194A11582A480068F2F743FF28491A
:1054B0000860601C84B2244800788442DCDB224906
:1054C0000978881EF3F79CF931460290204800685D
:1054D000F2F781FF39460090F2F77DFF01900299C3
:1054E000F2F7BEFF1A490860002017490870012032
:1054F0001649087006E00020134908701349087027
:1055000013490860FEBD0000C02100205D06002098
:1055100031060020B8200020F8200020482100207B
:105520002E0600202C060020200600202206002047
:10553000240600205806002025060020F421002023
:105540003C2200202F0600203006002032060020DA
:105550003406002070B504460D4604496018002248
:10556000294609F013FF002070BD0000100E024014
:10557000F8B504460E4615460548A9004018071917
:1055800001223146384609F001FF0020F8BD000035
:10559000300D024070B504460D4603496018294697
:1055A000FAF752FA70BD0000040D024070B50446CF
:1055B0000D46034960182946FAF746FA70BD000007
:1055C000000E024070B504460E461546214960188B
:1055D0000022314609F0DAFE00201F496118B200AE
:1055E00088502A781B49091F6018314609F0CEFE01
:1055F0006A7818490C396018314609F0C7FEAA7854
:10560000144910316018314609F0C0FEEA7811499A
:1056100014316018314609F0B9FE2A790D49183164
:105620006018314609F0B2FE6A790A4920316018E3
:10563000314609F0ABFE094880680121C90388435F
:10564000A979C9030122D2031140084303498860A4
:10565000002070BD0C0D0240000C0240000F024003
:1056600010B50346024818188C000251002010BDE6
:10567000000C024070B504460D4604496018012232
:10568000294609F083FE002070BD00000C0D024089
:1056900070B504460D461646034960183246294641
:1056A00009F074FE002070BD080D02400146042977
:1056B00001D1024800E002487047000000020040AB
:1056C000004000400146002906D0012907D00229E8
:1056D00007D0032909D106E00120800706E004482D
:1056E00004E0044802E0044800E000BF00BF704747
:1056F00000010040006000400064004070B588B0C8
:10570000044600250026042C01D0052C71D110215F
:10571000684610F043F92046FFF7C8FF05463621DA
:1057200061435D4A891808461030F2F7D3FD81B213
:105730006846418036216143574A8918084614302B
:10574000F2F7C8FDC1B26846417036206043524945
:1057500040180830007E01281AD100206946888050
:105760000CF038F90290362161434B4A89180846FB
:105770001C30F2F7AFFD81B26846C180362161432B
:10578000454A891808460830F2F7A4FD039013E053
:105790000320C002694688804B2149020291012101
:1057A00089026846C180362161433B4A8918084610
:1057B0000830F2F78FFD03903620604336494018D9
:1057C0000830407E69460870284601F025FA00211D
:1057D000284601F0EBF90121284601F0E7F9002104
:1057E000284601F002FA0121284601F0EAF951E0C9
:1057F000FFE7102104A810F0D1F82046FFF762FF60
:10580000064636216143244A891808461030F2F7CB
:1058100061FD81B268464182362161431E4A891882
:1058200008461430F2F756FDC1B2684641740CF0D8
:10583000D1F8069036216143174A891808461C3072
:10584000F2F748FD81B26846818236216143124AEF
:10585000891808460830F2F73DFD0790362060436E
:105860000D4940180830417E6846017404A930464D
:105870000DF054FF002130460DF01AFF0121304693
:105880000DF016FF002130460DF031FF01213046AA
:105890000DF019FF08B070BDF816002070B5044671
:1058A0000A212046F2F74CFC06010A212046F2F7B5
:1058B00047FC7018C5B2284670BD08B5002000909E
:1058C00000BF00980028FCD008BDF8B504460025AC
:1058D00000270FE00A212046F2F732FC8EB2304654
:1058E000B840284385B2381DC7B20A212046F2F7D6
:1058F00027FC84B2002CEDD12846F8BDF8B504464B
:10590000002500270EE00A212046F2F703FC0E4690
:105910003046B8400543381DC7B20A212046F2F789
:10592000F9FB0446002CEED12846F8BD10B500F076
:1059300089F810BD10B5C046C04610BD70B504460C
:105940000D460126002229462046083009F01EFD9A
:105950000026304670BD014601208A6808239A431C
:105960008A60002070470000F8B505460C46012704
:10597000244885420CD12448806A1021884322495A
:1059800088620846806A102108431F4988620BE03C
:105990001D48806A202188431B4988620846806A26
:1059A00020210843184988620020A860207AA86056
:1059B000606800012168884201D90120F8BD207A81
:1059C000402814D10120286061682068F2F7A2FB0A
:1059D000C008401EC6B2092E03DA0021284600F096
:1059E0001FF83146284600F016F8074608E0002068
:1059F0002860607A4000A17A08436072607A28616A
:105A00003846DBE70004004000200040014600204B
:105A1000CA68D0B27047024601205160002070472A
:105A200070B504460D46012601222946204608305D
:105A300009F0ACFC0026304670BD02460120D16062
:105A40000020704710B5F74800780F2871D00CDCA3
:105A50000C284FD004DC00280FD00B286AD117E0A7
:105A60000D2856D00E28F9D192E0153803000FF01A
:105A700096F805FDFCFBFAF961000521EA4800688B
:105A8000FFF75CFF0421E8480068FFF7C9FF9DE2CB
:105A9000E5480068406908280FD10521E248006800
:105AA000FFF74CFF0421E0480068FFF747FFA22101
:105AB000DD480068FFF7C1FF1BE0DB480068406974
:105AC000182816D10C20D74908700521D64800683F
:105AD000FFF734FF0421D4480068FFF72FFFD348B5
:105AE0000088FF22120210400112CF480068FFF721
:105AF000A4FF6BE2CC4800684069282808D10D203B
:105B0000C8490870C9480178C7480068FFF795FF81
:105B10005CE2C5480068406928280CD10521C248CC
:105B20000068FFF77DFF0421BF480068FFF706FF0C
:105B30002DE09CE03CE2BC480068406910281ED182
:105B40000521B9480068FFF7F9FE0421B64800684E
:105B5000FFF7F4FEA321B4480068FFF76EFFB448D6
:105B60000088012805D10221AF480068FFF7E6FE52
:105B70000DE00221AC480068FFF752FF07E0AA4899
:105B800000684069402802D10E20A64908701DE235
:105B9000A54800684069502831D1A54800880028F0
:105BA0005FD0A1480068FFF731FFA249096808707B
:105BB000A0480068401C9F49086005219A48006879
:105BC000FFF7BCFE042198480068FFF7B7FE98482D
:105BD0000088401E9649088008460088012808D1A0
:105BE0000F209049087002218F480068FFF7A6FE39
:105BF00037E002218C480068FFF712FF31E08A4845
:105C00000068406958282CD187480068FFF7FEFEDD
:105C100088490968087087480068401C8549086001
:105C200083480088401E8249088008460088002872
:105C300017D105217C480068FFF780FE04217A48CF
:105C40000068FFF7EDFE0CF0C5FA7B4908607B4861
:105C5000007810218843103078490870002071497D
:105C60000870B3E18CE1C0E078E068E032E06E48B3
:105C70000068406958282CD16B480068FFF7C6FEC1
:105C80006C49096808706B480068401C69490860E5
:105C900067480088401E664908800846008800283A
:105CA00017D1052160480068FFF748FE04215E48CF
:105CB0000068FFF7B5FE0CF08DFA5F4908605F4899
:105CC00000781021884310305C4908700020554945
:105CD00008707BE100205A490880534800684069F9
:105CE00008280FD1052150480068FFF727FE04213E
:105CF0004D480068FFF722FEA2214B480068FFF7DD
:105D00009CFE1BE0484800684069182816D1162000
:105D100044490870052144480068FFF70FFE04213C
:105D200041480068FFF70AFE40480088FF2212023F
:105D3000104001123C480068FFF77FFE46E13A48F8
:105D400000684069282808D117203649087037486C
:105D5000017835480068FFF770FE37E13248006887
:105D60004069282840D132480088401E34490988BB
:105D7000884221D10CF02EFA324908602D48006883
:105D80002F4A1288815C28480068FFF756FE2E488B
:105D9000008801280CD12D480088002808D12C4803
:105DA0000088002804DD2A480088401E2849088011
:105DB00018201C49087017E01D480088401E204923
:105DC0000988884210DD17201649087019480068B4
:105DD0001B4A1288815C14480068FFF72EFE1848A1
:105DE0000088401C16490880F0E00F4800684069B0
:105DF000282816D11448008800282BD1094908709A
:105E00000E4800781021884310300C490870052195
:105E100005480068FFF792FD042103480068FFF77A
:105E2000FFFDACE052000020840000208000002034
:105E300072000020540000206C000020820000202E
:105E400070000020680000207E0000207400002008
:105E50007800002060480088002830D05F48008823
:105E60005F49098840185D4908805E4800685C49C0
:105E7000098840185B4908605B480088002803DDFA
:105E800040205A49088006E0594800885749088050
:105E900000205749088000204F49088019205549A3
:105EA0000870012054490880052154480068FFF714
:105EB00045FD042151480068FFF7B2FD5FE04A4804
:105EC000008800281DDD454800884030434908808F
:105ED00044480068403043490860402043490880F6
:105EE000192044490870012043490880052143488E
:105EF0000068FFF723FD042140480068FFF790FD8C
:105F00003DE03B480088002821DD344800884030CF
:105F100032490880334800684030324908603448CC
:105F20000088324908800020314908801920314911
:105F30000870012030490880052130480068FFF7CB
:105F4000FDFC04212D480068FFF76AFD17E0284892
:105F50000088002813D12A48007810218843103087
:105F6000274908700020234908700521234800684C
:105F7000FFF7E4FC042121480068FFF751FD25E00C
:105F80001E4800684069102811D115201949087071
:105F900005211A480068FFF7D1FC04211748006862
:105FA000FFF7CCFCA22115480068FFF746FD0DE085
:105FB000002010490870052110480068FFF7BEFC5A
:105FC00004210E480068FFF72BFD00BF00BF0B48FF
:105FD0000068FFF7C0FC10BD7400002080000020A6
:105FE000760000205400002078000020720000207D
:105FF0007C000020520000207A0000208400002055
:106000008200002002480078C006C00F70470000E0
:1060100082000020024800788006C00F7047000010
:10602000820000201CB50220F5F7C6FC0721684657
:106030000FF0B4FC002168464170012181700021FD
:10604000C17001714171012181716A4603210020F3
:10605000FFF7B8FA002203211046FFF701FB0122E7
:1060600003210020FFF714FB1CBD10B500F004F85D
:106070000220F5F793FC10BDF0B587B00721684604
:106080000FF08CFC142102A80FF088FC0021684658
:1060900041706A4603210020FFF794FA042203218D
:1060A0000020FFF7DDFA012108200BF0CBFC0021D6
:1060B000684601724173C17201218173017300212D
:1060C0008172417202A90220F5F784FC0BF082FC78
:1060D00007460D49F2F71EF884B201200004001BA8
:1060E00085B229460220F5F711FC01200004001BAF
:1060F00086B231460220F5F719FC01210220F5F79E
:106100003BFC07B0F0BD0000E02801001CB50021F9
:1061100008200BF097FC0220F5F74EFC012202212B
:10612000C802FFF7B5FA072168460FF037FC0021D7
:1061300068464170012181700021C1700171417177
:10614000012181716A460B218020FFF73BFA002272
:106150000B218020FFF79CFA6A460C218020FFF774
:1061600031FA01220C218020FFF792FA6A460321BE
:106170000020FFF727FA002203211046FFF770FAEC
:10618000012203210020FFF783FA1CBD014800789B
:1061900070470000A80C002003480078002801D1B7
:1061A000012070470020FCE7580800201CB5FFF7CD
:1061B00063FF072168460FF0F1FB0021684641703C
:1061C000012181700021C170017101214171817132
:1061D0006A460221C802FFF7F5F901220221C8022E
:1061E000FFF756FA0CF0D5FC00200349087029206F
:1061F000F8F7EEFD1CBD00005808002010B52B4834
:106200000078002804D0012821D0022848D129E0B4
:106210002920F8F757FC00280BD02920F8F764FC58
:106220004B21C900112009F081F801201F49087095
:106230000CE000F077F8012808D100F087F8C821B9
:10624000112009F073F80120184908702CE004208F
:106250000CF01EFB012804D10CF09BFC022013491A
:10626000087021E01120F5F705FC002817D1042063
:106270000CF00EFB012812D100F038FD0A280ED1D7
:10628000F9F746FC00280AD1F8F792FD012806D15B
:106290000CF040FC00F05AF800200449087003E0BC
:1062A00000200249087000BF00BF10BD5808002040
:1062B00010B507480078012808D11020F5F7DAFB5F
:1062C000002803D102490870FFF7ACFE10BD0000A2
:1062D000D400002010B500240BF07CFF05490968AC
:1062E000441A05480068844201D3002010BD0120F3
:1062F000FCE700002C0400202804002010B5002436
:106300000BF068FF05490968441A05480068844293
:1063100001D3002010BD0120FCE700002404002070
:106320002004002001480078704700000908002080
:106330000146024800780840704700000708002026
:1063400001480078704700001B040020002001492C
:106350000870704709080020014603480078884308
:10636000014A10700120704707080020002801DD55
:10637000082800DD7047421E01239340D9B2034A2A
:1063800012788A43014B1A7000BFF3E71B04002008
:1063900003480078002801D1012070470020FCE765
:1063A0001904002003480078002801D1012070471B
:1063B0000020FCE70608002010B50BF0CBFC03F032
:1063C000DBFB10BD00200349087003490870034936
:1063D0000870704706080020070800200808002001
:1063E00010B579480078002802D001286FD1D3E099
:1063F000FFF7A6FF754908700846007803000EF005
:10640000CEFB09065067B0A0B0B0B097B0000D2029
:10641000F8F762FB000E6E490978884215D00D200E
:10642000F8F75AFB000E6A4908700D20F8F754FB84
:10643000000EAA2803D12C20F8F7CAFC05E00022A0
:10644000062141208001FFF723F92C20F8F73AFBC1
:10645000002822D00D20F8F73FFB000EAA281CD1FF
:106460002C20F8F741FB0BF0BDFC002811D10022D5
:1064700003210220F6F706FE0022062141208001BA
:10648000FFF706F90A21202008F050FF01204E49AD
:10649000087000204F49087002E000204A49087047
:1064A00078E00120FFF762FF0020484908704A4861
:1064B00000780121084348490870012047490870C5
:1064C0005A20F8F785FC00203F49087062E077E029
:1064D0000220FFF74BFF00203C49087000F0FAFB58
:1064E000FF21053188420ED11F20F8F7F5FA002868
:1064F00009D039480078082108433749087000203E
:106500003149087013E000F0E5FB3549884205D1B8
:1065100031480078202108432F4908702E48007820
:10652000022108432C49087000202749087031E0F7
:106530000420FFF71BFF002024490870224908703F
:1065400028E00320FFF712FF0020204908702248AE
:106550000078042108432049087000201A49087077
:1065600018E00120FFF702FF0220FFF7FFFE0320E3
:10657000FFF7FCFE0420FFF7F9FE0520FFF7F6FE0B
:106580000620FFF7F3FE0720FFF7F0FE0820FFF7D5
:10659000EDFE00BF00BF14E02020F5F76BFA0128E4
:1065A0000DD10122062141208001FFF771F801225F
:1065B00003210220F6F766FD00200349087000E081
:1065C00000BF00BF10BD0000060800200808002022
:1065D0000A0800200B0800200708002009080020F6
:1065E0000203000010B5F848007803000EF0D7FA57
:1065F0000A064C9EBEFAF9F8F7F6F5F4F34800786F
:10660000002812D00020F14908702220F5F732FA54
:1066100000280AD12320F5F72DFA012805D1EC48EE
:10662000007808210843EA490870F5F78DFAE9492E
:10663000087008460078002814D00846007800F05A
:10664000D0F9012805D1F5F711FB0020DE490870CB
:1066500019E0F5F70BFB022000F0F2F90120DA490E
:10666000087010E03220F8F72DFA002808D0322008
:10667000F8F73AFA0020D84908802C20F8F7A8FB50
:106680000020D14908709CE1FFF738FE002849D16D
:10669000D048007800F0A5F9012806D1022000F0CA
:1066A000CFF90220C84908703FE0CC480078401C70
:1066B000C0B2CA49087001282DDBC64800780228FC
:1066C00018D1C5480088401CC34908800846008886
:1066D0001E2816DD0022062141208001FEF7D8FF8A
:1066E000BB48007804210843B94908700020B64926
:1066F000087010BDB84800881E2802DD3220F8F767
:1067000067FBB348007801210843B14908700320B2
:10671000AD49087002E00120AB490870022000F08A
:106720008FF902E00120A84908704AE1FFF7E6FD71
:10673000002817D1A748007800F053F9012808D1A4
:106740000020A6490870F5F791FA00209E490870CC
:106750000BE0F5F78BFA022000F072F901209A495C
:10676000087002E00220984908702AE1FFF7C6FD90
:1067700000285BD19748007800F033F9012806D152
:10678000022000F05DF904208F49087051E0934821
:106790000078401CC0B291490870C8283FDB8D4882
:1067A000007802281FD18C480088401C8A49088044
:1067B000084600881E281DDD002206214120800198
:1067C000FEF766FF8248007804210843804908707C
:1067D00000207D4908708CE7EFE0D4E0A6E08EE071
:1067E00070E044E026E07C4800881E2802DD32206C
:1067F000F8F7EEFA764800780221084374490870E9
:106800000120724908700021222008F08FFD962196
:10681000232008F08BFD05206B49087002E003205F
:1068200069490870022000F00BF902E00320664974
:106830000870C6E0FFF762FD002814D165480078B3
:1068400000F0CFF8012805D10020644908705E49A6
:1068500008700BE0F5F70AFA022000F0F1F80320C7
:106860005949087002E0042057490870A9E0FFF771
:1068700045FD002822D15748007800F0B2F80128E1
:1068800006D1022000F0DCF806204F49087018E01D
:10689000FFF756FD02210840002808D14F49087033
:1068A0001E2000F0BBF807204749087009E00220CD
:1068B00000F0C6F805204449087002E0052042496E
:1068C00008707EE0FFF71AFD002814D141480078D7
:1068D00000F087F8012805D10020404908703A49A6
:1068E00008700BE0F5F7C2F9022000F0A9F80520C6
:1068F0003549087002E006203349087061E0FFF76F
:10690000E9FC00280BD13549087031480078042192
:1069100008432F49087000202B49087005E0022029
:1069200000F08EF80820284908704AE0FFF7E6FCDE
:10693000002824D12748007800F053F8012806D118
:10694000092021490870022000F07AF81AE0234853
:106950000078401CC0B22149087064280BDB00207D
:1069600008701B4800780221084319490870072065
:106970001549087006E007201349087002E0082056
:10698000114908701DE0FFF7B9FC002811D111482A
:10699000007800F026F8012805D100200F49087082
:1069A0000949087008E0F5F761F907200649087001
:1069B00002E009200449087003E000200249087041
:1069C00000BF00BF00BF94E6190400201C04002093
:1069D0001B04002030040020320400201A04002090
:1069E000704710B50446022C04D10A21802000F023
:1069F00007F810BD0B210120000300F001F8F8E7B3
:106A000070B504460D4629462046FEF7C3FD002812
:106A100001D0012070BD0020FCE7000010B5044645
:106A200004486043044908600BF0D4FB0349086044
:106A300010BD000040420F00280400202C0400205C
:106A400010B504467D20C000604381004018034912
:106A500008600BF0BFFB0249086010BD2004002055
:106A600024040020704710B5C046C04610BD10B5C4
:106A700002F026FFC046C04610BD00003EB50446E9
:106A80000D460A2168460EF089FF012109200AF00F
:106A9000D9FF0721684601700021C1708170002C68
:106AA00003D003206946487002E00220694648701E
:106AB0000021684601714171012181710804401B68
:106AC00081B2684601816946094802F03AFF0848E8
:106AD00002F012FF0121064802F021FF01220321EA
:106AE0001120F6F7CFFA0121014802F00EFF3EBD5A
:106AF000000F004010B50446012C08D101210920E7
:106B00000AF0A0FF0121064802F0FFFE07E0002185
:106B100009200AF097FF0021014802F0F6FE10BD9F
:106B2000000F00400149096888B27047400F0040DB
:106B30003EB504460A2168460EF030FF01212420AC
:106B40000AF080FF0721684601700021C170817042
:106B5000002C03D003206946487002E002206946F9
:106B60004870002168460171417181710181694657
:106B7000094802F0E6FE084802F0BEFE0021064881
:106B800002F0CDFE012203211120F6F77BFA01214C
:106B9000014802F0BAFE3EBD400F004010B502F0C1
:106BA000A1FE10BD10B502F0A2FE10BD70B50446E6
:106BB0000D46002229462046143008F0E7FB00204D
:106BC00070BD70B504460D4600222946201D08F010
:106BD000DDFB002070BD70B504460D46012229463C
:106BE000201D08F0D3FB002070BD70B504460D4693
:106BF00001222946201D08F0C9FB002070BD70B598
:106C000004460D460026294620461030F8F71CFFA2
:106C10000646304670BD0000F0B587B005460C460C
:106C20000127224A07CA04AB07C300200390002CA7
:106C300002D1042007B0F0BD002068606088617850
:106C40000843E1880843A188084321780843686025
:106C50002078402802D02078C02824D1E088C117AD
:106C6000C90D09184912890004AA515A8EB2E16867
:106C7000B1400846F1F7CFFD0290A068F1F7CBFDD7
:106C800001900299F1F7ECFB03903F21090603986C
:106C9000F1F750FB0290F1F7E7FD80B2A861042103
:106CA0002846FFF798FF00273846C3E700D60200C2
:106CB00001460868C0B2704702461068000A000228
:106CC000CBB2184310600020704710B502F0A4FE4C
:106CD00010BD00000348007800020349097808430A
:106CE000704700008F0700209007002003480078BD
:106CF000042801D1012070470A20FCE78F070020FB
:106D000010B501201749087017490020F1F7FAFA69
:106D10001321002001F0E4FB1321012001F0E0FB2E
:106D20001321022001F0DCFB1321032001F0D8FB2A
:106D30001321042001F0D4FB1321052001F0D0FB26
:106D40001321062001F0CCFB1321072001F0C8FB22
:106D50001321082001F0C4FB1321092001F0C0FB1E
:106D600010BD00003F04002040040020032803D091
:106D7000072801D0082833D14F49096A82004F4BB8
:106D80009A58120991434C4A116281004C4A515859
:106D9000090982004B4B9A5812091143464A526A1C
:106DA0008A4345494A628100474A5158090982008D
:106DB000464B9A58120911433F4A926A8A433E4908
:106DC0008A628100424A515809098200414B9A580F
:106DD00012091143384AD26A8A433749CA626AE0C3
:106DE00002283CD13449C96A8200394B9A581209A9
:106DF0009143314AD1621146896A8200324B9A58D6
:106E0000120991432C4A91621146496A82002C4B27
:106E10009A5812099143284A51621146096A820020
:106E2000264B9A5812099143234A11621146496828
:106E30008200244B9A5891431F4A51601146C968F9
:106E40008200244B9A5891431B4AD16011468968AD
:106E500082001E4B9A589143174A91602BE01649C5
:106E600009688200154B9A589143134A11608100BA
:106E7000134A51588200134B9A5811430E4A5268D4
:106E80008A430D494A6081000F4A515882000F4BD6
:106E90009A581143084A92688A4307498A608100D8
:106EA0000B4A515882000B4B9A581143024AD26840
:106EB0008A430149CA607047405C004040D50200E7
:106EC00018D5020068D50200F0D40200B8D502003F
:106ED000C8D4020090D50200F8B505460C462B0038
:106EE0000DF05DFE140B2532485E7287A1B0CFF421
:106EF000F2F1F0EFEEEDECEBEAE9A000D44908582E
:106F0000A100D44A515808430090A000D24E3058F6
:106F1000A600D24FBE5930430246A000D04E33588F
:106F2000A000D04E3158204602F0ECFB8EE100204C
:106F30000090A000CA490B58A000C7490A58002178
:106F4000204602F0DFFB81E1A000C1490858009013
:106F5000A000C34E3058A600C34FBE59304303466D
:106F6000A000BE4E3258A000BE4E3158204602F05E
:106F7000C9FB6BE1A000B64908580090A000B84ECC
:106F80003058A600B84FBE5930430346A000B24E59
:106F90003258A000B34E3158204602F0B3FB55E101
:106FA000A000AC4908580090A000AD490858A100C5
:106FB000AD4E715808430346A000A7490A58002166
:106FC000204602F09FFB41E1A000A1490858A10022
:106FD000A04A515808430090A000A34E3358A00087
:106FE0009D4E3258A0009F4E3158204602F08AFB39
:106FF0002CE1A00096490858A100964A5158084330
:107000000090A000944E3058A600944FBE593043D3
:107010000246A000944E3358A000924E31582046AC
:1070200002F070FB12E1A000894908580090A0000E
:107030008B490B58A00088490A580021204602F0CD
:1070400061FB03E1A00082490858A100814A515820
:1070500008430090A000824E3058A600824FBE59CF
:1070600030430346A0007C4E3058A6007B4FBE59EB
:1070700030430246A0007B4E3158204602F042FBCE
:10708000E4E0A00072490858A100724A5158084330
:107090000090A000724E3058A600734FBE59304386
:1070A0000346A0006C4E3258A0006E4E3158204668
:1070B00002F028FBCAE0C8E0C3E0B7E0A5E08CE03E
:1070C00078E062E048E034E01DE0FFE7A0006049BE
:1070D0000858A1005F4A515808430090A000604939
:1070E0000858A100604E715808430346A0005A4951
:1070F0000858A100594E7158084302460021204605
:1071000002F000FBA2E0A000524908580090A00045
:10711000514E3058A600514FBE5930430246A00090
:10712000514E3358A0004F4E3158204602F0EAFA33
:107130008CE0A00046490858A100464A515808432F
:107140000090A000454B1A58A000464B1958002348
:10715000204602F0D7FA79E000200090A000404ECF
:107160003058A600404FBE5930430346A0003A4E67
:107170003058A600394FBE5930430246A000394E60
:107180003158204602F0BEFA60E0A00030490858AD
:10719000A100304A515808430090A000324E3358A5
:1071A000A0002E4E3258A0002E4E3158204602F03C
:1071B000A9FA4BE0A00026490858A100254A5158D9
:1071C00008430090A00028490B58A00023490A5802
:1071D0000021204602F096FA38E0A0001C49085829
:1071E000A1001C4A515808430090A0001C490858AF
:1071F000A1001D4E715808430346A00017490A58C4
:107200000021204602F07EFA20E0A0001149085833
:107210000090A000144E3358A000104E3258A00029
:10722000104E3158204602F06DFA0FE00020009019
:10723000A0000D490B5800221146204602F062FAC8
:1072400004E02046FFF792FD00E000BF00BFF8BD5C
:10725000C8D4020090D5020018D5020068D50200FB
:10726000F0D4020040D50200B8D5020010B5FDF7F9
:107270000FFD4A4908704A480078002802D00128CA
:107280007ED138E005F0C2FE46490978884206D032
:1072900005F0BCFE434908700120414908703F4891
:1072A00000782021084040490978884208D03B48AE
:1072B0000078202108403C490870012038490870B6
:1072C00014F00AFC39490978884206D014F004FC0D
:1072D0003649087001203249087014F0DFFB344948
:1072E0000978884206D014F0D9FB31490870012092
:1072F0002B49087050E005F089FE0A2803D10120CF
:1073000001F0C8FB02E0002001F0C4FB2648007831
:10731000202803D1012001F001FB02E0002001F050
:10732000FDFA22480078012802D101F081F802E03C
:10733000002001F07DF81E480078012802D101F0FC
:10734000E5F802E0002001F0E1F81A480078002892
:1073500003D1012001F03EF802E0002001F03AF8EC
:1073600015480078032807D013480078042803D074
:1073700011480078052804D1012001F06BFB03E0DF
:1073800006E0002001F066FB00200549087003E0DC
:1073900000200349087000BF00BF10BD9707002000
:1073A0008C070020910700209207002093070020FF
:1073B000940700209507002096070020F3B583B0BE
:1073C0000E46092700BF0398029000210298F1F7AA
:1073D00011FB03D2F90702984840029033000DF0E8
:1073E000DEFB06040F1C2937455358480299F0F775
:1073F000FAFF029001F06EFB019001F0A7F84BE05C
:1074000053480299F0F7EFFF029001F063FB5149F6
:107410000843019001F09AF83EE04F480299F0F7D6
:10742000E2FF029001F056FB4C490843019001F045
:107430008DF831E04A480299F0F7D5FF029001F04B
:1074400049FBE121C9040843019001F07FF823E0E2
:1074500044480299F0F7C7FF029001F03BFB61211D
:1074600009050843019001F071F815E03E480299C2
:10747000F0F7B9FF029001F02DFB212149050843E7
:10748000019001F063F807E00298029001F022FBFE
:10749000019001F05BF800BF00BF0298F1F7F8F926
:1074A00004460D46204629460023584059400843CB
:1074B00020D016E00A22002320462946F0F754FE89
:1074C000D0B239467A1E57B20190C8B2019901F084
:1074D00007F80A22002320462946F0F745FE044615
:1074E0000D460021084661406840014306D0002F48
:1074F000E0DA03E00021092000F0F2FF002E15DDA4
:10750000062E13DA01F0E6FA0121C906B14008435C
:10751000019001F01BF806E039467A1E57B2C8B256
:10752000002100F0DDFFF01CB842F5DD002F0BDB81
:1075300000210398F1F75EFA06D239467A1E57B257
:10754000C8B2122100F0CCFF05B0F0BD0024744990
:107550000050C3470000C20700401C4600008407DB
:1075600000007A440000C84200002041F8B50746F8
:107570000C460825002F16D010E00A213846F0F7F7
:10758000C9FD009129466A1E55B2C8B2009900F0A3
:10759000A7FF0A213846F0F7BDFD0746002F19D096
:1075A000002DEADA16E00620001BC6B208E02946E4
:1075B0006A1E55B2C8B2002100F092FF701EC6B21A
:1075C000002E01D0002CF2D1002C03D10021082084
:1075D00000F086FF23000DF0E2FA05040A131C25D3
:1075E0002E0001F077FA009000F0B0FF29E001F0E2
:1075F00071FA012149040843009000F0A7FF20E040
:1076000001F068FA012189040843009000F09EFF10
:1076100017E001F05FFA0121C9040843009000F06F
:1076200095FF0EE001F056FA01210905084300908C
:1076300000F08CFF05E001F04DFA009000F086FFAD
:1076400000BF00BFF8BD0000F8B50446FFF758FBC7
:1076500023000DF0A4FA06CE042B7998CBCE01209E
:10766000400200F073FF02206B4908700846007862
:10767000F8F7D0F869490860084600680090684942
:107680000098F1F7B7F908D266490098F0F7E8FEDC
:1076900005460121FFF792FE07E062490098F0F7E6
:1076A000DFFE05460321FFF789FEB3E05E4800F0E8
:1076B0004DFF03205849087008460078F8F7AAF8EB
:1076C0005649086008460068009058490098F1F74C
:1076D00091F90BD253490098F0F7C2FE0121C90776
:1076E000484005460321FFF769FE2CE05049009809
:1076F000F1F780F90BD24B490098F0F7B1FE012168
:10770000C907484005460421FFF758FE1BE04949D8
:107710000098F1F76FF90BD242490098F0F7A0FEFC
:107720000121C907484005460521FFF747FE0AE049
:107730003C490098F0F794FE0121C90748400546EE
:107740000621FFF73BFE65E00720400200F0FEFE49
:1077500001203149087008460078F8F75BF82F4996
:10776000086008460068F1F756F807468F21C905FA
:10777000F0F776FE06462A49F0F772FE054601212B
:10778000FFF71CFE46E00120C00200F0DFFE55209E
:107790002149087008460078F8F73CF81F4908604E
:1077A000084600680A280DD20021072000F098FE44
:1077B0000021062000F094FE002118480068FFF721
:1077C000D5FE12E015480068642809D20021062081
:1077D00000F086FE002111480068FFF7C7FE04E0B4
:1077E00000210E480068FFF7C1FE13E000F040FEE4
:1077F00010E00E21022000F073FE0E21032000F0A5
:107800006FFE0A21042000F06BFE0121052000F02C
:1078100067FE00BF00BFF8BD980700209C0700204E
:1078200000007A440000C8420002000800247449A5
:107830008096184B20BCBE4CFEB50446FFF760FA9C
:1078400001F048F9054600F081FE23000DF0A7F98C
:107850000FFD0945819FD0FCFBFAF9F8F7F6F5F426
:10786000FD001120FE49087008460078F7F7F2FF86
:10787000FC490860084600680002010F012000F082
:107880002FFEF84800680003010F022000F028FED8
:107890001221032000F024FEF24800880004010FAA
:1078A000042000F01DFEEF4800880005010F0520B0
:1078B00000F016FE1221062000F012FEE9480078C2
:1078C0000006010F072000F00BFEE64800780107D4
:1078D000090F082000F004FE56E32220E04908705A
:1078E00008460078F7F7B6FFDE49086008460068EA
:1078F0000002010F012000F0F3FDDA4800680003E8
:10790000010F022000F0ECFD1221032000F0E8FD41
:10791000D44800880004010F042000F0E1FDD148A4
:1079200000880005010F052000F0DAFD1221062075
:1079300000F0D6FDCB4800780006010F072000F0CC
:10794000CFFDC84800780107090F082000F0C8FDE6
:107950001AE30121084600F0C3FD1221022000F0C5
:10796000BFFD0120BE49087008460078F7F772FF96
:10797000BC490860096809090A225143B94A1278CA
:107980001207120F88180021FFF7F0FDFCE2022118
:10799000012000F0A5FD1221022000F0A1FD02202F
:1079A000AF49087008460078F7F754FFAD49086002
:1079B0000120C00400F0CAFDAA480068010F05209C
:1079C00000F08EFDA74800680001010F062000F0BE
:1079D00087FDA44800680002010F072000F080FD29
:1079E000A04800680003010F082000F079FDCBE2F9
:1079F0000321012000F074FD1221022000F070FD2F
:107A000003209749087008460078F7F723FF954947
:107A10000860084600680002010F032000F060FDC6
:107A2000904800680003010F042000F059FD8D48C4
:107A300000880004010F09E07CE149E116E1EBE078
:107A4000C7E0A3E07FE05BE019E09CE2052000F0E6
:107A500047FD844800880005010F062000F040FD26
:107A6000804800780006010F072000F039FD7D48AE
:107A700000780107090F082000F032FD84E204209D
:107A80007749087008460078F7F7E4FE7549086002
:107A900008460068010F012000F022FD71480068CF
:107AA0000001010F022000F01BFD6E48006800027B
:107AB000010F032000F014FD6A4800680003010F65
:107AC000042000F00DFD674800880004010F052028
:107AD00000F006FD634800880005010F062000F055
:107AE000FFFC604800780006010F072000F0F8FC5A
:107AF0005C4800780107090F082000F0F1FC43E220
:107B00000421012000F0ECFC1221022000F0E8FC2E
:107B100005205349087008460078F7F79BFE514945
:107B2000086008460068F0F791FE00224E4B019174
:107B30000090F0F7EDFD0546F0F740FF0746032102
:107B4000FFF73CFC20E20521012000F0C9FC1221D6
:107B5000022000F0C5FC0620414908700846007864
:107B6000F7F778FE3F49086008460068F0F76EFEB8
:107B700000223D4B01910090F0F7CAFD0546F0F759
:107B80001DFF07460321FFF719FCFDE10621012037
:107B900000F0A6FC1221022000F0A2FC07203049D0
:107BA000087008460078F7F755FE2E490860084629
:107BB0000068F0F74BFE054600222B4BF0F7A8FDBE
:107BC00001910090F0F7FAFE07460321FFF7F6FB5C
:107BD000DAE10721012000F083FC1221022000F0ED
:107BE0007FFC08201E49087008460078F7F732FE2F
:107BF0001C49086008460068F0F728FE00221A4B6E
:107C000001910090F0F784FD0546F0F7D7FE074696
:107C10000321FFF7D3FBB7E10821012000F060FC4E
:107C20001221022000F05CFC09200D490870084672
:107C30000078F7F70FFE0B49086008460068F0F778
:107C400005FE0022084B01910090F0F761FD05460A
:107C5000F0F7B4FE07460321FFF7B0FB94E1000004
:107C600099070020A00700200000F0400921012012
:107C700000F036FC1221022000F032FC0A20C34939
:107C8000087008460078F7F7E5FDC1490860012053
:107C9000C00400F05BFCBE4800880004010F052012
:107CA00000F01EFCBA4800880005010F062000F015
:107CB00017FCB74800780006010F072000F010FC01
:107CC000B34800780107090F082000F009FC5BE1C8
:107CD0000A21012000F004FC1221022000F000FC27
:107CE0000220AA49087008460078F7F7B3FDA849B2
:107CF00008600120C00400F029FCA54800880004A9
:107D0000010F052000F0ECFBA14800880005010FE1
:107D1000062000F0E5FB9E4800780006010F0720D2
:107D200000F0DEFB9A4800780107090F082000F0F8
:107D3000D7FB29E10B209549087008460078F7F732
:107D400089FD93490860084600680190084600785C
:107D5000012836D10B21002000F0C2FB12210120A6
:107D600000F0BEFB68460179022000F0B9FB122149
:107D7000032000F0B5FB694648790A21F0F7E0F9E5
:107D8000C5B22946042000F0ABFB694648790A21B8
:107D9000F0F7D6F9CDB22946052000F0A1FB12215B
:107DA000062000F09DFB68468179072000F098FBD3
:107DB0001221082000F094FB6846C179092000F0E8
:107DC0008FFB73480078022836D10B21002000F089
:107DD00087FB1221012000F083FB68460179022015
:107DE00000F07EFB1221032000F07AFB69464879FF
:107DF0000A21F0F7A5F9C5B22946042000F070FB6E
:107E0000694648790A21F0F79BF9CDB22946052049
:107E100000F066FB1221062000F062FB68468179C3
:107E2000072000F05DFB1221082000F059FB684696
:107E3000C179092000F054FB55480078032878D117
:107E40001221002000F04CFB694648796421F0F7CC
:107E500077F9C5B22946012000F042FB694648790E
:107E60000A21F0F76DF906460A21F0F769F9CDB25B
:107E70002946022000F034FB694648790A21F0F7D0
:107E80005FF9CDB22946032000F02AFB69468879C4
:107E90008021084000281CD01221042000F020FB83
:107EA000694689794806400E0A21F0F749F9C5B2BA
:107EB0002946052000F014FB694689794806400EE2
:107EC0000A21F0F73DF9CDB22946062000F008FB63
:107ED00017E01321042000F003FB694688790A218A
:107EE000F0F72EF9C5B22946052000F0F9FA6946E7
:107EF00088790A21F0F724F9CDB22946062000F04E
:107F0000EFFA1321072000F0EBFA6946C8790A213D
:107F1000F0F716F9C5B22946082000F0E1FA6946E3
:107F2000C8790A21F0F70CF9CDB22946092000F0F2
:107F3000D7FA17480078042824D10B21002000F03C
:107F4000CFFA1221012000F0CBFA684641790220D5
:107F500000F0C6FA1221032000F0C2FA69468879BF
:107F60000A21F0F7EDF8C5B22946042000F0B8FA6E
:107F7000694688790A21F0F7E3F8CDB22946052051
:107F800000F0AEFA00E000BF00BFFEBD9907002080
:107F9000A007002070B50446FEF7B2FE00F09AFD7F
:107FA000054600F0D3FA012C02D0022C79D14DE025
:107FB0000121084600F094FA1221022000F090FA04
:107FC00001204B49087008460078F7F7C3FC49497F
:107FD0000860084600784007C00F002804D001213F
:107FE000052000F07DFA03E00021052000F078FA7A
:107FF000404800780007C00F002804D00121062067
:1080000000F06EFA03E00021062000F069FA39481A
:108010000078C007C00F002804D00121072000F01D
:108020005FFA03E00021072000F05AFA3148007897
:108030008007C00F002804D00121082000F050FA6A
:1080400003E00021082000F04BFA4FE0022101205C
:1080500000F046FA1221022000F042FA02202449E0
:10806000087008460078F7F775FC22490860084652
:108070000078C006C00F002804D00121052000F0C0
:108080002FFA03E00021052000F02AFA19480078B1
:108090008006C00F002805D00121062000F020FA3C
:1080A00004E022E00021062000F01AFA11480078CE
:1080B0004006C00F002804D00121072000F010FA6C
:1080C00003E00021072000F00BFA0A4800780006C0
:1080D000C00F002804D00121082000F001FA03E0BD
:1080E0000021082000F0FCF900E000BF00BF70BDD7
:1080F0009A070020A4070020F0B587B00546FEF7D8
:10810000FFFD2B000CF04BFD07FD052755A8E3FCF8
:10811000FD00A648407A552804D10120400200F015
:1081200015FA03E00520C00100F010FA0220A04972
:10813000087008460078F7F759FC9E490860084621
:10814000006805909C490598F0F78AF906460121D8
:10815000FFF734F926E19548407A552804D10720E5
:10816000400200F0F3F903E01D20C00100F0EEF939
:1081700001208F49087008460078F7F737FC8D49D1
:10818000086008460068F0F761FB064600228B4B4A
:10819000F0F7BEFA00228A4B01910090F0F7B8FA8E
:1081A00003910290F0F70AFC01210490FFF706F911
:1081B000F8E07E48407A552804D10120C00200F042
:1081C000C5F903E01120C00100F0C0F90A20784988
:1081D000087008460078F7F709FC764908600846F9
:1081E00000680121C907884219D372480068884392
:1081F0007049086008460068F0F728FB0646002230
:108200006E4BF0F785FA00226E4B01910090F0F76B
:1082100017FA03910290F0F7D1FB044613E065488A
:108220000068F0F713FB06460022644BF0F770FA83
:108230000022654B01910090F0F702FA0391029041
:10824000F0F7BCFB044661492046F0F709F9064601
:108250000021FFF7B3F8A5E05448407A552804D12F
:108260000120C00200F072F903E01120C00100F00B
:108270006DF90121084600F033F91221022000F0C7
:108280002FF904204A49087008460078F7F7AEFB3A
:108290004849086008460068F0F7D8FA0646002208
:1082A000464BF0F735FA0022474B01910090F0F76A
:1082B000C7F903910290F0F781FB04464449204638
:1082C000F0F7CEF806460021FFF778F86AE0374865
:1082D000407A552804D10120C00200F037F903E0AC
:1082E0001120C00100F032F90221012000F0F8F85D
:1082F0001221022000F0F4F807202D49087001E057
:1083000023E03EE008460078F7F770FB2949086053
:1083100008460068F0F79AFA06460022274BF0F765
:10832000F7F90022284B01910090F0F789F90391A9
:108330000290F0F743FB044625492046F0F790F8F9
:1083400006460021FFF73AF82CE01848407A5528F5
:1083500003D1202000F0FAF802E0A02000F0F6F8A7
:108360000E201349087008460078F7F73FFB1149C3
:10837000086008460068059003210598FFF71EF87D
:1083800010E00E21032000F0ABF80E21042000F0D5
:10839000A7F80A21052000F0A3F80421062000F028
:1083A0009FF800BF00BF07B0F0BD0000AA2C00205E
:1083B0009B070020A80700200050C3470000F040A2
:1083C00000408F40000039C0000039400000C84222
:1083D00000401C461249087012490978104A127868
:1083E00091421BD00E4909780E4A117001210E4AA4
:1083F0001170002809D00A4A11700C49097804222A
:108400009143091D094A117008E00021044A1170C6
:108410000649097804229143044A1170704700000C
:108420003D0400203E0400203F04002040040020C2
:1084300001210C4A1170002809D00B4A11700B4918
:10844000097849084900491C084A117008E00021D0
:10845000054A11700549097849084900034A117015
:10846000704700003F0400203B040020400400202F
:1084700010B501201749087017491848EFF742FF57
:108480000821002000F02CF80821012000F028F835
:108490000821022000F024F80821032000F020F831
:1084A0000821042000F01CF80821052000F018F82D
:1084B0000821062000F014F80821072000F010F829
:1084C0000821084600F00CF80821092000F008F8FF
:1084D00010BD00003F04002040040020FFFFFF0FFC
:1084E0000A280EDA01228240064B1B881A43054BEC
:1084F0001A80142902DA044A115402E01322024BB2
:108500001A54704736040020BF1D002001210C4A78
:108510001170002809D00B4A11700B49097802220A
:108520009143891C084A117008E00021054A117026
:108530000549097802229143034A117070470000EF
:108540003F0400203C0400204004002070B5044695
:1085500001204649087046480078002807D140228B
:108560002146914308464349EFF7CCFE09E04048D5
:108570000078012805D14021214308463D49EFF705
:10858000C1FE3D480078002809D03A48EFF7A2FE26
:108590001021084305463749EFF7B4FE08E0354897
:1085A000EFF798FE1021884305463249EFF7AAFEFF
:1085B00032480078002809D02E48EFF78BFE0821BA
:1085C000084305462B49EFF79DFE08E02948EFF7E1
:1085D00081FE0821884305462649EFF793FE284887
:1085E0000078002809D02348EFF774FE01210843E2
:1085F00005462049EFF786FE08E01E48EFF76AFEC1
:1086000045086D001B492846EFF77CFE1D480078A1
:10861000002809D01748EFF75DFE02210843054600
:108620001449EFF76FFE08E01248EFF753FE0221FE
:10863000884305460F49EFF765FE13480078002888
:1086400009D00C48EFF746FE0421084305460949C6
:10865000EFF758FE08E00748EFF73CFE0421884397
:1086600005460449EFF74EFE70BD00003F040020B0
:108670003804002040040020390400203A0400207F
:108680003B0400203C0400203D04002010B59E481F
:10869000007800281CD101209B490870FCF784FC5D
:1086A0009A4988420AD104209949087001209949C1
:1086B000087008460078FFF71FFD23E10120944968
:1086C00008709449087008460078FEF7BDFF19E16C
:1086D0000220FDF72DFE002834D000208E490870BE
:1086E0000220FDF739FE8A480078042810D1894815
:1086F000007803280CD101208549087000208549A5
:108700000870FEF7FDFA8248007800F027F9F9E0DA
:108710007F4800780428D0D003217D480078EFF707
:108720000FFDC8B27A49087008460078401C0870EE
:10873000002078490870FEF7E3FA7548007800F0E9
:108740000DF9DFE00120FDF7F3FD00285AD00020ED
:1087500071490870FEF7D4FA0120FDF7FDFD6C4861
:10876000007801280FD105216A480078EFF7E8FC6E
:10877000C8B26849087008460078401C087008466E
:108780000078FEF761FF6248007802280FD10E21C1
:1087900060480078EFF7D4FCC8B25E49087008461C
:1087A0000078401C087008460078FFF745F85848E4
:1087B0000078032811D157490878C10F09184910CA
:1087C0004900411A534A117010460078401C114666
:1087D000087008460078FFF7DDFB4D480078042854
:1087E00095D106214B480078EFF7AAFCC8B2494959
:1087F000087008460078401C087008460078FFF7AB
:108800007BFC7FE00420FDF793FD002815D00020BD
:10881000414908700420FDF79FFD3D480078042879
:1088200070D0FEF76DFA0120394908703949087097
:1088300008460078FEF708FF64E00820FDF778FDA1
:10884000002819D0002034490870FEF759FA082092
:10885000FDF782FD04202E49087000202D49087084
:108860002B48007800F07AF800F034F980210843B2
:108870000446FFF76BFE45E01120F6F723F90028C8
:1088800012D0002024490870FEF73AFA1120F6F7BA
:108890002BF901201E49087005201E490870084662
:1088A0000078FEF7D1FE2DE00020F6F70BF9002846
:1088B00012D0002018490870FEF722FA0020F6F7BF
:1088C00013F9042012490870012012490870084663
:1088D0000078FFF711FC15E01020F6F7F3F80028F8
:1088E00010D000200C490870FEF70AFA1020F6F7A5
:1088F000FBF8012006490870064908700846007810
:10890000FEF7A2FE10BD00008E0700208D7C6B5A82
:108910008F070020900700208D07002001210C4ABE
:108920001170002809D00B4A11700B4909780822F0
:1089300091430831084A117008E00021054A11707E
:108940000549097808229143034A117070470000D5
:108950003F0400203A0400204004002070B5044683
:10896000FEF7CEF9002C17DD052C15DA00F0B2F871
:108970000546FFF7EBFD12210320FFF7B1FD0A21A9
:108980000420FFF7ADFD21460520FFF7A9FD1221C8
:108990000620FFF7A5FD0FE00E210320FFF7A0FD45
:1089A0000E210420FFF79CFD12210520FFF798FD02
:1089B0000A210620FFF794FD70BD000010B5214884
:1089C0000078002802D0012836D123E01E48007824
:1089D000012803D11D480078012807D11A480078E2
:1089E000022803D018480078032807D13C21012031
:1089F00005F0CAFF0120134908700AE01248007808
:108A0000042806D11249012005F0BEFF01200D49BE
:108A1000087015E0012005F011FE00280BD101209F
:108A2000094908700949087008460078FEF70CFEED
:108A300000200449087003E000200249087000BFCC
:108A400000BF10BD8D0700208F0700209007002079
:108A5000302A000001210C4A1170012809D10B4A6B
:108A600011700B490978402291434031084A117036
:108A700008E00021054A1170054909784022914318
:108A8000034A1170704700003F04002038040020A2
:108A90004004002001210C4A1170002809D00B4A23
:108AA00011700B490978102291431031084A117056
:108AB00008E00021054A1170054909781022914308
:108AC000034A1170704700003F0400203904002061
:108AD0004004002010B50248EFF7FCFB10BD000079
:108AE0004004002010B509210020FCF7C3FD0A2135
:108AF0000020FCF7BFFD0B210020FCF7BBFD0C2183
:108B00000020FCF7B7FD04218020FCF7B3FD052110
:108B10008020FCF7AFFD00214020FCF7ABFD0121D8
:108B20004020FCF7A7FD02214020FCF7A3FD0C210B
:108B300001200003FCF79EFD0D2101200003FCF73E
:108B400099FD0E2101200003FCF794FD0A2140202D
:108B5000FCF790FD0B214020FCF78CFD0C21402000
:108B6000FCF788FD0D214020FCF784FD0E214020FC
:108B7000FCF780FD0F214020FCF77CFD0821C02080
:108B8000FCF778FD0921C020FCF774FD0A21C02004
:108B9000FCF770FD0B21C020FCF76CFD0621802046
:108BA000FCF768FD07218020FCF764FD0821802088
:108BB000FCF760FD09218020FCF75CFD0821002006
:108BC000FCF758FD03214020FCF754FD0421402010
:108BD000FCF750FD05214020FCF74CFD062140200C
:108BE000FCF748FD10BD000007480078002809D1B7
:108BF00006480078002805D105480088002801D1E2
:108C0000012070470020FCE7340400203F040020CE
:108C1000360400200D480078022805D10C48007861
:108C2000022801D10020704708480078042805D1A7
:108C300007480078002801D00020F4E705480078B4
:108C4000002801D00020EEE70120ECE78F0700208C
:108C5000900700208C0700201FB5082102A80CF007
:108C60009DFE082168460CF099FEFFF73BFF0121AD
:108C7000162008F0E7FE2E480090001401900F2106
:108C8000490501988843019001210903019888430F
:108C90000190019800090001019049000198884362
:108CA0000190490001988843019049000198884348
:108CB00001904900019888430190890001988843F8
:108CC0000190490001988843019049000198884328
:108CD0000190684600F0D8FD012168460172032129
:108CE000417200218172C17203210173012141731C
:108CF000002181730121C17302A800F067FD00F01B
:108D000057FD00200B4908700B4908800B4908707B
:108D10000B4908700B4908700B4908700B49087023
:108D20000B4908700B4908700B49EFF7EBFA1FBDB0
:108D30000000FFFF34040020360400203804002027
:108D4000390400203A0400203B0400203C040020A9
:108D50003D0400203F0400204004002010B5002006
:108D6000154908701549087015490870FCF71CF979
:108D70001449884206D10420134908700120134980
:108D8000087004E0012010490870104908700120A3
:108D90000F49087000200F4908700F4908700F49EB
:108DA00008700F49087001200E49087000200E4914
:108DB00008600E49086010BD8C0700208D07002058
:108DC0008E0700208D7C6B5A8F07002090070020B3
:108DD00091070020920700209307002094070020AD
:108DE00096070020950700209C070020A807002078
:108DF00010B5022005F022FC002814D10121022028
:108E000005F0C2FDFEF732FAFFF7D8FD00F012FCC4
:108E1000F5F792F8012803D10020FFF7DBFA02E012
:108E20000120FFF7D7FAFFF731FC10BD10B5FE485F
:108E30000078002806D0012814D002287ED003280C
:108E40007DD1FFE2F9480078002803D1F848008876
:108E5000002806D00120F449087009F0BBF9F54953
:108E60000860D4E3F1480078002869D0F24800781F
:108E7000C107C90FF14840788006C00F81420BD06E
:108E8000EE48407820218843EB49097849012022A7
:108E900011400843E9494870E74800788007C10F4E
:108EA000E64840780007C00F81420DD0E348407883
:108EB00008218843E04909788907C90FC9000822B9
:108EC00011400843DD494870DB4800784007C10F76
:108ED000DA48203080784007C00F81420FD0D74851
:108EE0002030807804218843D34909784907C90F85
:108EF0008900042211400843D04920318870CE48AF
:108F000000780007C10FCD4840784007C00F81426C
:108F10000DD0CA48407804218843C7490978090719
:108F2000C90F8900042211400843C4494870C2484F
:108F30000078C006C00FC149097B02E07EE265E30C
:108F4000AAE18907C90F88420DD0BC48007B0221E5
:108F50008843B9490978C906C90F4900022211405E
:108F60000843B6490873B44800788006C00FB34977
:108F700009798907C90F88420DD0B04800790221CC
:108F80008843AD4909788906C90F4900022211407A
:108F90000843AA490871A84800784006C00FA749AD
:108FA000097A8907C90F88420DD0A448007A0221A6
:108FB0008843A14909784906C90F49000222114096
:108FC00008439E4908729C480078C0099B49097A69
:108FD0004907C90F88420DD09848007A0421884378
:108FE000954909780906C90F8900042211400843F0
:108FF00092490872904840788007C00F8F490978DD
:109000008907C90F88420DD08C4800780221884317
:10901000894949788907C90F49000222114008434C
:1090200086490870844840784007C00F8349097812
:109030004907C90F88420DD0804800780421884331
:109040007D4949784907C90F890004221140084326
:109050007A490870784840780007C00F7749097945
:109060004907C90F88420DD074480079042188430C
:10907000714949780907C90F890004221140084342
:109080006E4908716C4880788007C10F6B48407842
:10909000C007C00F81420AD06848407840084000AD
:1090A000654989788907C90F08436449487062484F
:1090B00080784007C00F6149097BC907C90F884202
:1090C0000AD05E48007B400840005B498978490728
:1090D000C90F084359490873574880780007C00FE3
:1090E0005649097AC907C90F88420AD05348007AFD
:1090F00040084000504989780907C90F08434F4983
:1091000008724D488078C006C00F4C490979C907DC
:10911000C90F88420AD049480079400840004649B2
:109120008978C906C90F08434449087142488078C4
:109130008006C00F41490978C907C90F88420AD083
:109140003E480078400840003B4989788906C90FAD
:1091500008433A490870384880784006C00F3749BC
:1091600009784906C90F88420DD03448007840215B
:109170008843314989784906C90F89014022114045
:1091800008432E4908702C488078C1092B482030AC
:109190004078C00981420FD0284820304078802193
:1091A0008843254989780906C90FC90180221140E1
:1091B00008432249203148701F48C078C107C90FB1
:1091C0001E48203040788006C00F81420DD01B48D9
:1091D00020304078202188431749C978490120224E
:1091E000114008431549203148701348C078800762
:1091F000C00F12490978C906C90F88420DD00F481F
:109200000078102188430C49C9788907C90F0901E2
:10921000102211400843094908700748C0784007E8
:10922000C00F0649097B0BE0340400203F040020F6
:10923000360400204404002040040020405C00402C
:109240004907C90F88420DD0F248007B04218843AA
:10925000F149C9784907C90F890004221140084320
:10926000EC490873EC48C0780007C10FE948407822
:10927000C00981420DD0E748407880218843E64903
:10928000C9780907C90FC901802211400843E14983
:1092900048700020E1490870E148008800287DD02E
:1092A000DF480078C007C00F00280DD0DC480088D8
:1092B00040084000DA4908800020FDF757FDD949F1
:1092C00008780021FDF708FED548008802210840F3
:1092D00000280CD0D24800888843D149088001205A
:1092E000FDF744FDCF4948780121FDF7F5FDCC4855
:1092F00000880421084000280CD0C9480088884311
:10930000C74908800220FDF731FDC649887802214F
:10931000FDF7E2FDC24800880821084000280CD073
:10932000BF4800888843BE4908800320FDF71EFD22
:10933000BC49C8780321FDF7CFFDB948008810214A
:10934000084000280CD0B64800888843B4490880FB
:109350000420FDF70BFDB34908790421FDF7BCFD9E
:10936000AF4800882021084000280CD0AC48008875
:109370008843AB4908800520FDF7F8FCA9494879E6
:109380000521FDF7A9FDA6480088402108400028D6
:109390000ED0A34800888843A14900E046E0088039
:1093A0000620FDF7E3FC9F4988790621FDF794FD2F
:1093B0009B4800888021084000280CD098480088ED
:1093C0008843974908800720FDF7D0FC9549C87964
:1093D0000721FDF781FD92480088FF2101310840F7
:1093E00000280CD08E48008888438D4908800820CA
:1093F000FDF7BCFC8B49087A0821FDF76DFD884814
:10940000008801214902084000280CD084480088C7
:109410008843834908800920FDF7A8FC8149487AE0
:109420000921FDF759FD00207D49088002207E4971
:10943000087008F0CFFE7D490860E8E003207A4913
:109440000870E4E074480078C107C90F714840789B
:109450008006C00F81427DD16F4800788007C10F20
:109460006C4840780007C00F8142F4D16A48007808
:109470004007C10F6748203080784007C00F814205
:10948000E9D1654800780007C10F6248407840077D
:10949000C00F81425ED160480078C006C00F5D49B0
:1094A000097B8907C90F884254D15B480078800640
:1094B000C00F584909798907C90F88424AD15648CF
:1094C00000784006C00F5349097A8907C90F8842BE
:1094D00040D151480078C0094E49097A4907C90F5F
:1094E000884237D14C4840788007C00F49490978F5
:1094F0008907C90F88422DD1474840784007C00FDF
:10950000444909784907C90F884278D142484078D0
:109510000007C00F3F4909794907C90F88426ED13A
:109520003D4880788007C10F3A484078C007C00F97
:10953000814264D1384880784007C00F3549097BA3
:10954000C907C90F88425AD1334880780007C00F35
:10955000304900E053E0097AC907C90F88424ED16B
:109560002D488078C006C00F2A490979C907C90F5C
:10957000884244D1284880788006C00F2549097860
:10958000C907C90F88423AD1234880784006C00FE6
:10959000204909784906C90F884230D11E48807891
:1095A000C1091C4820304078C009814227D11A489F
:1095B000C078C107C90F1748203040788006C00F17
:1095C00081421CD11448C0788007C00F1149097826
:1095D000C906C90F884212D10F48C0784007C00F92
:1095E0000C49097B4907C90F884208D10A48C0784D
:1095F0000007C10F07484078C009814202D001200E
:109600000649087000200849087000E000BF00BF4C
:1096100010BD0000405C0040400400203F040020DA
:1096200036040020BF1D0020340400204404002024
:109630007047000010B52848007801280FD127484E
:10964000007800280BD026480078F6F7E3F8254983
:109650000968884203D021480078FDF7F5FF1E48CD
:10966000007802280FD11D48007800280BD01E4832
:109670000078F6F7EFF81D490968884203D01748CB
:109680000078FEF7D9F81448007803280FD1134862
:10969000007800280BD016480078F6F75BF91549DA
:1096A0000968884203D00D480078FEF773FC0A4829
:1096B000007804280FD10948007800280BD00E4804
:1096C0000078F6F793F90D490968884203D00348FA
:1096D0000078FEF711FD10BD8F07002090070020D5
:1096E000980700209C07002099070020A007002071
:1096F0009A070020A40700209B070020A80700204D
:109700007047000070B5049C8DB2002D05D0274D28
:109710002D688EB23543254E356095B2002D05D0AB
:10972000224D6D6896B23543204E75609DB2002D76
:1097300005D01E4DAD689EB235431C4EB560A5B236
:10974000002D05D0194DED68A6B23543174EF560D2
:109750000D0C2D04002D06D0144D2D6A0E0C360371
:109760003543124E3562150C2D04002D06D00F4DD9
:109770006D6A160C360335430C4E75621D0C2D04B4
:10978000002D06D0094DAD6A1E0C36033543074E39
:10979000B562250C2D04002D06D0044DED6A260C73
:1097A00036033543014EF56270BD0000405C004059
:1097B00000210549002004E000220A60091D421C26
:1097C000D0B21028F8DB7047405C00402D49096892
:1097D0000722520291430278520207235B021A4089
:1097E0001143284A116011460968DA109143427802
:1097F0009201DB101A401143224A11601146096898
:10980000202291438278520120231A4011431D4A9D
:1098100011601146096818229143C278D2001823BA
:109820001A401143174A11601146096806229143F4
:109830000279520006231A401143124A1160114660
:1098400049689215914342791202FF2301331A406D
:1098500011430C4A51601146496880229143827934
:10986000D20180231A401143064A5160114609680B
:1098700049084900C279D207D20F1143014A116049
:1098800070470000005C0040024A0168D1604168F6
:1098900011617047005C004010B512F06BFF03E0EF
:1098A000F3F718F8F3F746F911F0DEFC0028F7D1CA
:1098B00000F084F900210148017210BDAA2C00209B
:1098C00010B5064800F035F8002805D0034800F030
:1098D00013F801200249087010BD0000000F00407D
:1098E000A404002010B5042008F0ECFE10BD10B553
:1098F000052008F0E7FE10BD10B504460022114611
:109900002046143005F042FD10BD70B505460C46EA
:109910002246002128460C3005F038FD70BD70B598
:1099200005460C4622460A2128460C3005F02EFD3D
:1099300070BD10B50446002120461030F6F784F8BB
:1099400010BD30B502467D23DB00D0680724E40259
:10995000A0430C78E4020725ED022C402043D060A0
:10996000D0683024A0434C78240130252C4020437B
:10997000D060D06801246402A0438C786402012581
:109980006D022C402043D060D0686C10A043CC788E
:1099900024026D102C402043D060D0680824A043DE
:1099A0000C79E40008252C402043D060D0680424C2
:1099B000A0434C79A40004252C402043D060D068FB
:1099C0000224A0438C79640002252C402043D060FF
:1099D00005E0D0680006C00F002800D004E018465B
:1099E0005C1EA3B20028F4D100BF002B01D10920D6
:1099F00030BD5068000C00040C89204350600020EA
:109A0000F6E700000348C06A400840000149C86208
:109A1000704700000024004010B5FFF7F3FF10BDB1
:109A200010B508F00EFC00287ED0F1F7C1FA00282E
:109A3000FAD004F059FE0028F6D003F007FB002806
:109A40007ED0F3F709F800287AD0042008F02EFF22
:109A5000002875D0052008F029FF002870D0FCF7F9
:109A600097FC00286CD0FFF7BFF8002868D0F9F702
:109A700073FD002864D0FCF78FFB002804D10F2071
:109A8000F5F720F801285BD1FCF78CFC002857D0B3
:109A9000F5F78EF9002804D10F20F5F713F8012807
:109AA0004ED1FFF7B7F800284AD0FBF783FA002819
:109AB00004D10F20F5F706F8012841D108F0CEF9BE
:109AC00000283DD008F0EAF8002804D10F20F4F770
:109AD000F9FF012834D100F0D3FF002804D10F2072
:109AE000F4F7F0FF01282BD1F1F7B8FE002804D1DC
:109AF0000F20F4F7E7FF012822D105F0C1FA002872
:109B000004D10F20F4F7DEFF012819D1042009F059
:109B100099F9002814D0052009F094F900280FD0F5
:109B2000042009F057FC00E00AE0002808D00520D6
:109B300009F050FC002803D0F2F7BAFE002801D14A
:109B4000002010BD0120FCE710B5024600230020D4
:109B5000002100BF0BE0074C0419237D002B04D02B
:109B6000072902DA53544C1CE1B2441CE0B20A2823
:109B7000F1DB10BD600E10001CB5072168460BF02C
:109B80000DFF01216846417081700021C170017193
:109B90004171012181716A460B2101200003FBF70D
:109BA00011FD03220B2101200003FBF7E1FC012240
:109BB00003210220F3F766FA1CBD00000748006885
:109BC00007490840884205D10448006880B203492B
:109BD000086002E00020014908607047247F0020EF
:109BE00000005AA50248006880B201490860704729
:109BF000247F00200548006805490840884203D1B9
